:020000022000DC
:1060000000000420A9AC02006DAE060003B4060037
:106010006DAE06006DAE06006DAE0600000000001D
:106020000000000000000000000000006DAE06004F
:106030006DAE0600000000006DAE06006DAE0600FD
:106040009DAB02006DAE060019B00200EDAE02007D
:10605000FDAE02006DAE0600318702006DAE060097
:106060006DAE0600F9AF020009B0020079AC020083
:106070006DAE06006DAE06006DAE06006DAE06009C
:1060800051B6020089AC02006DAE06006DAE06008E
:106090006DAE06006DAE06005DAF02006DAE06008F
:1060A0006DAE06006DAE06006DAE06006DAE06006C
:1060B0006DAE06006DAE060000000000000000009E
:1060C0006DAE06006DAE06006DAE06000DAF0200AF
:1060D00099AC02006DAE06006DAE060039B002004C
:1060E00029B002006DAE06006DAE060035AF0200AD
:0860F000000000006DAE060087
:1070000040F8044B40F8045B40F8046B40F8047B04
:1070100040F8048B40F8049B40F804AB40F804BBF4
:1070200040F804CB40F804DB6846704781F000412B
:1070300002E000BF83F0004330B54FEA41044FEA5D
:10704000430594EA050F08BF90EA020F1FBF54EAF8
:10705000000C55EA020C7FEA645C7FEA655C00F094
:10706000E2804FEA5454D4EB5555B8BF6D420CDD65
:107070002C4480EA020281EA030382EA000083EAE8
:10708000010180EA020281EA0303362D88BF30BD88
:1070900011F0004F4FEA01314FF4801C4CEA1131DE
:1070A00002D0404261EB410113F0004F4FEA03333D
:1070B0004CEA133302D0524263EB430394EA050FC8
:1070C00000F0A780A4F10104D5F1200E0DDB02FA37
:1070D0000EFC22FA05F2801841F1000103FA0EF2CB
:1070E000801843FA05F359410EE0A5F120050EF191
:1070F000200E012A03FA0EFC28BF4CF0020C43FAC2
:1071000005F3C01851EBE37101F0004507D54FF0CE
:10711000000EDCF1000C7EEB00006EEB0101B1F51E
:10712000801F1BD3B1F5001F0CD349085FEA300064
:107130004FEA3C0C04F101044FEA445212F5800F6F
:1071400080F09A80BCF1004F08BF5FEA500C50F10C
:10715000000041EB045141EA050130BD5FEA4C0CEF
:10716000404141EB0101013C28BFB1F5801FE9D24C
:1071700091F0000F04BF01460020B1FA81F308BF6F
:107180002033A3F10B03B3F120020CDA0C3208DD3B
:1071900002F1140CC2F10C0201FA0CF021FA02F116
:1071A0000CE002F11402D8BFC2F1200C01FA02F186
:1071B00020FA0CFCDCBF41EA0C019040E41AA2BFAB
:1071C00001EB0451294330BD6FEA04041F3C1CDA73
:1071D0000C340EDC04F11404C4F1200220FA04F093
:1071E00001FA02F340EA030021FA04F345EA03013D
:1071F00030BDC4F10C04C4F1200220FA02F001FAFF
:1072000004F340EA0300294630BD21FA04F0294680
:1072100030BD94F0000F83F4801306BF81F4801119
:107220000134013D4EE77FEA645C18BF7FEA655C8C
:1072300029D094EA050F08BF90EA020F05D054EA5E
:10724000000C04BF1946104630BD91EA030F1EBF63
:107250000021002030BD5FEA545C05D14000494167
:1072600028BF41F0004130BD14F580043CBF01F55A
:10727000801130BD01F0004545F0FE4141F4700140
:107280004FF0000030BD7FEA645C1ABF194610461B
:107290007FEA655C1CBF0B46024650EA013406BF1C
:1072A00052EA033591EA030F41F4002130BD00BFDB
:1072B00090F0000F04BF0021704730B54FF4806498
:1072C00004F132044FF000054FF0000150E700BF19
:1072D00090F0000F04BF0021704730B54FF4806478
:1072E00004F1320410F0004548BF40424FF0000165
:1072F0003EE700BF42004FEAE2014FEA31014FEAA8
:1073000002701FBF12F07F4393F07F4F81F06051F6
:10731000704732F07F4208BF704793F07F4F04BF41
:1073200041F40021704730B54FF4607401F000451E
:1073300021F000411CE700BF50EA010208BF70477E
:1073400030B54FF000050AE050EA010208BF70476F
:1073500030B511F0004502D5404261EB41014FF4D8
:10736000806404F132045FEA915C3FF4D8AE4FF0E0
:1073700003025FEADC0C18BF03325FEADC0C18BFC3
:10738000033202EBDC02C2F1200300FA03FC20FA14
:1073900002F001FA03FE40EA0E0021FA02F1144461
:1073A000BDE600BF4FEA4102B2F1E04324BFB3F5AE
:1073B000001CDCF1FE5C0DD901F0004C4FEAC0026C
:1073C0004CEA5070B2F1004F40EB830008BF20F050
:1073D0000100704711F0804F21D113F13872BCBF0A
:1073E00001F00040704741F480114FEA5252C2F15F
:1073F0001802C2F1200C10FA0CF320FA02F018BFA8
:1074000040F001004FEAC1234FEAD32303FA0CFCFA
:1074100040EA0C0023FA02F34FEA4303CCE77FEA89
:10742000625307D150EA01331EBF4FF0FE4040F4D3
:107430004000704701F0004040F0FE4040F4000082
:10744000704700BF80F0004002E000BF81F00041C3
:1074500042001FBF5FEA410392EA030F7FEA226CFA
:107460007FEA236C6AD04FEA1262D2EB1363C1BF8A
:10747000D218414048404140B8BF5B42192B88BFF9
:10748000704710F0004F40F4000020F07F4018BF1C
:10749000404211F0004F41F4000121F07F4118BF3C
:1074A000494292EA030F3FD0A2F1010241FA03FCE4
:1074B00010EB0C00C3F1200301FA03F100F00043CC
:1074C00002D5494260EB4000B0F5000F13D3B0F194
:1074D000807F06D340084FEA310102F10102FE2A03
:1074E00051D2B1F1004F40EBC25008BF20F0010073
:1074F00040EA03007047490040EB0000013A28BF12
:10750000B0F5000FEDD2B0FA80FCACF1080CB2EB94
:107510000C0200FA0CF0AABF00EBC2505242184312
:10752000BCBFD0401843704792F0000F81F40001B7
:1075300006BF80F400000132013BB5E74FEA41038A
:107540007FEA226C18BF7FEA236C21D092EA030FF6
:1075500004D092F0000F08BF0846704790EA010F70
:107560001CBF0020704712F07F4F04D1400028BF9D
:1075700040F00040704712F100723CBF00F500007F
:10758000704700F0004343F0FE4040F400007047B5
:107590007FEA226216BF08467FEA23630146420261
:1075A00006BF5FEA412390EA010F40F48000704774
:1075B0004FF0000304E000BF10F0004348BF40421A
:1075C0005FEA000C08BF704743F0964301464FF056
:1075D00000001CE050EA010208BF70474FF00003B2
:1075E0000AE000BF50EA010208BF704711F00043F3
:1075F00002D5404261EB41015FEA010C02BF8446C3
:107600000146002043F0B64308BFA3F18053A3F521
:107610000003BCFA8CF2083AA3EBC25310DB01FA68
:1076200002FC634400FA02FCC2F12002BCF1004FEC
:1076300020FA02F243EB020008BF20F0010070477D
:1076400002F1200201FA02FCC2F1200250EA4C00D1
:1076500021FA02F243EB020008BF20EADC70704717
:107660007BB972B90029BEBF00204FF0004106E08F
:1076700008BF00281CBF6FF000414FF0FF3000F042
:107680001DBBADF1080C6DE904CE002909DB002B10
:107690001ADB00F081F8DDF804E0DDE9022304B034
:1076A0007047404261EB4101002B1BDB00F074F896
:1076B000DDF804E0DDE9022304B0404261EB410162
:1076C000524263EB43037047524263EB430300F0C3
:1076D00063F8DDF804E0DDE9022304B0404261EB29
:1076E00041017047524263EB430300F055F8DDF867
:1076F00004E0DDE9022304B0524263EB4303704728
:1077000053B94AB9002908BF00281CBF4FF0FF3108
:107710004FF0FF3000F0D2BAADF1080C6DE904CEA5
:1077200000F03AF8DDF804E0DDE9022304B0704728
:1077300007EE900AF5EEC07AF1EE10FA01D400F0EF
:107740000BB8F1EE677A08B517EE900A00F004F86E
:10775000404261EB410108BDD0B5FFF7CBFD0C4BBA
:10776000002206460F4600F07FF900F0A9FA044611
:10777000FFF79EFD074B002200F076F902460B460C
:1077800030463946FFF756FC00F09AFA2146D0BD44
:107790000000F03D0000F0412DE9F047089D04464F
:1077A0008E46002B4DD18A42944669D9B2FA82F2B4
:1077B00052B101FA02F3C2F1200120FA01F10CFAF0
:1077C00002FC41EA030E94404FEA1C48210CBEFB28
:1077D000F8F61FFA8CF708FB16E341EA034306FBB1
:1077E00007F199420AD91CEB030306F1FF3080F040
:1077F0001F81994240F21C81023E63445B1AA4B28D
:10780000B3FBF8F008FB103344EA034400FB07F72E
:10781000A7420AD91CEB040400F1FF3380F00A816F
:10782000A74240F207816444023840EA0640E41B64
:1078300000261DB1D4400023C5E900433146BDE810
:10784000F0878B4209D9002D00F0EF800026C5E9B2
:10785000000130463146BDE8F087B3FA83F6002ECA
:107860004AD18B4202D3824200F2F980841A61EB42
:10787000030301209E46002DE0D0C5E9004EDDE760
:1078800002B9FFDEB2FA82F2002A40F09280A1EB48
:107890000C014FEA1C471FFA8CFE0126200CB1FB9D
:1078A000F7F307FB131140EA01410EFB03F0884296
:1078B00008D91CEB010103F1FF3802D2884200F223
:1078C000CB804346091AA4B2B1FBF7F007FB1011B5
:1078D00044EA01440EFB00FEA64508D91CEB040453
:1078E00000F1FF3102D2A64500F2BB800846A4EBAE
:1078F0000E0440EA03409CE7C6F12007B34022FA99
:1079000007FC4CEA030C20FA07F401FA06F31C43C7
:10791000F9404FEA1C4900FA06F3B1FBF9F8200CD4
:107920001FFA8CFE09FB181140EA014108FB0EF01A
:10793000884202FA06F20BD91CEB010108F1FF3A6A
:1079400080F08880884240F28580A8F10208614476
:10795000091AA4B2B1FBF9F009FB101144EA014184
:1079600000FB0EFE8E4508D91CEB010100F1FF342F
:107970006CD28E456AD90238614440EA0840A0FBC7
:107980000294A1EB0E01A142C846A64656D353D09D
:107990005DB1B3EB080261EB0E0101FA07F722FAC1
:1079A00006F3F1401F43C5E9007100263146BDE8EA
:1079B000F087C2F12003D8400CFA02FC21FA03F34D
:1079C000914001434FEA1C471FFA8CFEB3FBF7F0CE
:1079D00007FB10360B0C43EA064300FB0EF69E42F3
:1079E00004FA02F408D91CEB030300F1FF382FD28C
:1079F0009E422DD9023863449B1B89B2B3FBF7F634
:107A000007FB163341EA034106FB0EF38B4208D90C
:107A10001CEB010106F1FF3816D28B4214D9023E4D
:107A20006144C91A46EA004638E72E46284605E76B
:107A30000646E3E61846F8E64B45A9D2B9EB02083C
:107A400064EB0C0E0138A3E74646EAE7204694E7CC
:107A50004046D1E7D0467BE7023B614432E73046FF
:107A600009E76444023842E770B54FF0FF0C4CF46C
:107A7000E06C1CEA11541DBF1CEA135594EA0C0F6C
:107A800095EA0C0F00F0DEF82C4481EA030621EAA7
:107A90004C5123EA4C5350EA013518BF52EA0335E2
:107AA00041F4801143F4801338D0A0FB02CE4FF094
:107AB0000005E1FB02E506F00042E0FB03E54FF0C4
:107AC0000006E1FB03569CF0000F18BF4EF0010EBC
:107AD000A4F1FF04B6F5007F64F5407404D25FEAB8
:107AE0004E0E6D4146EB060642EAC62141EA55516B
:107AF0004FEAC52040EA5E504FEACE2EB4F1FD0CAD
:107B000088BFBCF5E06F1ED8BEF1004F08BF5FEA2A
:107B1000500E50F1000041EB045170BD06F00046DC
:107B200046EA010140EA020081EA0301B4EB5C0489
:107B3000C2BFD4EB0C0541EA045170BD41F4801181
:107B40004FF0000E013C00F3AB8014F1360FDEBFA6
:107B5000002001F0004170BDC4F10004203C35DA82
:107B60000C341BDC04F11404C4F1200500FA05F305
:107B700020FA04F001FA05F240EA020001F00042A6
:107B800021F0004110EBD37021FA04F642EB06011C
:107B90005EEA430E08BF20EAD37070BDC4F10C0446
:107BA000C4F1200500FA04F320FA05F001FA04F20A
:107BB00040EA020001F0004110EBD37041F10001F6
:107BC0005EEA430E08BF20EAD37070BDC4F1200501
:107BD00000FA05F24EEA020E20FA04F301FA05F269
:107BE00043EA020321FA04F001F0004121FA04F211
:107BF00020EA020000EBD3705EEA430E08BF20EAE1
:107C0000D37070BD94F0000F0FD101F0004640001A
:107C100041EB010111F4801F08BF013CF7D041EA9C
:107C2000060195F0000F18BF704703F000465200A0
:107C300043EB030313F4801F08BF013DF7D043EA71
:107C40000603704794EA0C0F0CEA135518BF95EA27
:107C50000C0F0CD050EA410618BF52EA4306D1D1AE
:107C600081EA030101F000414FF0000070BD50EACD
:107C7000410606BF1046194652EA430619D094EA57
:107C80000C0F02D150EA013613D195EA0C0F05D141
:107C900052EA03361CBF104619460AD181EA030195
:107CA00001F0004141F0FE4141F470014FF000004D
:107CB00070BD41F0FE4141F4780170BD704700BFD6
:107CC0004A0011D212F5001211D20DD56FF478735B
:107CD000B3EB62520ED44FEAC12343F0004343EAB0
:107CE000505323FA02F070474FF00000704750EAFB
:107CF000013002D14FF0FF3070474FF00000704765
:107D000030B5144685B019A3D3E90023FFF7F8FC7A
:107D10000546A5F16150A0F5351001A9A0F56070E8
:107D20003CF066FD9DF807309DF806200E491B04C7
:107D300043EA42539DF8082043EAC2239DF80920F4
:107D400043EA42139DF80A2043EA5203BDF8042097
:107D500025F00105A2F2BC7243EA4263A5FB0101D2
:107D6000236005B030BD00BF00CA9A3B00CA9A3BF1
:107D700000000000182A2DE9F74F0446C0F8002142
:107D800022D0202A23D0102A24D140F20A43A4F87A
:107D90000431204643F023FB0022034694F80551AA
:107DA000AA4201F1040103F1040315D3364EDFF8B2
:107DB000DCE000EB850394F804210132B5EB820F7F
:107DC0001CD303B0BDE8F08F40F20C63DFE740F650
:107DD0000E03DCE70023DAE711F8045C03F8045C27
:107DE00011F8035C03F8035C11F8025C03F8025C11
:107DF00011F8015C03F8015C0132CFE794F805212A
:107E0000B5FBF2FA02FB1A5913F8041C13F8038CA1
:107E100013F802CC13F8017C0192B9F1000F0AD1DA
:107E200016F808B016F80C8016F807C0775C1EF834
:107E30000A108BEA0101D4F80021202A08D1B9F1F7
:107E4000040F01BF715C16F8088016F80CC0F75DCE
:107E5000019AAA1A043310F8229000EB820281EAF8
:107E6000090103F8041C517888EA010803F8038C1F
:107E700091788CEA010C03F802CCD278574003F8D1
:107E8000017C013597E700BF025509004253090004
:107E90002DE9F04FDFF8A0C1614E624FDFF89CE1A1
:107EA000002901DCBDE8F08F436C5F4C1A4684FB6F
:107EB00002825E4CD0F84880254684FB0898A2EBED
:107EC000080252004264584C826C84FB028285FB9B
:107ED000038313445B008364036C554C1A4684FB94
:107EE000028205F1AF6505F5A435D0F84C809F35C9
:107EF00085FB0898A2EB080252000264C26C84FB66
:107F0000028285FB038313445B00C364C36B494C4B
:107F10001A4684FB0282D0F8508086FB0898A2EBB8
:107F200008025200C263026D84FB028286FB038357
:107F300013445B000365836B1A4687FB0282D0F80B
:107F400054808CFB0898A2EB080252008263426DB9
:107F500087FB02828CFB038313445B004365436B06
:107F60001A468EFB0282DFF8D880D0F8589088FB42
:107F700009A9A2EB090252004263826D8EFB0292B4
:107F800088FB039313445B008365036BDFF8B490B5
:107F90001A4689FB0282DFF8B080D0F85CA088FB2B
:107FA0000ABAA2EB0A0252000263C26D89FB02A266
:107FB00088FB039313445B00C365C36ADFF88C90AE
:107FC0001A4689FB0282DFF88880D0F860A088FB1F
:107FD0000ABAA2EB0A025200C262026E89FB02A236
:107FE00088FB039313445B000366836ADFF86490A5
:107FF0001A4689FB0282DFF86080D0F864A088FB13
:108000000ABAA2EB0A0252008262426E89FB02A205
:1080100088FB039313445B004366013948303FE714
:108020004A3FE3D7A740DD7DF053C26DAA0025BECD
:10803000E4EBDC70736E8D797611B7E8B7206D7F55
:108040002FFEE4F3407EE47FC7A3C1FA63B2FC7F56
:10805000C6BD2EFE94C6FF7F5DC286FF2DE9F04FA0
:10806000044685B0084643F0BAF98A4602460390B2
:108070002146002042F0CFFE231D019304F110039E
:1080800001260293039A25462146002311F8230076
:10809000334F385C01F823000133042BF6D1019BE8
:1080A00001318B42F1D1617963786170617A6171DC
:1080B000617B6172A17A6373A378A170A17BA372C3
:1080C000A379A171E17BA373E378E170E17AE173B5
:1080D000E179E172E3719AF80431B34239D095F84D
:1080E00000B095F80180AF78E9788BEA080087EA5C
:1080F000010380EA0309039359F01FFA8BEA000099
:1081000089EA0000287088EA070059F016FA039BF4
:1081100088EA000089EA00006870184659F00DFAF4
:10812000784089EA0000A8708BEA010059F005FA4E
:108130004840029B89EA000985F803900435AB4268
:10814000CDD13046214601360392F6B242F063FEAD
:1081500098E72146304605B0BDE8F04F42F05BBEDF
:10816000025509002DE9F04F594D8146884659487E
:1081700003F0030189B005EB811550F8211001913E
:1081800099101F298C46A8BF4FF01F0C1C290E46C2
:10819000A8BF1C266C68EB680292033626EAE676D6
:1081A00034410594AC680020344133410490069476
:1081B000079359F8046B484B1E4226F0004412D135
:1081C00008AB03EB840454F8103C002E40EA030093
:1081D000B8BF5B4248F8043B029B013B0293E8D1E5
:1081E00009B0BDE8F08F3D4B1E420AD1002955F879
:1081F0002440BABFCCF1000304FA03F344FA0CF3B1
:10820000E3E7374B1E4214D1103C364B019F53F825
:10821000243083FB0747ACF10304002C54DA64429A
:108220006FF0004343FA04FEBE45CEDB07FA04F3C9
:10823000CBE76304B3F1006FB6BF630500240424E9
:10824000B3F1005FBCBF9B000234274F274AB3F154
:10825000804FBCBF5B000134BB4207F14F4707F5BD
:10826000F21707F58267D8BF3A469346204F214A56
:10827000CCBFBE4696469A465A4682FB0ABADEF8FC
:10828000047057449A4687FB0ABADEF808705744D0
:108290009A4687FB0ABADEF80C70574487FB03A3A3
:1082A000154ADEF8107052F8242003923B4417461A
:1082B00083FB07E7FB00019F83FB07E70F4B53F8A6
:1082C0002440ACEB0404A8E747FA04F37DE700BFC1
:1082D0006061090050600900FCFFFF7FF0FFFF7F35
:1082E000C0FFFF7FA06009009979825A6321851041
:1082F000286009003C600900806009006060090096
:108300002DE9F74F00F5A0470023D0F854A087F8D7
:10831000B43D87F8AE3DB1F1000903624FF0FF3381
:1083200014BF4FF00C0B4FF0FF0B4362836D0BEB50
:108330000A029A42C4BFA3EB0A0303F1FF3B00F514
:10834000DA7600F15408036C04465A46314640463A
:1083500098478345054604D00623E3614FF0000AA1
:1083600011E0BAF1000F40F08480974905223046B1
:108370004DF0C1FB58B19549052230464DF0BBFB8D
:1083800028B10823E361504603B0BDE8F08F94F8AC
:10839000BB2194F8BA3194F8BEB103EB02232360F9
:1083A00094F8BD21A36094F8BC3103EB0223636011
:1083B000E360CBF302130133A361B9F1000F02D0E4
:1083C0004FF0010ADFE794F8BF3187F8B03D1BF0AA
:1083D000800F87F8AF9D50D00BF0070B0BF1010B0E
:1083E0004FF0030A05F5DA710AFA0BFA236C5246CC
:1083F00021444046984797F8B5CD0544BCF1010F9C
:1084000004F58D5000F114002DD8022202FA0BF26F
:108410002146024491F8C2314FEA930E91F8C131DE
:10842000DB08DB0243EA4E1391F8C3E143EADE03C3
:10843000BCF1000F01D05BBA9BB220F8023B824234
:1084400001F10301E6D14FF0030A0AFA0BFA0AF12F
:108450000D0A16F80A302C2B00F0BC803B2B0FD1F4
:108460000723E361ACE7524604F2C1114DF055FB1E
:10847000EDE7D1464FF0000AEBE74FF00D0AE8E7D1
:10848000212B40F0988006EB0A020AF10201537892
:10849000FE2B65D0FF2B1DD0012B5BD0F92B40F0BC
:1084A0009180735C042B13D1D17887F8AF1D50797C
:1084B000137903EB00230A204343012BD8BF642325
:1084C0002362C90744BF937987F8B13D0AF10801D7
:1084D0008A46BEE716F801A04B1CA5EB030B0AF178
:1084E0001F025A4514DB01F2B5115A4621443046A9
:1084F00000934DF03AFB009B0BF5DA7199440AF1B9
:108500002002236C21444046984700230BEB0005D2
:10851000BAF10B0F18D106EB030B2D49009352460D
:1085200058464DF0E8FA009B70B99BF80B20032ADF
:108530000AD19BF80C20012A01BF9BF80E109BF872
:108540000D2002EB012262620AEB0301BAF1000F77
:10855000C0D1BDE7735C4A1C9918002BFAD1B7E76C
:1085600016F801A04B1CA5EB030B0AF11F025A459C
:1085700014DB01F2B5115A462144304600934DF008
:10858000F4FA009B0BF5DA7199440AF12002236C8E
:1085900021444046984700230BEB0005A26B22B90B
:1085A00003EB0902A263A4F83CA00AEB0301BAF1B1
:1085B000000FD5D18CE7A16DA1EB09011F2901DCCA
:1085C0000723CAE60123C8E65A5E0900605E090077
:1085D0002856090006EB0A030AF10A0B99785A7823
:1085E00002EB012222611979DA7802EB0122626141
:1085F00099795A7902EB01222260197ADA7902EB31
:10860000012262605B7A87F8B33D1A063AD503F01F
:108610000703013305F5DA7103229A4000932144E0
:10862000236C01924046984797F8B51D019A05447E
:10863000012904F5A55000F1140059D8009B022728
:108640009F40A24407449AF8BF319A089AF8BE3175
:10865000DB08DB0243EA42139AF8C02143EAD20363
:1086600009B15BBA9BB220F8023B87420AF1030AC8
:10867000E9D1009A032393409B4404F5A0430122CF
:1086800083F8B42D16F80B30284A04F5A0470BF1F7
:10869000010187F8B23DD35CA3610023636341F21B
:1086A000B47A8D427FF78CAE4B1C16F801B0606B2C
:1086B0000093EA1A50449345204406EB03011FDC63
:1086C0005A464DF02AFA626B009B5A4462630BEBE8
:1086D0000301BBF1000FE4D14FF0010A8D4287F88E
:1086E000AEAD7FF76DAE636C4944404698474AE6AD
:1086F00006EB0B0100924DF010FA009A9344BCE790
:1087000000924DF00AFA009A616B236C1144616388
:108710005144ABEB02022144404600929847636B00
:10872000009A1A4462632946D3E700BF045F090038
:108730002DE9F04F00248DB0CDE90644634B644829
:108740006449012225461E6846B1D0F804631642EA
:1087500004D01D601E680396039E144304338B42AD
:108760004FEA4202EFD15A4BD3F87C218AB1002262
:10877000C3F87C21D3F87C310493049B4FF0A043D1
:1087800044F00044D3F810350693534BD3F810351A
:108790000793E3B2D3B1514F01260025344210D0E4
:1087A000AB0003F1804303F5C043D3F81005D3F8C1
:1087B000101557F8253023B1C1F30141C0F305204E
:1087C00098470135082D4FEA4606E7D1002C79DAA3
:1087D0000AAE00230A9373604FF0FF33CDE90833EC
:1087E000DFF8F8903E4F0025A84617F9013B5C1CC6
:1087F0004FD0C3F3C20103F00702DCB203F03F0A1B
:108800000CAB0B4413F8100CD040C00741D509EB5A
:108810000A00A40990F9280059F820B0BBF1000F14
:108820000CD1032C35D1012000FA02FC705C40EA27
:108830000C00705404E04FF00108D6E7032CF2D08E
:1088400005A80193CDF814A02EF00CF90599019B11
:1088500001F5E07113F8183C50F82110D340DB0704
:10886000C1F3014105D5022913D1032C0BD12146B7
:1088700004E003290DD1032C05D10221504654F008
:1088800033F90135EDB2BBF1000F02D0214650465D
:10889000D847B8F1000FCED0A5B14FF0A04306994C
:1088A000D3F8102503F540739142D3F8103502D167
:1088B0000799994206D006920A9ACDE907320B9B96
:1088C00009938FE70DB0BDE8F08F00BF0061004055
:1088D000006000402061004000030050B45A0120B5
:1088E0000C5B01202DE9F04FB1B00E46099302F563
:1088F0000863049300F13C0303930023CDE90133A3
:10890000DDF8E8B00592039B019AA3F13C07DBF880
:108910000030934229DC059B243603EB8203019A45
:108920000493DBF804309342A6F1240500F3208180
:1089300016460027DBF80830019A934200F30682BE
:108940000022019B1F2B40F35182029B002B00F061
:1089500061820023029A002A80F25782013B30464E
:10896000CBF81C3031B0BDE8F08F099BD3E90593FB
:1089700033B1DBF81430019A9342C8BF4FF00009BD
:10898000DBE903A3019ADBF818709342C8BF4FF0EC
:10899000000A049B062FA3F5086306937FDC0025DD
:1089A0000398C7F107070DF1500C06F124012B467F
:1089B00082683A41D21A43683B41551B9B1A51F8D1
:1089C000042DCCF824503A41B1424CF804390A60E5
:1089D000A0F10800ECD1159B5B1015930C9B0CA823
:1089E0005B100C931CF0FCFE15A81CF0F9FE59EA74
:1089F0000A0567D1DFF8F0C3DFF8E4A3B6462846DE
:108A00000DF15008D8F824305AF8042958F8041900
:108A100082FB0393A3EBA102DEF8009003EBA1031A
:108A20004EF8043BC9F100035CF8081B9B1A83FB5A
:108A3000014102EB81015CF8042C83FB0242069B9E
:108A4000049C43F820106FF003034343C9EB8202F8
:108A5000E250002381EAE173A3EBE173002182EA93
:108A6000E271A1EBE27120300B43B0F5907F45EA53
:108A70000305C7D13B463146019A069842F0F7F903
:108A8000029B284303430293019B01330193049B00
:108A900004330493039B48332436039333E7039B47
:108AA000002014AD0246A3F148079968891A5A6854
:108AB000083B081A521ABB42686245F80429F4D1EF
:108AC000002788E70DF1780852463046414602F00B
:108AD000D3FDC24B902000FB09302FAB089300253B
:108AE000BF4B079300F148092A460DF1500A079C35
:108AF000DAF8243054F804C95AF8041907948CFBA6
:108B000003E3C3EBA10E03EBA10346F8223050F8B8
:108B100022108EFB0131089C58F8223059F804CD00
:108B20000B4454F8041908949B008EFB0C4C069CD3
:108B300061444FEAC21C890044F80C306FF07F0496
:108B400004FB02FC049C44F80C104FF0000C83EA78
:108B5000E37CACEBE37C002381EAE173A3EBE173FC
:108B600001324CEA0303092A45EA0305BFD181E734
:108B7000DBE903A3019A9342C8BF4FF0000ADBF878
:108B80001830062B00F3DF80C3F107030393294657
:108B90003B4607F148001A68039C22411A605A6854
:108BA00022415A6051F8042B08332241834241F894
:108BB000042CF0D10CA938461CF09CFE12A9381DDB
:108BC0001CF098FE18A907F108001CF093FE52460D
:108BD0001EA9284602F050FD049A82490020069002
:108BE00002F5C0701EAB0DF130080DF138090B9085
:108BF00053F8040B0024800080EAE074A4EBE074D6
:108C000010609868079480004FF0000A80EAE07ACC
:108C1000AAEBE07AC2F8800151F8040BD8F80CC036
:108C200080FB0CEC586900240CEB800080EAE074B7
:108C3000A4EBE074C2F8000388680894D9F80CE04B
:108C4000CC46044684FB0E0E186A00240EEB80000E
:108C500080EAE074A4EBE074C2F880044869DCF8B0
:108C600000C00994A9F1040980FB0CEC51F8040C34
:108C7000D8F824E0044684FB0E0ED86AF4440CEBCA
:108C80008000002480EAE074A4EBE074C2F80006DF
:108C9000D8F800C0086A0A9408F1040880FB0CECBC
:108CA0008868D9F828E0044684FB0E0E986BF444DB
:108CB0000CEB80004FF0000C80EAE07CACEBE07C39
:108CC000079CC2F8800744EA0A0A089C0B984AEA03
:108CD000040A099C4AEA040A0A9C4AEA040A069C15
:108CE0004AEA0C0C803244EA0C04824206947FF477
:108CF0007FAF129B9B1046F8243C139B9B1046F8B9
:108D0000203C149B9B1046F81C3C18A9A6F11803A4
:108D100051F8042B921043F8042BB342F8D1039B73
:108D2000019A0498294642F0A2F8069B034318468C
:108D3000029B03430293019B01330193049B483739
:108D400024360433EBE50023039333E7DBE9032305
:108D5000019928468B42C8BF00221EA902F08CFC54
:108D6000019B019A43F3000A059B03EB820105F185
:108D700020031EA8A5F1040E4FF0000C02F001091B
:108D80001C46026892000A60B84682EAE278A8EBC4
:108D9000E27843688AEA83034B441A434CEA020CA4
:108DA000C1F880303A4683EAE372A2EBE372029B99
:108DB0004EF8047F42EA08021343A645029300F1ED
:108DC000080001F58071DCD1019BBCF1000F18BFD8
:108DD0001E46013324350193ACE500BF9C87090092
:108DE000005F0900BC880900E05F0900059B01994C
:108DF00003EB8101002341F823202033B3F5107FDA
:108E0000F9D1019B013301939BE5029A5200013392
:108E100002929FE52023A1E52DE9F04F04468DB095
:108E2000084642F0DCFA0D46024607EE900A21465B
:108E300095F8040141F0EFFF95F80461231D013E10
:108E4000099304F11003F6B20A93627A637B6273AA
:108E50006279627262786271A27A6370A378A2709A
:108E6000A27BA372A379A271E279A373E378E27083
:108E7000E27AE271E27BE272E37325462246002346
:108E800012F823105348415C02F823100133042BDD
:108E9000F6D1099B01329342F1D117EE902A214677
:108EA000304641F0B8FF002E00F0918095F800A008
:108EB000EB780793504658F040FB029058F03DFB8A
:108EC000039058F03AFB95F8019095F8028083469C
:108ED000484658F032FB024658F02FFB049058F0F9
:108EE0002CFB0746404658F028FB059058F025FB20
:108EF000069058F022FB079B019018460B9358F000
:108F00001CFB079058F019FB089058F016FB029BC9
:108F10001946039B81EA030C8BEA0C0C0499069B0F
:108F200082EA0C0C8BEA02024A4005997A404A40D8
:108F300001994A40089987EA0C0C83EA0C0C4A40D4
:108F4000019B0599424083EA0C0C8AEA02020B9BC2
:108F500088EA02025A406A70039A82EA0B027A4057
:108F600080EA0C0C4A40069989EA0C0C88EA0C0C41
:108F70004A40019983EA0C0C85F800C04A400799E1
:108F80004A4042408AEA020289EA02025340AB7038
:108F9000029B019983EA0B0B049B83EA0B0B87EA84
:108FA0000B07079B79405940089B594048408AEA83
:108FB000000A89EA0A090A9B88EA090885F80380F9
:108FC0000435AB427FF472AF013EF6B23DE70DB01F
:108FD000BDE8F08F025409002DE9F04F2DED028B12
:108FE0000D4608EE103AA9B016468346002801F057
:108FF000B785096841F01CFB031E0493C1F2B485D8
:109000002B6803442B60DBF80080B8F1000F0BD114
:10901000584618EE101A42F0F8F96FF0060029B021
:10902000BDEC028BBDE8F08FDBF80470002FEFD0B1
:1090300098F8004098F81C20002C3AD1032A4FF0F1
:1090400009010CBF4FF011094FF0200920A8CDE90C
:109050002034CDE9224958F0FDF9386098F81C30E9
:10906000032B0CBF0521032120A858F0F3F907F1C9
:10907000080A7860DBF8BC379C420CDB4FF0000A32
:10908000DBF8C4379A4580F2C580902303FB0A744D
:10909000002305938FE00AF11003012120A8059316
:1090A00058F0D8F9059B4AF8040B9A45F5D10134DC
:1090B000E0E7032A4FF008010CBF4FF009094FF019
:1090C0001109209320A80023CDE92133CDF88C90FD
:1090D00058F0C0F9386098F81C30032B0CBF012100
:1090E000022120A858F0B6F97860C7E70C2120A823
:1090F00058F0B0F90921A06220A858F0ABF9082176
:10910000E06220A858F0A6F9206398F80030002B00
:109110000CBF0421092120A858F09CF901216063AB
:1091200020A858F097F9A063002855D0022120A864
:1091300058F090F90121E06320A858F08BF905213F
:10914000206420A858F086F90521606420A858F012
:1091500081F90023E364A064032120A858F07AF980
:109160000321206520A858F075F90321606520A827
:1091700058F070F9E36BA0652BBBC4E90A33636355
:10918000E36DC3F11403236698F80030002B3FD140
:10919000012120A858F05EF96066012120A858F04E
:1091A00059F90121A06620A858F054F9059BE06602
:1091B000013305934834DBF8BC37059A9A4295DBB6
:1091C0000AF1010A5CE7022B04D1236C13B90823CE
:1091D000E365D5E70723FBE7C4E90F00052120A8D5
:1091E00058F038F90521606420A858F033F90521BA
:1091F000A06420A858F02EF90421E06420A858F0BB
:1092000029F90321E06520A858F024F92066BBE77E
:109210000020C1E73B68CBF8D8372B684B442B6064
:10922000049B03EB090433681B1B3360DBF8B8278E
:10923000DBF8B03772B1002B59D1DBF8CC2733689B
:109240009A4264DD584618EE101A42F0DEF84FF0EC
:10925000FF30E4E6002B4AD10123CBF8B037D5F834
:109260000080D6F800A0A8EB0404474651463846D3
:1092700042F0DFF8002807EB000324DB395C22789A
:1092800091421BD159786278914217D1A1789A788E
:109290004A4012F0FC0F11D18C0748BF03F1FF3395
:1092A000A3EB0803002BCBF8B4370FDA584618EEBF
:1092B000101A42F0AAF86FF00200B0E60330DF1C8B
:1092C000AAEB000AD2E74FF0FF33EBE7049ADBF892
:1092D000C8171A441346DBF8C0274B445343DBF846
:1092E000C427DB004A4393FBF2F3CBF8B837DBF833
:1092F0000030DBF8B4273BB15B69003B18BF0123AA
:109300001344CBF8CC3798E74FF0FF33F8E7DBF89E
:10931000DC07DBF8D8370BF11C01984209913FDBE1
:10932000C11A1A46099B194418464CF01EFC099BA9
:10933000DBF8D807DBF8CC27296818444CF0EDFBA4
:10934000DBF8CC17DBF8D8270A44CBF8DC272B68EE
:109350000B442B603368DBF8CC279B1A3360DBF8B7
:10936000DC37DB000C930BF5FC63149300230593AF
:1093700028230F93002307930493DBF8C437049A40
:109380009A4281F2F583902353431993059B0A93E4
:109390000F9B1393149B1893002308939A46D7E2CC
:1093A000099B2968034418464CF0B7FBDBF8CC173F
:1093B000DBF8DC270A44CBF8DC272B680B442B6056
:1093C0003368DBF8CC279B1A584618EE101A336026
:1093D00042F01BF86FF0010021E6002D00F07681CD
:1093E000DBF804300693002B00F07081DBF80840B6
:1093F000002C00F06B81099B20930023CDE92133E1
:10940000079A0C9B9A18D31D48BF02F10E03DB107C
:109410002393079B1BB1194620A858F01BF82A7804
:10942000002A40F04281049990234B43482101FBDC
:109430000A3306990B44A849586B11F8106001EBE8
:1094400040014F78D96B022940F08D80D3F84080DD
:10945000B8F1000F0ED00A9B154604EB0308314605
:1094600020A857F0F7FF0135082D08F8010BF6D1B9
:109470004FF00308089B059A08EB480513441D4468
:1094800025440DF180093146484657F0E3FF314647
:10949000E875484657F0DEFF31462876484657F0D3
:1094A000D9FF08F10108B8F1060F687605F1030548
:1094B000E9D10A9BE5183946484657F0CBFF3946B3
:1094C00085F82900484657F0C5FF394685F82A0037
:1094D000484657F0BFFF08F10108B8F10C0F85F8B6
:1094E0002B0005F10305E6D1049B7C225A433E2361
:1094F00003FB0A221444002384F83B30A387049A18
:1095000090235343482202FB0A33069A1A44936A73
:10951000189A1360209A099BD31A229AC2EBC302AD
:10952000D31002F007020D92079A18980D99C2EB1A
:10953000C3020A4450F8041B1890881A0690099830
:10954000184412900C98002BA0EB02021E9202DB32
:10955000884280F2C380584618EE101A41F055FF39
:109560006FF007005BE5049BBBB9089B049D1C449E
:10957000A1460DF180083146404657F06BFF01359A
:109580000B2D09F8010BF6D13946404657F062FF22
:1095900060550135152DF7D1B1E74FEA0A13069A48
:1095A000083302EB0308D558D5B1089B0599E2189A
:1095B0000139062312F8010B5054013BFAD1D8F8B7
:1095C0000430D3B90A9B062504EB0309314620A8D1
:1095D00057F040FF09F8050001350B2DF6D11FE0CB
:1095E0000A9B04EB0309314620A857F033FF0135ED
:1095F000062D09F8010BF6D1E1E7049D3E2303FB9C
:109600000AF37C20E21800FB053323449179997119
:10961000D179D971117A1972517A5972927A9A72F2
:10962000D8F808302BB3089B05990B3323440B2241
:109630000139013213F8010B5854102AF9D1D8F826
:109640000C3023B3089B05991033234410220139B1
:10965000013213F8010B5854152AF9D1049B7C22CE
:109660005A433E2303FB0A22144400236375A37567
:1096700045E70A9B0B2504EB0309394620A857F060
:10968000E9FE09F805000135102DF6D1D7E70A9B50
:10969000102504EB0308394620A857F0DBFE08F834
:1096A00005000135152DF6D1D8E7089B059A1398CA
:1096B00006999A1804F1F80301932B6A0093014468
:1096C0005346224420A801F08BFE18E7079B0D9318
:1096D0004FF0FF3328E700BFAE5E0900DBF8004023
:1096E000002C00F0D681DBF804300793002B00F04B
:1096F000D081DBF80830002B00F0CB81DBF80C3098
:109700001093002B00F0C581069B002BC0F2C18195
:10971000049A616B902353434820079A00FB0A3355
:1097200013449A6B002A00F03E81DA6B022A40F063
:109730003A811B6C002B40F01E81049A9023534306
:1097400000FB0A30079B18440322C36D013393FBCF
:10975000F2F301EB4301B1F92E2002EB42024FF488
:109760001071049890234343482000FB0A33079864
:1097700003444FF41069DC6A6300B3F5107FA8BF9F
:109780004FF410739342D4BF21932192109A0993FE
:1097900002EB8A021C9202F580528B42D4BF2293C4
:1097A00022912393099900232093C2F80012109A62
:1097B000119309FB0A22199B1B9220AA179240338E
:1097C0000D9A0E92C318129A0B921F93179B1C6846
:1097D000119B01331193179B53F8045F17932D1BB3
:1097E000002D40F38682069B002BC0F25281119A15
:1097F0001F9B0B9953F82260BF4B03EBC6031B79E9
:109800000C930E9B0C985B4213F007031EBF11F8DC
:10981000017BC3F1200207FA02F21B9F08BF1A4620
:1098200007EB8404002840F0D080231D002244F878
:10983000202043F8202002308542F7DC90460E9B22
:109840000B9A434402EBE30203F007030E93069BDB
:109850000B92A3EB08030693119B032BB6D1069B37
:10986000002B40F3C982049A0B99099D902353431E
:10987000482202FB0A33079A1A444FF00009D36EBC
:109880009E4A52F823009E4A52F823600E9B5B4288
:1098900013F007031EBF11F8014BC3F1200204FAB5
:1098A00002F21B9C04EB85040794069CC6F120067B
:1098B000A4EB0305099C0996924EC4F50F7430443D
:1098C00008BF1A464F4601340C90BC4200F3188280
:1098D0001C9B03F580530021D3F800020744C3F812
:1098E00000724FF41070109BB7F5107FC7F510721F
:1098F00000FB0A704FEA820203EB8000C8BF00221F
:109900004CF04BF9069A0E9B134403F007020792A2
:109910000B9A02EBE303199A48321992139A4832D0
:109920001392089A3E3208920A9A3E320A92129A8A
:109930009B1A00F1AE80129A1A4409920D9AC2EB5A
:10994000C303079A13441E9AD31A0C930AF1010A0F
:10995000DBF8BC37DBF800509A45FFF63EAD002D32
:1099600040F04E82584618EE101A41F04EFD6FF04E
:109970000900FFF754BB23785BB9049A9023534343
:1099800000FB0A30079B1844C36D013331F91320E3
:10999000E5E6B1F93620B1F93430D31AB1F90C202B
:1099A00002EB4302DBE6049B90205843482303FB71
:1099B0000A00079B1844C36D006E013331F9132070
:1099C0000344013331F91310CBE64F4F57F826C04B
:1099D0004E4F07EB4C0015900698A0EB03080C982F
:1099E000012840F0958037F81C6006F00F064FF014
:1099F000000EC6F12006B8F10F0F53DD0F46C3F17C
:109A0000180017F802CB49780CFA00F0C3F1100CDB
:109A100001FA0CF101430A431033A8F1100839464A
:109A200004F1080722FA06F0159C013034F8100002
:109A3000040B10F0F00F02FA04F2A3EB103318BF7E
:109A400002F00044C0F3031C1EBF520003F1FF33B9
:109A500044EA0C0C10F4706FC0F303241FBF03F131
:109A6000FF3302F000402043520008BF20467345F8
:109A70000FDB023D002D47E902C03C4637DCA3EB7B
:109A80000E039844069BA3EB0808B8F1000F80F280
:109A90003281584618EE101A41F0B7FC6FF00800FA
:109AA000FFF7BDBA08EB03000028F2DDB8F1000FA4
:109AB000C1BF11F8017BC3F1180C07FA0CF73A4348
:109AC000B8F1080FC1BF11F8017BC3F1100307FA09
:109AD00003F31A434FF00047431E47FA03F31A40BB
:109AE0004FF00B0E00F10B034FF0000898E70A2B24
:109AF00007F1080796DC7EE7F8640900048E090088
:109B0000FC8D09000C8E0900F865090078660900D3
:109B10000C98871E012FBCD8B848159F50F836C046
:109B2000002016900CF101001A90CCF120001D903D
:109B3000B8F10F0F2ADD8E46C3F118061EF8029BFE
:109B4000497809FA06F6C3F1100901FA09F131431F
:109B50000A431033A8F1100871460A2BE8DDB7F864
:109B600000E00EF00F0ECEF1200622FA06F60136C6
:109B700037F816605FEA16392FD107EB4607A3EBDB
:109B80000E0302FA0EF226463446E6E708EB030619
:109B9000002E7FF77EAFB8F1000FC1BF11F801EBC7
:109BA000C3F118090EFA09FE42EA0E02B8F1080FD5
:109BB000C1BF11F801EBC3F110030EFA03F31A430E
:109BC0004FF00040731E40FA03F30B201A4016902A
:109BD00006F10B034FF00008BFE7A3EB090302FAFD
:109BE00009F2C6F30319B9F10F0FC6F3032637467E
:109BF00027D10C98032827D11A9803EB080E002EC2
:109C000018BF0130704581463FF743AF9945AEEB31
:109C1000030857DCB8F1000F0ADA73464FF0004032
:109C20000EF1FF3E40FA0EFE02EA0E024FF000086F
:109C30001D9822FA00F909F10F09A3EB0C0302FAAF
:109C40000CF2B9F1000F05D002F0004E4EEA0909FE
:109C50005200013B0F2E22D10C98032844D11A98B0
:109C600003EB080E70453FF714AF1A989842AEEB1D
:109C7000030831DCB8F1000F09DA0EF1FF364FF0BE
:109C8000004040FA06F6734632404FF000081D9837
:109C900022FA00F70F37A3EB0C0302FA0CF227B1FC
:109CA00002F0004637435200013B16988342FFF60C
:109CB000F0AE2646023D002D46F8089B676015DD94
:109CC000159F61E711F8018BC3F1180008FA00F83D
:109CD00042EA0802083399E711F8016BC3F118074B
:109CE000BE4032430833C0E73746D9E7169A9B1A7D
:109CF000C7E64FF00008069B98457FF7A0ADC8E681
:109D00000F2D57DD0E46C3F1180016F802CB497827
:109D10000CFA00F0C3F1100C01FA0CF101430A43F4
:109D20001033103D3146079E1036099822FA00FC88
:109D30000C9810F80C004FEA101C02FA0CF210F00C
:109D40000808A3EB10131FBF02F0004803F1FF3314
:109D5000520048F0010810F0040E1FBF02F0004E40
:109D600003F1FF3352004EF0010E10F0020C1FBF42
:109D700002F0004C03F1FF3352004CF0010C10F0E4
:109D800001001FBF02F0004003F1FF3340F001006B
:109D900052004B45FFF69CAD0437A74246E9048EBE
:109DA00046E902C00796BFF690AD092B06F11006F2
:109DB000BBDC8AE5E81800287FF78AAD002DC1BF1B
:109DC00011F8016BC3F1180C06FA0CF63243082D9A
:109DD000C1BF11F8015BC3F1100305FA03F31A4385
:109DE0004FF00045431E45FA03F31A404FF00A09AD
:109DF00000F10A03002596E7002769E5F8640900E9
:109E0000DBF80470002F3FF4ADADDBF80890B9F13A
:109E1000000F3FF4A7ADDBF80C40002C3FF4A2ADDF
:109E2000DBF8101000293FF49DAD01F54673069351
:109E30000F9B00261F44059BCDE9206609EB030A12
:109E400004F59058069B089308F10808DBF8BC3726
:109E50009E42C0F2A5832B6A002B40F0BA832B6A86
:109E60005A0840F0F4832A6AD30714D504F58053C6
:109E70002E78D3F80012059B3E334B44521020A895
:109E8000002E40F02B84CDE90120069A0092204656
:109E90002A4640F037F92B6AA3B1209840F0CFFF53
:109EA00004F580540138C4F80802219840F0C7FF37
:109EB000D4E980239342B8BF1346C4E98033013804
:109EC000C4F80C020F9B049A06939023534300247A
:109ED0004FF012080893DBF8BC379C42C0F20B84A9
:109EE000049ADBF8C847544318EE102A5C4302EB8F
:109EF0004404DBF80C20002A00F02986DBF814204B
:109F00000A92002A00F02386DBF818200692002A25
:109F100000F01D86022B40F08D840A9B1093231DB8
:109F2000089300230E9302F500530B930E9B0B9A9C
:109F30000699109803F001030D930A9B03F58054D2
:109F40000025D4F8183B0093D2F800220D9B3FF077
:109F5000C5FDD4F81C3B0B9A069910980093D2F8D3
:109F600000220D9B803100F510603FF0B7FD0B9B88
:109F70000D99D3F800324FF4886202FB0133069A40
:109F800002EB83094FF0007452F82320D9F85C30BB
:109F90002F46C2FB07456FF07306C3FB06454FF023
:109FA0000072D9F88000D9F8DC103B46C0FB0723CB
:109FB000C1FB06234FF45578D9F80400D9F858109E
:109FC000C0FB0845A6F5D766C1FB0645D9F8840055
:109FD000D9F8D810C0FB0823C1FB062341F6D47E74
:109FE000D9F80800D9F85410C0FB0E457B4EC1FBD0
:109FF0000645D9F88800D9F8D410C0FB0E23C1FB60
:10A00000062346F2B86CD9F80C00D9F85010C0FB02
:10A010000C45734EC1FB0645D9F88C00D9F8D01019
:10A02000C0FB0C23C1FB06236E4FD9F81000D9F8F2
:10A030004C10C0FB07456C4EC1FB0645D9F890009B
:10A04000D9F8CC10C0FB0723C1FB0623D9F81400B4
:10A05000D9F84810C0FB0C4545F28406C1FB064503
:10A06000D9F89400D9F8C810C0FB0C23C1FB062313
:10A07000D9F81860D9F84410C6FB0E4540F22C7789
:10A08000C1FB0745D9F89860D9F8C410C6FB0E2368
:10A09000C1FB0723D9F81C60D9F84010C6FB08455E
:10A0A0007427C1FB0745D9F89C60D9F8C010C6FBDE
:10A0B000082316469846C1FB07680C2720464FF038
:10A0C000140A05FA07F345FA0AF520FA0AF040EAFD
:10A0D000030040F0BFFE089B23F8040C304608FA4A
:10A0E00007F348FA0AF820FA0AF040EA030040F0C1
:10A0F000B1FE089B09F5805423F8020C22684FF446
:10A10000D0764FF000730025C2FB06354FF000708B
:10A11000D4F880200021C2FB060141F67C0662686B
:10A12000C2FB0635D4F88420C2FB060149F2FC7656
:10A13000A268C2FB0635D4F88820C2FB06012B4E6C
:10A14000E268C2FB0635D4F88C20C2FB0601284E1B
:10A150002269C2FB0635D4F89020C2FB06016FF0DD
:10A16000B3066269C2FB0635D4F89420C2FB06012F
:10A170004FF41276A269C2FB0635D4F89820C2FBD0
:10A1800006016FF01306E269C2FB0635D4F89C2085
:10A190000446C2FB0641184605FA07F245FA0AF5DD
:10A1A00020FA0AF040EA020040F054FE089B98872B
:10A1B000204601FA07F341FA0AF120FA0AF040EAD0
:10A1C000030040F047FE089BDFF828A0D88704333F
:10A1D0001193089B043B12930EE000BF7CAFFFFF7E
:10A1E0003CB6FDFF78940400C44902004CE803002B
:10A1F0002464FFFFDC890900DAF840E0D9F80001A7
:10A20000D9F85C114FF000730022C0FB0E324FF002
:10A210000074DAF844500027C0FB0547C5F1000C74
:10A22000C1FB0C321393C1FB0E47D9F8DC31D9F8CE
:10A23000801116934FF000754FF00008C1FB0E58C7
:10A24000D9F880014FF0007103460026DAF8440087
:10A25000C3FB0016169BC3FB0C580B461699C1FB9B
:10A260000E361593DAF848E0D9F804C1D9F8580148
:10A27000139BCCFB0E32DAF84C10CCFB0147C1F13A
:10A28000000CC0FB0C321393C0FB0E47D9F8D83139
:10A29000D9F884111693C1FB0E58D9F88401159989
:10A2A0000346DAF84C00C3FB0016169BC3FB0C58A0
:10A2B0000B461699C1FB0E361593DAF850E0D9F823
:10A2C00008C1D9F85401139BCCFB0E32DAF85410B4
:10A2D000CCFB0147C1F1000CC0FB0C321393C0FB57
:10A2E0000E47D9F8D431D9F888111693C1FB0E580E
:10A2F000D9F8880115990346DAF85400C3FB001613
:10A30000169BC3FB0C580B461699C1FB0E361593D2
:10A31000DAF858E0D9F80CC1D9F85001139BCCFBFE
:10A320000E32DAF85C10CCFB0147C1F1000CC0FB27
:10A330000C321393C0FB0E47D9F8D031D9F88C11E9
:10A340001693C1FB0E58D9F88C0115990346DAF81B
:10A350005C00C3FB0016169BC3FB0C580B461699FA
:10A36000C1FB0E361593DAF860E0D9F810C1D9F8C0
:10A370004C01139BCCFB0E32DAF86410CCFB014786
:10A38000C1F1000CC0FB0C321393C0FB0E47D9F88F
:10A39000CC31D9F890111693C1FB0E58D9F8900121
:10A3A00015990346DAF86400C3FB0016169BC3FB3D
:10A3B0000C580B461699C1FB0E361593DAF868E077
:10A3C000D9F814C1D9F84801139BCCFB0E32DAF846
:10A3D0006C10CCFB0147C1F1000CC0FB0C32139395
:10A3E000C0FB0E47D9F8C831D9F894111693C1FBB8
:10A3F0000E58D9F8940115990346DAF86C00C3FB9E
:10A400000016169BC3FB0C580B461699C1FB0E3663
:10A410001593DAF870E0D9F818C1D9F84401139B04
:10A42000CCFB0E32DAF87410CCFB0147C1F1000C02
:10A43000C0FB0C321393C0FB0E47D9F8C431D9F8D6
:10A4400098111693C1FB0E58D9F898011599034637
:10A45000DAF87400C3FB0016169BC3FB0C580B46BE
:10A460001699C1FB0E361593DAF878E0D9F81CC1BD
:10A47000D9F84001139BCCFB0E32DAF87C10CCFBF0
:10A480000147C1F1000CC0FB0C3216972746169C01
:10A490002146C0FB0E711691D9F8C001D9F89C1164
:10A4A0001397C1FB0E58D9F89C4115992746DAF845
:10A4B0007C40C7FB0416C0FB0C58C0FB0E164FF0C7
:10A4C000140C18460C24674602FA04F342FA0CF204
:10A4D00020FA0CF040EA030040F0BCFC119B23F88A
:10A4E000040C28463D4608FA04F348FA07F820FA17
:10A4F00007F040EA030040F0ADFC119B169F23F8E3
:10A50000020C139807FA04F347FA05F720FA05F04E
:10A5100040EA030040F09EFC129BA3F87C00084632
:10A5200006FA04F346FA05F620FA05F040EA0300BD
:10A5300040F090FC129BA3F87E00119B0433119312
:10A54000129B043B1293B94B0AF1400A9A4509F554
:10A5500080797FF451AE0B9B0D9AD3F800329B1A91
:10A560000B9A03F00703C2F800320E9B01330E93DF
:10A57000109B80331093089B803308930E9B122B03
:10A580007FF4D4AC049B013304930F9B90330F935F
:10A59000059B7C330593149B08331493FEF7EDBEA3
:10A5A000089B00974FF41060CDE901A3A8F10802C1
:10A5B0002B4600FB06400A913FF084F9089B48F8BF
:10A5C000040B18330A990893013648370AF13E0AFA
:10A5D0003CE404F58053D3F80822002A04DDD3F8C4
:10A5E0000C22002A3FF73BACD3F80002904F002327
:10A5F0006FF0404607E054F82320B2F1404F1BDCD7
:10A6000044F8237001338342F5DB04F58053DFF80F
:10A6100020C2D3F80462002204F510636FF04047B3
:10A62000B242BFF61CAC1868B0F1404F0ADCC3F868
:10A6300000C001320433F3E7B2F1804FA8BF44F801
:10A640002360DFE7B0F1804FA8BF1F60F1E7DA07B2
:10A6500020D5D1F830236B6B9AB9D1F8442301325D
:10A6600033F912300022211F164617469446BB428A
:10A6700018DC209B33432093219B13432193FFF746
:10A68000F2BBD1F8402303EB4203B3F9303003EBC4
:10A690004303E7E704F58052D2E980318B42B8BF2B
:10A6A0000B46DFE751F8048FD1F8000908EB000EE4
:10A6B000A8EB0000C1F800E0C1F80009E0468EEA0E
:10A6C000EE78A8EBEE7846EA0806E64680EAE07EF9
:10A6D000AEEBE07E42EA0E020137C8E7CDE9022088
:10A6E00009F1F8020192069A009220462A463FF0AC
:10A6F00067FEFFF7D0BBDBF8002042B9584618EEE2
:10A70000101A40F082FE6FF00A00FEF788BCDBF8FA
:10A710000430002BF2D0DBF80C50002DEED0DBF82B
:10A7200014A0BAF1000FE9D0516B1278002A0CBFC7
:10A730000822062231F91260089996FBF8F64822A1
:10A7400002FB04121A44D16B022966D004F5906210
:10A7500055F8227040F226229742D7BF07372027AC
:10A7600097FBF8F701372097013F4FF4106909FB79
:10A7700004F905EB0900394605EB84050B930A90B3
:10A78000FDF786FB05F5805C08FB07F7DCF8001297
:10A79000089B0A980837B9420AEB840505F58055ED
:10A7A000B8BF3946CCF80012113191FBF8F1219174
:10A7B000D5F8002B22924827D5F8082B239207FBC7
:10A7C00004370B9BD5F8102B24921F444FF4906153
:10A7D0003A6C002A08BF00262596DCF8082226924B
:10A7E00020AA0092069A01FB04A1134401F590519E
:10A7F0000AEB0902FEF776F8C5F8000BFB6BC5F80B
:10A80000083B259BC5F8103B279BC5F8183B069BCA
:10A81000483301340693FFF75EBB176C1FB1771EF8
:10A8200020963FB2A1E720979FE700BF9C8D0900CB
:10A83000010000C0069B002503F500534034089337
:10A84000AA4605F001030B930A9B089A0A980699F9
:10A8500003F5805300EBC510D3F8183B0093D2F8F2
:10A8600000220B9B3FF03AF9089B0B99D3F800327A
:10A870004FF4886202FB0133069A02EB830752F819
:10A880002310FA6D4FF000735046C1FB0A306FF091
:10A890007301C2FB01304FF455797968BA6DC1FB81
:10A8A0000930B549C2FB013041F6D478B9687A6DF8
:10A8B000C1FB0830B149C2FB013046F2B86CF968FF
:10A8C0003A6DC1FB0C30AE49C2FB0130AD4A39696B
:10A8D000C1FB0230AC49FA6CC2FB01307969BA6C39
:10A8E000C1FB0C3045F28401C2FB0130B9697A6CBE
:10A8F000C1FB083040F22C71C2FB0130F9693A6C9F
:10A90000C1FB09307421C2FB01304FF00C08024634
:10A910004FF01409184602FA08F342FA09F220FA35
:10A9200009F040EA030040F095FA07F5805124F859
:10A93000400C0A684FF0007053464FF4D07CC2FBC5
:10A940000C0341F67C0C4A68C2FB0C0349F2FC7C08
:10A950008A68C2FB0C038D4ACE68C6FB02038C4A90
:10A960000E69C6FB02036FF0B30C4A69C2FB0C030D
:10A970004FF4127C8A69C2FB0C03CA696FF01301A1
:10A98000C2FB010303FA08F243FA09F320FA09F0C3
:10A9900040EA020040F05EFAA4F14003CDE90D4325
:10A9A000DFF8F48124F8200CD8F844E0D7F800212F
:10A9B000D7F85CC1D8F840104FF000705346C2FB86
:10A9C00001034FF00071D146C2FB0E19CEF1000217
:10A9D000CCFB0203D8F84020CCFB0219D8F84CC0BD
:10A9E000D7F804E1D7F85821D8F84860CEFB060321
:10A9F000CEFB0C19CCF1000CC2FB0C03C2FB0619F8
:10AA0000D8F854C0D7F808E1D7F85421D8F85060E6
:10AA1000CEFB0603CEFB0C19CCF1000CC2FB0C03E1
:10AA2000C2FB0619D8F85CC0D7F80CE1D7F8502162
:10AA3000D8F85860CEFB0603CEFB0C19CCF1000C05
:10AA4000C2FB0C03C2FB0619D8F864C0D7F810E1AA
:10AA5000D7F84C21D8F86060CEFB0603CEFB0C196A
:10AA6000CCF1000CC2FB0C03C2FB0619D8F86CC079
:10AA7000D7F814E1D7F84821D8F86860CEFB060370
:10AA8000CEFB0C19CCF1000CC2FB0C03C2FB061967
:10AA9000D8F874C0D7F818E1D7F84421D8F8706016
:10AAA000CEFB0603CEFB0C19CCF1000CC2FB0C0351
:10AAB000C2FB0619D8F87CC0D7F81CE1D7F84021B2
:10AAC000D8F87860CEFB0603CEFB0C19CCF1000C55
:10AAD000C2FB0C03C2FB06190C264FF0140C03FA40
:10AAE00006F243FA0CF320FA0CF040EA020040F0C0
:10AAF000B1F90E9B23F8020F4FF0140C0E93084689
:10AB000009FA06F349FA0CF920FA0CF040EA0300BE
:10AB100040F0A0F90D9B23F8020D0D931D4B08F199
:10AB20004008434507F580777FF43EAF089B0B9ABA
:10AB3000D3F8003201359B1A089A03F00703122D4F
:10AB4000C2F8003204F140047FF47BAE1AE55846A7
:10AB500018EE101A40F059FC6FF00B00FEF75FBAC8
:10AB60006FF00400FEF75BBA6FF00500FEF757BA0E
:10AB70000020FEF754BA00BFD4F8FFFF7CAFFFFF00
:10AB80003CB6FDFF78940400C44902004CE8030081
:10AB90002464FFFF9C8D0900DC89090010B54FF08B
:10ABA0008043D3F80443620707D54FF4847051F013
:10ABB000E5FF10B11E4B1B689847A30608D54FF45C
:10ABC0008A7051F0DBFF18B11A4B00201B689847C0
:10ABD000600608D54FF48C7051F0D0FF18B1154BBA
:10ABE00001201B689847210608D54FF48E7051F05C
:10ABF000C5FF18B1104B00201B689847E20508D527
:10AC00004FF4907051F0BAFF18B10B4B01201B6844
:10AC10009847A3050AD54FF4927051F0AFFF28B1C1
:10AC2000054BBDE810401B680220184710BD00BF4F
:10AC3000445C0120485C01204C5C0120DFED0A7A75
:10AC40009FED0A7ADFED0A6AA0EE277ADFED097A36
:10AC5000E7EE007AB7EE007AA0EE267A67EE807A09
:10AC600087EE870A704700BF6BD30DBCBA132FBDA8
:10AC7000AEE534BF75AA2A3E0248032200211BF02C
:10AC800049BF00BF00B000400248042201211BF070
:10AC900041BF00BF001001400248042202211BF006
:10ACA00039BF00BF0040024008B5834B8348DA1C1F
:10ACB000121AC11E22F00302994288BF0022804965
:10ACC0004AF02BFF7F4B8048DA1C121AC11E22F07B
:10ACD0000302994288BF002200214AF05EFF4FF034
:10ACE0008053D3F83021082A4ED14FF08042002102
:10ACF000C2F80C11C2F81011C2F8381502F5404222
:10AD0000D3F80414C2F82015D3F80814C2F8241597
:10AD1000D3F80C14C2F82815D3F81014C2F82C1567
:10AD2000D3F81414C2F83015D3F81814C2F8341537
:10AD3000D3F81C14C2F84015D3F82014C2F84415F7
:10AD4000D3F82414C2F84815D3F82814C2F84C15C7
:10AD5000D3F82C14C2F85015D3F83014C2F8541597
:10AD6000D3F83414C2F86015D3F83814C2F8641557
:10AD7000D3F83C14C2F86815D3F84014C2F86C1527
:10AD8000D3F84434C2F8703515F0E8FE18B14F4BD3
:10AD90004F4AC3F88C2615F0E1FE18B14D4BFB224B
:10ADA000C3F8182515F0DAFE70B14FF080414FF06E
:10ADB0008053D1F8E42ED3F8583222F00F0203F07A
:10ADC0000F031343C1F8E43E15F0C8FE20B1424B17
:10ADD0004FF40072C3F840264FF08053D3F830315F
:10ADE000082B09D14FF08043D3F80024D10744BF8A
:10ADF0006FF00102C3F80024384AD2F8883043F4D7
:10AE00007003C2F88830BFF34F8FBFF36F8F4FF0DE
:10AE10001023D3F80C22D2071DD5314B0122C3F8E1
:10AE20000425D3F80024002AFBD04FF01022D2F8DA
:10AE30000C3223F00103C2F80C32294BD3F8002462
:10AE4000002AFBD00022C3F80425D3F80024002AEE
:10AE5000FBD000F069FDD3F80022002A03DBD3F811
:10AE60000432002B22DA1E4B0122C3F80425D3F84A
:10AE70000024002AFBD04FF010221221C2F8001249
:10AE8000D3F80024002AFBD04FF010231222C3F87D
:10AE90000422134BD3F80024002AFBD00022C3F86D
:10AEA0000425D3F80024002AFBD0D2E70D4B0E4A2C
:10AEB0001A6035F09DFF00BF6006012000000120F0
:10AEC000A493090060670120600601200050004043
:10AED0004881030000F000400090024000ED00E0D7
:10AEE00000E00140000001200090D0030149024829
:10AEF0003AF03CBD785B01200030004002494FF041
:10AF000040203AF033BD00BFAC5B012008B50748D4
:10AF1000D0F8183143B14FF48C7151F0B3FDBDE856
:10AF20000840034849F0E3BC08BD00BF00300240C0
:10AF3000185B012008B50748D0F8183143B14FF429
:10AF40008C7151F09FFDBDE80840034849F0CFBC2B
:10AF500008BD00BF00F002403C5B0120F7B5224C69
:10AF6000022501A853F058FB052812D11F4C204E92
:10AF70004FF40C750DF102012046ADF8025053F06C
:10AF8000EBFA28B30C2802D11A4852F037FD03B06F
:10AF9000F0BD019B032B19D004D8022BE1D1002373
:10AFA0002370DEE7A3F10902022ADAD80A2B09D0BE
:10AFB000092B09D00B2B0CBF01204FF0FF303AF0CA
:10AFC000B5FBCEE70020FAE70220F8E72570C8E7D6
:10AFD000D6F80031002BCDD01F68D3E901122046EE
:10AFE00090473B46F6E700BF4367012084580120A5
:10AFF000505C0120253C0900014902484AF026B96D
:10B00000605B012000900040014902484AF01EB9EF
:10B010006C5B012000A000400149024855F089B94D
:10B02000E05B0120002000400149024855F081B951
:10B03000045C0120008002402DE9F04FB64BB74A76
:10B04000D3F80013002385B01C4601201D4621FAC9
:10B0500003F6F6070BD552F8236046B100FA03F663
:10B06000344342F82350BFF36F8FBFF34F8F013348
:10B07000192BECD1E20736D5A74B0122C3F81425D2
:10B08000C3F8102500221546930003F1804303F511
:10B090001C330132082A5D609D62F5D19E4B5D62D2
:10B0A0009D64C3F85851D3F80024D3F800140A4320
:10B0B000C3F80024D3F80023C3F80823984AC3F840
:10B0C0000423984BDC22002118464AF066FD4022FA
:10B0D00082820281012101A8CDE9015503958DF8F5
:10B0E000051011F09DFD14F4006F8E4D08D08A4BB1
:10B0F000D3F8A8369BB2A5F8D230012385F8D73013
:10B10000A3021ED5844ED6F8143513F4807302D0F2
:10B110003EF08CFB0123D6F81025D70540F136818F
:10B1200095F8D7304BB1B5F8D220002085F8D7007C
:10B13000012392B2882146F05BFC0121032046F0F6
:10B140004AFC600226D5744BD3F8006406F4E06232
:10B15000F105C3F8002405D50121C3F82C150420FE
:10B1600046F039FC72050FD56B4B0122C3F8082558
:10B170009A65D3F8002312F4001208BFC3F85421D3
:10B180004FF40012C3F80423B30503D501210520B1
:10B1900046F021FC270237D55F4BD3F880E4D3F883
:10B1A0008424D3F88814D3F88C74D3F89064D3F83B
:10B1B00094045FFA81FCD3F89814D3F89C341EF001
:10B1C0007F0F5FFA8EF8D2B2FFB2F6B2C0B2C9B248
:10B1D000DBB201D1052A17D04FF4C06E8DF80D00F7
:10B1E0008DF80E1001A80121CDF804E08DF808803B
:10B1F0008DF809208DF80AC08DF80B708DF80C6061
:10B200008DF80F3011F00CFD474B23405BB195F8E2
:10B21000D830002B40F0C2804FF0E023D3F8F03D4F
:10B22000DE0700D500BEDFF8FC80DFF8EC90DFF829
:10B2300000B1474600264FF0140A06F10C0324FA29
:10B2400003F3D807F1B222D50AFB0693082ED3F8F0
:10B2500008273B6853FA82F33B604FF0180303FB67
:10B260000653D2B2D88812FA80F080B2D88000F0AB
:10B2700099803889904240F09580DB88BA889BB2EB
:10B280009A4240F28F8011B9584615F049F80136BC
:10B29000092E07F11807D0D1244B2340002B6BD087
:10B2A0001D4BD3F86C94C3F86C94BFF36F8FBFF34E
:10B2B0004F8F14F4806407D0D3F88044D3F88034DF
:10B2C0001906C4F3C01479D54FF0000A154F0026B3
:10B2D0004FF0180B29FA06F3DA07F0B201D44EBB8F
:10B2E00044B30D4B142202FB0633FA68D3F8083638
:10B2F00052FA83F2FA600BFB0652518A89B251FA74
:10B3000083F39BB25382538A398A9BB2994258D9AC
:10B310003EF040FA0EE000BF0070024000710240B3
:10B320000514C0016C1F0120FCFB1F00000400017C
:10B330004C7002400136082E07F11807CAD10024CC
:10B340001826012704F1100329FA03F3DB07E0B202
:10B3500003D464B9BAF1000F09D006FB0452B8F85F
:10B360000410D3889BB2994234D93EF033FA0134A9
:10B37000082C08F11808E5D11748184B0360002382
:10B38000436005B0BDE8F04F05F0DABA002B7FF45A
:10B39000D4AE4FF40013C6F80833CEE6002385F888
:10B3A000D83040E7182303FB06530020DA88BA8020
:10B3B000DA88012392B246F01BFB68E74FF0010ADE
:10B3C00084E7528A40F08001012392B2002046F0C7
:10B3D0000FFBAFE79772CAE73C610120CB0508007D
:10B3E0002DE9F0478AB08C46DDE9121E11F001010B
:10B3F000DCF80C400646174602D0012B00F0A28074
:10B40000B4F5C87F72DA2011052290FBF2F20292A5
:10B4100002EB8202821A0392C4F38102049204F0C6
:10B4200003040022059415461446DCF81480B8F194
:10B43000020F40F0BC80DCF81800002808BF4FF075
:10B44000010805EB45058148454410F82580CDF8F5
:10B45000188000EB850568780790A8780890E87850
:10B46000099011B3012B20D10DF108090EF1040848
:10B4700006AB4D4603CD9D42C8F80000C8F8041045
:10B48000A94608F10808F4D10EF114080DF12809B5
:10B490001D4603CD4D45C8F80000C8F804102B46E2
:10B4A00008F10808F4D1CEF80020DCF81430CCF80C
:10B4B0003C40022B40F0C080DCF81840002C00F02B
:10B4C000A3807C1E7D1D0299304655F0C3FF04F811
:10B4D000010FAC42F7D1032301240DF1180A03EB4D
:10B4E000430599463D444FF0000877E0B4F5FA7FF4
:10B4F00012DAA4F5C874A0100522B0FBF2F2029291
:10B5000002EB8202821A04F00304039200220494E4
:10B5100005921446012588E7A4F5FA740320B4FBCC
:10B52000F0F000EB4002A41ADCF81820029000258D
:10B53000CDE90455039412B1CDE903042A46012450
:10B54000022572E7B4F5B47F04F001024FEA640506
:10B5500010DA242495FBF4F004FB10550624029025
:10B5600095FBF4F004FB105500240495039005941A
:10B5700003255AE7F32D0CDCB43D2811029000247A
:10B58000C5F3810005F00305049503900594042597
:10B590004BE7F43D0320B5FBF0F0029000EB4000D8
:10B5A0002D1A00240395CDE9044405253DE74FF00D
:10B5B000000846E702AB304653F82410019155F0DD
:10B5C00049FF01992875304655F044FF0199687587
:10B5D000304655F03FFF08F10108A8755AF82420BD
:10B5E000904508EB090305F10305E3DB0134042C66
:10B5F0007FF475AF002387F83D3087F83C3087F83B
:10B600003B300AB0BDE8F087234666E702AB304620
:10B6100053F8241055F01EFF08F8010B01355AF8B5
:10B620002420954205EB0903F0DB0134042C07D1FB
:10B630000023BB757B75E4E700231C460DF1180A57
:10B64000994607EB03080025E9E700BF665E09009D
:10B6500010B5074CD4F800314BB1064B5B689847E6
:10B6600020464FF48071BDE8104051F00BBA10BD78
:10B6700000000140285C0120022A2DE9F0415AD146
:10B680003B4B826883FB02423A4E846986FB04543A
:10B6900022440A60384C426884FB0252374FC56925
:10B6A00087FB05C52A444A60026883FB0252056A8B
:10B6B00086FB05752A448A60314F026887FB025277
:10B6C000304D066A85FB06C63244CA604FF06046BC
:10B6D000426886FB02C2D0F81CC086FB0CEC6244B8
:10B6E0000A61826885FB02C2D0F818C087FB0CECA7
:10B6F00062444A61426983FB02C28A61026984FB37
:10B7000002C2CA61C26883FB02420A62C36887FB45
:10B7100003234B62036986FB03238B62436985FB2A
:10B720000323CB620023C1E91033C1E90E33C1E921
:10B730000C33BDE8F081144B902404FB023202F17B
:10B74000480C01F144058C3200F1240E50F8043B02
:10B7500052F804695CF8047B1C4687FB048441F8BA
:10B76000044B86FB0343864545F80439EED1E0E7F8
:10B77000D8E3CEB8281C310733C3BEB2CD3C410D4F
:10B780009A615FC9669EA0F69C8709002DE9F34186
:10B7900090F8653090F86620013BDBB280F86B30A2
:10B7A000531EDBB280F86C30012A84BF90F86C30F5
:10B7B00003F1FF334FF000058CBFDBB2012380F8AB
:10B7C0006D30044680F86E500126856540F20337DF
:10B7D00094F86330EAB2934215D82368324A934210
:10B7E00030D002F58052934257D002F580529342F6
:10B7F00055D002F58032934253D002F580529342E5
:10B800003FD104231FE0A36C03EB021301A81B7BB1
:10B8100001934FEA02182BF025F9019A02F5E07224
:10B8200040F8227094F86D303342A36C4344187B87
:10B8300005D051F096F97600F6B20135C8E751F01F
:10B8400066F9F8E70023194850F8332000EBC303EA
:10B85000002593F9043001215160002BC2F80455F2
:10B86000D160C2F80855C2F810554FF48035C2F8BF
:10B87000045306DB5A0903F01F0399400C4B43F8AD
:10B880002210236801224FF47A715A60DA60C3F8FB
:10B8900040151A6002B0BDE8F0810123D3E702230E
:10B8A000D1E70323CFE700BF0080004078620900A2
:10B8B00000E100E000280DDB4309012200F01F0039
:10B8C00002FA00F02033044A42F82300BFF34F8FFE
:10B8D000BFF36F8F704700BF00E100E04309012212
:10B8E00000F01F0002FA00F02033044A42F823005F
:10B8F000BFF34F8FBFF36F8F704700BF00E100E0D1
:10B900000028ACBF00F16040064B4FEA4111ACBFCC
:10B9100000F5614000F00F00C9B2B4BF195480F8BF
:10B920000013704714ED00E0BFF34F8F0549064B3D
:10B93000CA6802F4E0621343CB60BFF34F8F00BFCD
:10B94000FDE700BF00ED00E00400FA05014B1868B8
:10B95000704700BF0800012070B510EE105A25F0A6
:10B9600000440123B4F1FF4FB0EE403A06460360B5
:10B9700004DB60EE003AB0EE630A70BD34B9DFED6F
:10B98000CA7AB7EE007AC7EE273AF4E7B4F1E45F7B
:10B990000BDA002DBEBF4FF0FF330360B1EE400A5B
:10B9A0001CF0A0FFF1EE403AE5E7002D80F2C282E4
:10B9B000B4F1964FE3DAB4F17A5F9FEDBC5A78DACE
:10B9C000DFEDB90A20EE050A002000F021FEF0EEBE
:10B9D000403AF5EE403AF1EE10FAD0D023EE230AC9
:10B9E000B0EEC00A85EE000A1CF07CFFF5EEC03A0E
:10B9F000F1EE10FA4CBF4FF0FF330123B4F17E5F3C
:10BA0000F0EE402A336000F08F82B4F1804FB1EE47
:10BA1000433A00F089826B0000F1D281A44B9C4232
:10BA200000F3F380B0EE430A1CF05CFFA14B9C4294
:10BA3000F1EE407A40F39B80F7EE003A33EEC33AE2
:10BA400023EE037ADFED9C6A9FED9C6ADFED9C3A62
:10BA5000A7EE266ADFED9B6AE6EE076A9FED9A6A1B
:10BA6000A6EE876ADFED996AE6EE076A9FED986AAF
:10BA7000E6EE873ADFED976AE7EE066A9FED966A93
:10BA8000A6EE876ADFED956AE6EE076A9FED946A97
:10BA9000A6EE876ADFED936AE6EE076A63EE833A05
:10BAA000E6EE873AB6EE007AE3EE473A73EEA73A4F
:10BAB000F7E1B1EE407AB0EE470A17F087F8B4EE3E
:10BAC000407AF1EE10FA19D0B6EE000A27EE007AAD
:10BAD000B0EE470A17F07AF837EE400A30EE000A67
:10BAE000F0EE407AFEEECF7A17EE903A062B39D878
:10BAF000DFE803F02312121F1F2B2B00DFED7A7AF1
:10BB000077EEC37A17EE903A03F0010307EE903A0E
:10BB10009B00B8EEE70AE9E7F6EE007A37EEC00AD6
:10BB2000DFED610A20EE050A00F036FBF1EE403A47
:10BB30004FE7F7EE007A37EEC00ADFED5B0A20EE42
:10BB4000050A002000F064FDF0E7F7EE087A30EE19
:10BB5000670ADFED550A20EE050A00F01DFBB1EE85
:10BB6000400AE3E7F0EE007A30EE670AE5E75F4B64
:10BB70009C4264DDDFED5E3A73EE633A63EEA34A06
:10BB80009FED5C6ADFED5C6ADFED5C5A9FED5C5A0D
:10BB90009FED5C0A24EEA37AE7EE066A9FED5A6AEF
:10BBA000A6EE876ADFED596AE6EE076A9FED586AEE
:10BBB000A6EE876ADFED576AE7EE265ADFED566A92
:10BBC000E5EE876ADFED555AE6EE875ADFED546AF7
:10BBD000E5EE876ADFED535AA7EE255ADFED525A9C
:10BBE000E5EE075A9FED515AA5EE875ADFED505A00
:10BBF000E5EE075AE5EEA36ADFED4E3AE6EEC73A08
:10BC0000D4EE863A73EEC03A50E74B4B9C4206DDC9
:10BC1000F0EE003A33EEC33ADFED237A10E7474BFC
:10BC20009C4206DDDFED463ADFED1F7A73EE633AA4
:10BC3000A4E7F7EE007A33EE673ADFED1B7ADFED2B
:10BC4000416A9FED417A9FED416AA3EE267ADFEDCE
:10BC5000406AE7EE036A9FED3F7AA6EE837ADFED56
:10BC60003E6AE7EE036A9FED487AA6EE837ADFED3F
:10BC70003B6AE3EE066A9FED3A6AA6EE836ADFED61
:10BC8000396AE6EE036A9FED386AA6EE836AF7EE3C
:10BC9000006AE6EE036A27EE037AC7EE263ABEEEA6
:10BCA000007AE3EE073A01E700000000DB0F4940AD
:10BCB0006666663F1F4A3B3FA283D3376797673963
:10BCC0003F239E3DA1549C3A7E02F23B01F0893D08
:10BCD000752C3C384584E23834B6053AC66E3D3B97
:10BCE0001599A83C661AA53E0000004B07336D3E2F
:10BCF0000C5BEC3E6B7BA53976F4B7BA67F8663A15
:10BD000085300DBACDCDF83D07E7C73B474D06BDA1
:10BD10005EB9F73E27F9A3B9FE7771BB3D37933C77
:10BD20003C2117BEF7E9AF399916143BFEFC28BC3D
:10BD3000155A843D521CE63117A6DD3F1FA69D3FD4
:10BD4000C316BB3F5E3C5B3C78756A3EDBD5523B1D
:10BD5000B24B7A3FE73ABA3FF400223FAF72D53D8B
:10BD6000DFEF443F2D390840BE2E1D4067FF0538E8
:10BD7000B435F13ABDD7F536E440DA3CE6DC153EA1
:10BD80007ACCA63E5A245C3E3F239EBDD6EE4B3A6B
:10BD900054BF983C6E0F303EC5D0383F3B2DB23F6C
:10BDA000E8C4D5BAD23D5B3A1D7FD63E5C061CBACC
:10BDB000FD0C503A610B36BBABAAAA3D0000000057
:10BDC000B4F1824FF7EE003A7DDABDEEC36A5FED63
:10BDD000197A1FED197A5FED196AB8EEC60A16EEE8
:10BDE000103A33EE403A033BA3EE277A5FED1E7A1A
:10BDF000E7EE037A1FED1F7AA7EE837A5FED207AD4
:10BE0000E7EE037A1FED217AA7EE837A5FED227ABF
:10BE1000E7EE037A1FED237AA3EE267A5FED246A1C
:10BE2000E7EE036A1FED257AA6EE837A5FED266AB8
:10BE3000E7EE036A1FED277AA6EE837AF0EE636AD7
:10BE4000E7EE036A67EE837AC7EEA63AF6EE007A6B
:10BE5000E3EE273A042B24D8DFE803F0322F2C2915
:10BE60000300F1EE087A33EE270AF1EE047A73EE5E
:10BE7000277A67EE807AB1EE000A33EE000A60EEB0
:10BE8000277AB0EE080A33EE000A20EE270AF0EE19
:10BE9000007A33EE273A23EE000A1CF023FD73EEFE
:10BEA000803A002DBFF667AD72EEE33A63E5B7EE78
:10BEB000000ADAE7F7EE007ADDE7F7EE007AE0E76E
:10BEC000B7EE000AE3E7B0EE430A1CF00BFDB4F155
:10BED000B94F30EE630A24DA83EE837A1FED506A9D
:10BEE0005FED506A5FED503A67EE077AE7EE866ADB
:10BEF0001FED526AA6EEA76A5FED536AE6EE276A67
:10BF00001FED546AA6EEA76A5FED556AE6EE276A52
:10BF1000F6EE007AE6EE873A33EE673AE3EE003A61
:10BF2000BFE763EE003ABCE75FED5C3ABCE75FED6C
:10BF30005D3A20E5B4F17E5FF9D0B4F1804FF6D0E0
:10BF40005FED622A67E500BFF0B510EE105A854A32
:10BF500025F00043934285B0044605DC002380EDC4
:10BF6000000A4360002020E07F4A934238DC002D25
:10BF7000DFED7E7A7E4A23F00F0318DD934230EE28
:10BF8000670A09BFDFED7B7ADFED7B7A30EE670A67
:10BF9000DFED7A7A30EE677A30EE470A80ED007A8C
:10BFA00030EE670A80ED010A012005B0F0BD934232
:10BFB00030EE270A09BFDFED6F7ADFED6F7A30EEE2
:10BFC000270ADFED6E7A30EE277A30EE470A80EDF1
:10BFD000007A30EE270A80ED010A4FF0FF30E4E7E7
:10BFE000674A934274DC9FED677AB0EEC00AF6EEC2
:10BFF000007AE0EE077AFDEEE77AB8EEE77A17EE20
:10C00000900ADFED5A7AA7EE670A1F28DFED5A7A09
:10C0100067EE277AB1EE476A70EE676A16EE901AFD
:10C020001EDC594E471E25F0004256F8276022F0CC
:10C03000FF02B24214D0216094ED007A30EE470A3C
:10C04000002D30EE670A84ED010AAEDAB1EE477AD0
:10C05000B1EE400A84ED007A84ED010A4042A4E783
:10C06000C1F3C756DA15C6EBD353082BE3DDDFED7A
:10C07000417ADFED425AF0EE406AE6EE276A30EE92
:10C08000660AA6EE270AF0EE407AD7EE257A76EE1B
:10C09000E75A15EE901AC1F3C753D31A192B04DCD3
:10C0A000C4ED005AB0EE660AC6E7DFED385AB0EECE
:10C0B000660AA6EE250A76EEC07ADFED356AE6EE70
:10C0C000257AD7EE267A30EE677A84ED007AB3E7E8
:10C0D000B3F1FF4F06DB30EE400A80ED010A80ED40
:10C0E000000A3FE7DA15863AA3EBC25307EE903A0F
:10C0F000BDEEE77ADFED276AB8EEC77A77EEC77A4A
:10C100008DED017A67EEA67ABDEEE77AB8EEC77AD2
:10C1100077EEC77A8DED027A67EEA67AF5EE407A71
:10C12000F1EE10FACDED037A1AD1B5EE407AF1EEC8
:10C1300010FA14BF02230123214601A800F08CF855
:10C14000002DBFF632AFD4ED007AF1EE677AC4ED80
:10C15000007AD4ED017AF1EE677AC4ED017A7DE7D9
:10C160000323E9E7D80F493FE3CB1640800FC93FCF
:10C17000D00FC93F004435374344353708A3852ED7
:10C18000800F494384F9223F8057090000A3852E80
:10C1900032318D240000804310EE103A23F000432A
:10C1A000B3F1485FB7EE006A05DAFDEEC07A17EE2C
:10C1B000902A002A3DD060EE005ADFED1F7A9FEDF5
:10C1C0001F7ADFED1F6A1F4AA5EEA77A9342DFEDC3
:10C1D0001E7AE7EE257A9FED1D7AA7EEA57ADFEDB0
:10C1E0001C7AE7EE257AB0EE667AA7EEA57AF6EE2F
:10C1F000006A65EEA67A67EE256A20EEC07AA5EEA3
:10C20000A67A04DC37EEC77A36EE470A7047114A41
:10C210009342DABF03F17F4306EE903AF5EE026AED
:10C2200077EEE67A36EE660A77EEC77A30EE670A80
:10C230007047B0EE460A70474ED747ADF6740F31DF
:10C24000ABAA2A3D9999993E7CF293B4010DD0375F
:10C25000610BB6BA0000483F2DE9F04F2DED048B7D
:10C26000D7B09B460291D11E48BF111DC9104D1C6D
:10C270008146581EEB0003930C1A1AAF0BF1090C00
:10C280009FEDC47AC44B9246A2EBC50504EB0C0E9D
:10C290003E46002CA4BFE25C07EE902A04F10104A4
:10C2A000ACBFF8EE677AF0EE477A7445E7EC017AB6
:10C2B000EFD109EB8B0306EB8B0601930DF5847E22
:10C2C000DFEDB47A37464C46F4EC016A019B37ED5A
:10C2D000017A9C42E6EE877AF6D101308445EEEC95
:10C2E000017A06F10406EBD1AB48DFEDAC8A9FED95
:10C2F000AC9A0B180926049356AB03EB860111ED9B
:10C30000140A42AB06A94FEA860803EB86000F46E3
:10C31000344660EE287A013CFDEEE77AF8EEE77AE3
:10C32000A7EEC90ABDEEC00AA7EC010A30ED010A6A
:10C3300037EE800AEDD12846059132F07FFEB0EE4F
:10C34000408AB4EE000A28EE000A16F03FFCF2EE36
:10C35000007AA0EE678A002D0599FDEEC87AB8EE46
:10C36000E70A17EE907A38EE408A37DD06F1FF3C97
:10C3700006ABC5F1080E53F82C4044FA0EF0074402
:10C3800000FA0EF0241AC5F1070043F82C400441CE
:10C39000002C31DD00200137864651F8043B00288F
:10C3A00066D123B1C3F5807341F8043C01200EF13E
:10C3B000010E7645F1D1002D03DD012D5DD0022D5A
:10C3C00065D0022C18D1B7EE000A30EE488A98B139
:10C3D000284632F033FE38EE408A0DE005D1701E5B
:10C3E00006AB53F820402412D2E7F6EE007AB4EE02
:10C3F000E78AF1EE10FA39DAB5EE408AF1EE10FA7A
:10C4000078D1711E00238C46BCF1080F47D1002B58
:10C410004FD10EA8012150F80449002C46D056AB4C
:10C42000984406EB0B001AAB741CA8F14C0803EB04
:10C4300080000E44B4423FF75FAF049B1B5D07EEE4
:10C44000903AF8EE677A4F46E0EC017ADFED517AE8
:10C450000146F7EC016A019B31ED017A9F42E6EE5D
:10C46000877AF6D1E8EC017A0134E3E7022491E718
:10C47000C3F1FF0341F8043C99E706F1FF3C06AB2A
:10C4800053F82C1001F07F0143F82C1099E706F1C6
:10C49000FF3C06AB53F82C1001F03F01F4E706AA6D
:10C4A00052F82C000CF1FF3C0343ADE70131B2E739
:10C4B000013906AB083D53F82130002BF8D028464F
:10C4C000B7EE000A019132F0B9FD01998B001A1DF7
:10C4D00042AB98180B46002B39DA0B46002B65DB74
:10C4E00042A800EB8306DFF8BCC0DFED2A7A002506
:10C4F000C81A45E0039BB0EE480AA3EB0A0032F0ED
:10C500009DFDB4EEC90AF1EE10FA17DB60EE287A51
:10C5100006AAFDEEE77A711CF8EEE77A0835A7EE79
:10C52000C90AFDEEE77ABDEEC00A10EE103A42F8F5
:10C53000263017EE903A42F82130C0E7BDEEC00A2F
:10C5400006AA10EE103A314642F82630B7E706AD9B
:10C5500055F82350019507EE905AF8EEE77A013B23
:10C5600067EE807A20EE280A60ED017AB3E7FCECF2
:10C57000016AB6EC017A01350A2DE6EE877A01D020
:10C580008542F4DD56AD05EB800040ED287A013B95
:10C59000A4E700BF00000000005809000000803B35
:10C5A0000000804374920900000000002EAB1FEDD4
:10C5B000027A13440A46002A1ADAFCB1F1EE477AED
:10C5C000029BC3ED007ADDED2E7A77EEC77A2FAAB3
:10C5D0000123994215DA0CB1F1EE677A029B07F05C
:10C5E0000700C3ED017A57B0BDEC048BBDE8F08FB6
:10C5F00073ED017A013A37EE277ADCE7F0EE477AFD
:10C60000DEE7B2EC017A013377EE877AE1E700BF2B
:10C6100010EE103A23F00043B3F1485F04DAFDEE68
:10C62000C07A17EE903A5BB320EE007ADFED157A10
:10C630009FED156AA7EE276ADFED147AE6EE077A1A
:10C640009FED136AA7EE876ADFED127A60EE076A44
:10C65000E6EE077A30B99FED106AA7EE276AA6EEDC
:10C66000260A704767EEE67AB6EE006AE0EE867A52
:10C67000D7EE870ADFED097AE6EEA70A30EE600A08
:10C68000704700BFD3C92E2F342FD7B21BEF3836D7
:10C69000010D50B98988083CABAA2ABEABAA2A3E34
:10C6A00010EE103A23F00042B2F1465F16DAFDEECA
:10C6B000C07A17EE901A39BB431C134306D1F0EE33
:10C6C000C07AB7EE007A87EE270A7047012800F09B
:10C6D0009E80FFEE007A87EE800A70474C498A42BE
:10C6E00012DBDFED4C7A002BB8BFB1EE400A37EE1B
:10C6F000C00ADFED497AB8BFF1EE600A77EEE00AD2
:10C7000030EE800ADFED450A9FED456ADFED456AB0
:10C71000DFED455A3E4920EE007A8A4267EE077AFD
:10C72000E7EE866A9FED416AA6EEA76ADFED406AF2
:10C73000E6EE276A9FED3F6AA6EEA76ADFED3E6A46
:10C74000E6EE276A9FED3D6AA7EEA56ADFED3C5A4B
:10C75000E6EE275A9FED3B6AA5EEA76ADFED3A5A4F
:10C76000E6EE275A9FED396AA5EEA76AF0EE667AE3
:10C77000E6EE077A60EE075AF0EE606AE7EEA56A29
:10C78000DFED337AE6EE870AE5EEA70A30EE207A8F
:10C790001DDB07EE900AF8EEE77A27EE076A37EE20
:10C7A000277A9B17C6EE076A03F00203C3F1010361
:10C7B000B0EE007A76EEE00A70EE600A00EE103A13
:10C7C000E0EEC77AB8EEC00A20EE270A70470128CB
:10C7D0001BD0FFEE007AC7EE876A1E4B17EE102AB9
:10C7E0001A4006EE102A16EE902A36EE400A134042
:10C7F00070EEC00A00EE103AF7EE007AE6EE007A2C
:10C80000E0EE807AA7EEA60A7047B0EE470A7047BE
:10C8100040A12C3FDA0F493F68212233000000007D
:10C820005FAE9BB745F4A3388453D937C8261A3A6C
:10C8300016696B3BA427B33C8988083E7AC09538BB
:10C84000B937813948DEBE3A1F37113CD10D5D3D05
:10C85000ABAAAA3E00F0FFFFF8B50E4605462549F3
:10C8600030464AF0FAF905F1080718B390F850304D
:10C87000D90602D5204824F0E5FF43F0100380F8E4
:10C880005030394646F053FC95F82A3003F00C033B
:10C89000002B90F8513014BF0122002262F34103B3
:10C8A00080F8513005D190F8503043F0020380F801
:10C8B0005030F8BD114930464AF0CFF90446B8B1BE
:10C8C00090F82A309A07D5D443F00203394680F80D
:10C8D0002A3046F0E3F995F82A3013F00C0F204681
:10C8E00018BF0121BDE8F84008BF002146F0C4B9D7
:10C8F0000348C0E7C8900800B82B0800608C080007
:10C90000C72B08002DE9F74F0646002508466A4662
:10C9100001A901954AF0F3FC0199022902D82348A4
:10C9200024F07CFF7068DFF888900122890017F0FE
:10C930003BFE756007463581019BACB2A34205F111
:10C94000010505D85B007760338103B0BDE8F08F47
:10C95000009B53F824A040F24642DAF8040002217A
:10C960001DF012F9DAF8080040F2A4511DF068F940
:10C9700040F2A45347F6FF72494683461DF0F4F88F
:10C98000DAF80C0040F2A9511DF05AF94FEA840878
:10C99000B844824640F2A95347F6FF7249461DF05B
:10C9A000E3F827F824B0A8F802A0C5E7572E08003E
:10C9B0000080FFFF2DE9F04F2DED028B90468DB0EA
:10C9C000C268BDF864B0DDF86890BDF86C701D9D5C
:10C9D00006468A461C46B0EE408A2AB143689A420F
:10C9E00000F0B58009F0C6F8BBF11F0F01D81F2F6A
:10C9F00077D9BAF1000F40F0A080002F554614BF40
:10CA00004FF0080A4FF00A0AB8F1000F00F09C80BE
:10CA100040F20122ADF81820621CADF81A20002265
:10CA2000079206A851F0BEFD8046002853D1182277
:10CA300001460DEB020049F0B0F89FED460A9FED6C
:10CA4000467A464B079528EE008A002FC8EE077AF3
:10CA500003FB04F408BF4FF0000942F21073404694
:10CA6000B4FBF3F40125189B8DF818A0ADF8244011
:10CA70008DF82D500293ADF80CB0CDF81090B6EEB5
:10CA8000007A77EE877AADF81470FCEEE77ACDED98
:10CA9000087A3FF0CAFD8046E8B9314C06AA02A9DF
:10CAA000204651F05FFD8046A8B92E49324606F176
:10CAB000280004F0E5FF9DF970202178284651F008
:10CAC0007BFD804638B92078294651F04DFD8046DF
:10CAD00008B9189BF36040460DB0BDEC028BBDE871
:10CAE000F08FBAF1000F20D05DB3F0EE0C7AB4EE07
:10CAF000E78AF1EE10FA6946284610D807EE904A08
:10CB00009FED197AF8EE677AF4EEC77AF1EE10FA33
:10CB100005D83FF04DFA6D464FF0020A74E73FF03A
:10CB200047FA6D464FF0030A6EE7002F554614BFD3
:10CB30004FF0040A4FF0050A66E700254FF0060A99
:10CB400062E74FF0010A5FE7CDE9068869E74FF039
:10CB50001108C0E70024744900401C4440420F0003
:10CB600033060120C5C706006666A63F2DE9F843D7
:10CB7000416098464B680B9F91469A790A9B80F8D2
:10CB80002C2003858D7D044605F0300605F0060552
:10CB900072B34B68D86840F0E2FEE0842DB1002308
:10CBA000C4E90298C4E90433A361002384F82D305A
:10CBB00084F82A30A384089BE361099B23621AB39B
:10CBC000EFB11B492246384604F05AFF5DB115F01B
:10CBD000040118BF012160681ABF84F82B100022DD
:10CBE000012209F09BF8DEB1B20616D4012315E04C
:10CBF0004FF6FF73C3842B4635461E46CEE70C48DE
:10CC0000214604F021FFE1E767B10A492246384690
:10CC100004F036FF26B17307E8D4022384F82B30E2
:10CC2000BDE8F8830348214604F00EFFF2E700BF99
:10CC3000EBCF070057D007002DE9F04F89B005462C
:10CC40009DF8487016465FFA81F81C46002B3DD0CF
:10CC50004268DFF890A0137912680621C2F8001527
:10CC6000342202FB03A3002F4FF0020283F82D2091
:10CC70004FF0000914BF002320234FF6FF77A7428F
:10CC800028BF2746CDE90479CDE9066969688DF8A2
:10CC90000C9008798DF80D804FF0340C09680193E1
:10CCA00003AA00FB0CA038F0F3FE0D4B984283461C
:10CCB00003D1E41B019B3E44DFD168682AF072FA7D
:10CCC000584609B0BDE8F04F38F032BE414609F091
:10CCD00075FA002814BF0020132009B0BDE8F08FBA
:10CCE0000000AD0B785B012013B5124B9889D989F0
:10CCF00093F90040421A92B2402A28BF4022002CE9
:10CD00000EDA884212D099680B48019248F005FF6C
:10CD10000949019A802002B0BDE810403BF0FAB802
:10CD200088424FF0000003D10021F4E78020FBE7A8
:10CD30000149F0E7541F012008500120064A002352
:10CD400052F8041B814201D1184670470133082B69
:10CD5000F6D14FF0FF307047A04601200D4B1878F8
:10CD600001280FD10C4B1B78FF2B0DD10B4B1B68EF
:10CD7000D9070AD4DA030AD413F4801F0CBF0020A9
:10CD8000042070470228F1D1704705207047012028
:10CD9000FAE700BF8067012090670120845F0120CF
:10CDA0002DE9F041094F05460E4600244FF6FF7865
:10CDB00037F81400404503D03246294651F016FC9E
:10CDC0004434B4F5AA7FF3D1BDE8F081C006012058
:10CDD000034B53F8203013B19A6801329A607047C0
:10CDE000941E012038B5154B53F82040FCB1207932
:10CDF0004FF0A9FE054660794FF0A5FE6D0005F4E1
:10CE0000FF75A2790E49E379284300F0030040EA58
:10CE10008202A0718A5C134494F908205BB29342A9
:10CE2000E37105DBE3680133E3600023E37138BDA0
:10CE300052429342FBDCE368013BF5E7C046012028
:10CE40009A3E09002DE9F04F0446A9B08A460146F2
:10CE500040F25C404AF0CEFC0BAD002844D1CDE955
:10CE600015000EAA7E21204620F028FCB04B11931D
:10CE700001224023CDE9122318AB149311AB109378
:10CE8000AC4B0B950C93082107A8002454F03DF8F7
:10CE90002846CDE9054453F0F5FAA146A0462746B9
:10CEA0009DF85CB0BBF1000F00F0A781284653F05D
:10CEB000E9FABBF15D0F00F0958054D8BBF13A0F51
:10CEC00048D8BBF12B0F1BD8BBF1220F00F0CF804D
:10CED00007D8BBF10D0FE3D038D8ABF10901012918
:10CEE000DED9954824F0AEFC012120461FF078FFE2
:10CEF00043680C9300230B940D938DF85C30C2E7CC
:10CF0000ABF12C030E2BECD801A252F823F000BF9A
:10CF1000A1CE02003DD10200E3CE0200E3CE02002A
:10CF20003DD102003DD102003DD102003DD10200C1
:10CF30003DD102003DD102003DD102003DD10200B1
:10CF40003DD102003DD10200A1CE0200BBF1200F75
:10CF5000A6D0C6E7BBF15B0FC3D1002048F093FB1E
:10CF6000044601261CE0BBF1740F69D032D8BBF136
:10CF7000660F48D0BBF16E0FB3D19DF85C30752BB6
:10CF8000AFD1284653F07EFA6C28AAD1284653F038
:10CF900079FA6C28A5D1284653F074FA00260E249D
:10CFA000002F40F0FD80204621F06EFD8046002ECF
:10CFB00040F00C81BAF1000F00F02481002C90D0D9
:10CFC000059B002B8DD107A853F077FF204629B091
:10CFD000BDE8F08FBBF17B0F00F0DE80BBF17D0F71
:10CFE0007FF47FAF002F3FF47CAF059B002B00F058
:10CFF0001481013B069A059352F82370384621F0BC
:10D0000043FD80464CE79DF85C30612B7FF469AFAF
:10D01000284653F037FA6C287FF463AF284653F064
:10D0200031FA73287FF45DAF284653F02BFA652858
:10D030007FF457AF284653F025FA00261E24AFE7A9
:10D040009DF85C30722B7FF44CAF284653F01AFAEF
:10D0500075287FF446AF284653F014FA65287FF40C
:10D0600040AF284653F00EFA00263E2498E70023EE
:10D0700008939DF85C1000293FF433AF222909D1B1
:10D08000284653F0FFF9DDE9081022F0A3FC002642
:10D09000044685E75C290CD1284653F0F3F975283E
:10D0A000014606D86D2808D862283ED0662808BFF9
:10D0B0000C2107A853F087FE33E0A0F16E03072B85
:10D0C000F7D801A252F823F0E9D00200B3D0020051
:10D0D000B3D00200B3D00200EDD00200B3D0020002
:10D0E000F1D00200F5D002000A21E2E70D21E0E7CD
:10D0F0000921DEE704260024284653F0C3F940F056
:10D100002000C0B2A0F13003DBB2092B84BF573836
:10D11000C3B2013E43EA0414EED1214607A853F0FE
:10D1200065FE284653F0AEF9A3E70821C1E700BF2A
:10D13000545608003D040800524508000024089495
:10D14000594607A853F03FFE9DF85CB0BBF12E0F87
:10D1500018D00BF0DF03452B14D0BBF12B0F12D0EE
:10D16000BBF12D0F0FD0584639F002F8064650B9E2
:10D17000DDE908105CB100963346324623F046FFE5
:10D1800004460DE70124284653F07CF9D8E73346DE
:10D190000A2224F099F8F3E700204AF00FF9DFE6BD
:10D1A000214B984514D1214638464AF072F8002E9A
:10D1B0003FF476AE069BDBB9012103A822F0FEF90D
:10D1C000069B1F60204621F05FFC8046274667E6ED
:10D1D000B9F1000F04D1002E7FF483AEA1465FE6C3
:10D1E00049462246384649F078FD4FF00009DEE70F
:10D1F000394603A84AF04DF8E4E73C46DAE628460B
:10D2000053F040F99DF85C60304638F0C5FF0028C7
:10D21000F5D1002E3FF4D2AE63E63C46BAF1000FE2
:10D220007FF4D1AEEEE700BFF8570800C20713B590
:10D23000044603D5C0F3470002B010BD830707D1F1
:10D2400002680E4B9A4203D121F00CFCC0B2F3E706
:10D25000204622F00DF948B1204621F07DFBFCEE7E
:10D26000C07ACDED017A9DF80400E5E7204621F073
:10D270000BFC5E22C188024824F0D8FAE81D0800A1
:10D28000193708002DE9F041314ECCB031238DF82B
:10D29000083073880124B3F57F7F07468DF8094075
:10D2A0000DD3002402222B480094234602A98DF8B6
:10D2B000092008F085FE20464CB0BDE8F08102212F
:10D2C00002A800F0E7FB054608B10024F3E7B6F832
:10D2D000028008F10403BB42EDD815F03DF8311D82
:10D2E00004AA08F80150074646F07DFD044650B9EF
:10D2F0009DF81C30184913F0100F14D11649384608
:10D3000046F019FE04463AF0A1FAB4B900231148D8
:10D310000093022202A908F053FE002CD5D10D483B
:10D3200008F036FEC7E70D4A1368526803A81B1AB7
:10D330009A4206D83AF08AFA022402238DF809307C
:10D34000E4E7384636F0C4FB04460028DBD1D5E7D5
:10D3500088510120A84F01208C510120505C0120F0
:10D360002DE9F04F0746E1B0594841F0D4FE061EC2
:10D3700009DB584C6588B5F57F7F06D340F2512311
:10D38000238032F06BF900253EE02B1DBB4200F2FA
:10D390009D8014F0E1FF271D6A1E04A9D35D2F2B89
:10D3A0004FF000030CBFBB547B554B4A46F014FBB7
:10D3B00040F2511347F8043C0027C4E90177E760C5
:10D3C000054618B1032363703046DAE718A904A8AC
:10D3D00046F0EFFBAA46D8B1002104A8DFF800B15F
:10D3E00046F0E7FB4FF00009C4F808A0CA451AD17F
:10D3F00004A845F0F4FF0023A26863803046626011
:10D40000E360A36132F02AF9284661B0BDE8F08FED
:10D410009DF87A30002BDFD018A904A846F0C9FB8C
:10D420000AF1010AD7E718A904A846F0C2FBBDF823
:10D430006A30BDF86810C4F8049003F01F0252006F
:10D44000480A0192C3F344120092DB0A01F01F0262
:10D4500000F2BC70C1F3431152F0DAFC1F4B002202
:10D46000C01842F10001A0FB0B030BFB0133C4E920
:10D4700004039DF86C3013F0100314BF0123E36024
:10D480000DF17A000DBF189BE360A261A36152F019
:10D4900019FA60808046304632F0E0F80027B8453F
:10D4A00002D809F10109A1E7A8EB0702042A4FF00D
:10D4B00000030DF17A0128BF042239440448009387
:10D4C000039208F07DFD039A1744E8E701259BE7E6
:10D4D000A84F0120885101208C51012080436D38D4
:10D4E00000CA9A3B70B52A4B1D682A4B1B681A6804
:10D4F000012151641B68284AD3F84465002352F87F
:10D50000044B14B12179814232D00133082BF6D17A
:10D5100070BD6369A269EB1AB21AC3EB03431344EB
:10D520004FF6FE714FF6FF728B4288BF1346E289B9
:10D53000218A89B211FA82F2A189B2FBF1F001FBD2
:10D540001022A16821F81230238AA2899BB293424B
:10D5500004D2238A01339BB2238216E0E3899BB273
:10D560000133B3FBF2F102FB11339BB2E3810CE018
:10D57000E379002BCDD04FF0E6FA6379003818BF7D
:10D580000120834201D00023E3716561A661BFE7FA
:10D59000705F01201C610120A04601202DE9FF41A0
:10D5A0004368DB6853F8215004460F4640F25A4066
:10D5B00029464AF01FF9064600285AD043682846F3
:10D5C0009847B36801A95B6880469847B3680546E9
:10D5D0009B6800214046984763682A49DB6853F8F6
:10D5E000270049F03AFB0246C0B190F85030B0F93C
:10D5F00038106FF3041380F85030B0F93C30994282
:10D6000039D001A9383044F051FC012592F850304E
:10D610006FF3041382F850300023936263681A4951
:10D62000DB6853F8270049F018FB064668B190F80C
:10D630002A306FF3410301A980F82A3012F04CF828
:10D6400000210546304645F029FB7DB194F82A308B
:10D65000DB0704F1180210D4114601A844F026FC9F
:10D6600094F82A3043F0010384F82A3004B0BDE86E
:10D67000F0810546B0E70025C8E701A9104644F04F
:10D680003CFCEDE7C8900800608C0800F8B5194B29
:10D6900000241C70184BFF271F70184F0D461646AC
:10D6A00000F008FE00230022DFF85CC0C7E9002379
:10D6B0002146234620469D420DD158B191ED017A75
:10D6C000DFED0F7A67EE277A17EE900AFAF730F857
:10D6D000C7E90001F8BD56F82320940708D1146863
:10D6E000644505D110B1074824F0ACF8114601207B
:10D6F0000133E0E78067012090670120F00A0120F4
:10D7000000007A44E82D080020670800012B2DE96D
:10D71000F04701D0242B06D9FEF718F91623036031
:10D720000020BDE8F087DFF8E4C00D462E4615F86E
:10D73000014B14F80C7017F00807F7D12D2C32D1DB
:10D740002C780127B51C002B5BD0102B09D1302C75
:10D7500007D12C7804F0DF04582C4DD16C781023BD
:10D76000023507F1004808F1FF384FF0000CB8FB14
:10D77000F3F9664603FB198AA4F1300EBEF1090FD6
:10D7800016D87446A34224DDBCF1000F1EDBB14560
:10D790001CD301D1A24519DB06FB03464FF0010C57
:10D7A00015F8014BE8E72B2C04BF2C78B51CCAE711
:10D7B000A4F1410EBEF1190F01D8373CE2E7A4F104
:10D7C000610EBEF1190F04D8573CDBE74FF0FF3C68
:10D7D000E6E7BCF1000F05DA22230360464642B9B2
:10D7E00030469EE707B17642002AF9D0BCF1000F1F
:10D7F00000D0691E1160F3E73024002BB1D108235B
:10D80000AFE7302CA5D00A23ABE700BFA1920900F7
:10D810002DE9F043364F86460D46284615F8014B54
:10D82000E65D16F00806F8D12D2C2FD12C780126B4
:10D83000851C002B57D0102B09D1302C07D128780C
:10D8400000F0DF00582849D16C78102302354FF0E2
:10D85000FF380027B8FBF3F803FB08F96FEA090962
:10D860003846A4F1300CBCF1090F14D86446A34229
:10D8700022DD002F1DDB80451BD301D1A14518DB24
:10D8800000FB0340012715F8014BEAE72B2C04BFEE
:10D890002C78851CCDE7A4F1410CBCF1190F01D8FF
:10D8A000373CE4E7A4F1610CBCF1190F04D8573CF4
:10D8B000DDE74FF0FF37E6E7002F07DA2223CEF847
:10D8C00000304FF0FF3032B9BDE8F08306B140427E
:10D8D000002AF9D007B1691E1160F5E73024002B4A
:10D8E000B5D10823B3E7302CA9D00A23AFE700BF96
:10D8F000A19209002DE9F84390F82A309B070446CD
:10D900002ED4BDE8F883DB6853F8267040F25A4005
:10D91000394649F06FFF054668B143683846984775
:10D92000AB6804F108019B689847013663689A6800
:10D930009642E8D3E5E74146384649F08EF920B1F2
:10D9400004F1080145F0F3FBEFE74946384649F09A
:10D9500084F90028E9D004F1080145F09FF9E4E7D3
:10D96000DFF80880DFF808900026DFE7C89008009D
:10D97000608C080090F95030214930B5002B836A43
:10D98000B4BF428A028AB0F90C408589002B08BFD7
:10D990000B46224494B29A7BC2B193F905105A887F
:10D9A00011FB05F1114409B2A0F8461093F90520C6
:10D9B0005B8812FB04F213441BB29942D2BFA0F859
:10D9C0004A30A0F84A10A0F8463030BD93F9041050
:10D9D0001A8811FB05F1114409B2A0F8441093F91B
:10D9E00004201B8812FB04F213441BB29942D2BFDD
:10D9F000A0F84830A0F84810A0F84430E5E700BF90
:10DA00001C06012090F95030214930B5002B836A63
:10DA1000B4BF028A428AB0F90E40C589002B08BF04
:10DA20000B46224494B29A7BC2B193F904101A882F
:10DA300011FB05F1114409B2A0F8441093F9042038
:10DA40001B8812FB04F213441BB29942D2BFA0F808
:10DA50004830A0F84810A0F8443030BD93F90510C4
:10DA60005A8811FB05F1114409B2A0F8461093F948
:10DA700005205B8812FB04F213441BB29942D2BF0B
:10DA8000A0F84A30A0F84A10A0F84630E5E700BFF9
:10DA90001C06012013B50C4B1C780A4644B10B4BF5
:10DAA0001B7843B10A490B782BB901220A701C4636
:10DAB000204602B010BD05234370002301460093A9
:10DAC000044808F07DFAF3E756670120510601206B
:10DAD000FC650120A84F012008B510EE103A23F094
:10DAE0000042B2F17E5FF0EE405A10D308D19FEDB4
:10DAF000300A9FED306A002BA8BFB0EE460A08BD81
:10DB000070EE405ADFED2B7A87EEA50AF7E7B2F107
:10DB10007C5F11D2B2F14A5F9FED276A44D920EEB3
:10DB2000000AFDF78BF8DFED257AE0EE657A35EE39
:10DB3000E70A36EE400AE2E7002BB7EE000AF6EEFF
:10DB4000007A14DA35EE800A9FED1D6A20EE270A6E
:10DB5000F1EEC05AFDF772F8A0EE256A9FED160AA5
:10DB600075EE865A30EE650A30EE000AC7E730EEF1
:10DB7000650A20EE270AB1EEC05AB0EE407A15EEE3
:10DB8000103A23F47F6323F00F0306EE103AA6EE5B
:10DB9000467A75EE067AC7EE275AFDF74FF8E0EEA3
:10DBA000055A36EE250ADFE7B0EE460AA7E700BFC2
:10DBB000DA0F494000000000DA0FC93F6821A233A4
:10DBC0006821A2B308B510EE103A23F000425B00C2
:10DBD000F0EE407A0FD4B7EE000A77EEC07ABDE8D7
:10DBE000084037EEA77AA7EEA77AB1EEC70A37EE5C
:10DBF000800A1AF0CBBDB2F18B4F13D2FFEE006A50
:10DC0000E0EE006ABDE80840B1EEE67AF7EE006AA1
:10DC100037EE007A86EE870AB0EE007A97EE870A32
:10DC20001AF060BE1AF05EFEDFED027A30EE270ACF
:10DC300008BD00BF1872313F70B588B00D460C208A
:10DC400000211646039347F0A1FE0D4B036005AB80
:10DC500001930C4B039A0093044603233146284654
:10DC600048F0B7F89DF81830059A626023729DF865
:10DC70001C3013B1204606F0DBFF204608B070BD13
:10DC8000086408002442090010B58EB003AB51F8B7
:10DC9000044B0193194B0093013803231BF0F0FE52
:10DCA00040F27741606806AA1FF008FD237A5B0006
:10DCB00043F001030893039B099340F626130A934C
:10DCC000049B5B0043F001030B93059B6FF0004244
:10DCD00093421FBF40F2E6425B000C9243F0010307
:10DCE00014BF0221012106AA4FF0020018BF0D93B4
:10DCF00048F0E3F90E200EB010BD00BFA4410900AA
:10DD000010B58EB003AB51F8044B0193194B00933F
:10DD1000013803231BF0B4FE40F2A251606806AA4A
:10DD20001FF0CCFC237A5B0043F001030893039BB4
:10DD3000099340F626130A93049B5B0043F001030A
:10DD40000B93059B6FF0004293421FBF40F2E642E7
:10DD50005B000C9243F0010314BF0221012106AACB
:10DD60004FF0020018BF0D9348F0A7F90E200EB037
:10DD700010BD00BF6C42090010B596B003AB51F85E
:10DD8000044B01932D4B0093013806231BF078FEC2
:10DD900009AA606840F2A3511FF090FC237A5B004F
:10DDA00043F001030B93039B0C93049B0D9344F2EC
:10DDB00036230E93059B5B0043F001030F93069BF4
:10DDC0006FF00042934235D05B0043F0010344F210
:10DDD0001622119310920923032116AA02EB830243
:10DDE00043F6E60042F8340C16AA02EB8300079AC9
:10DDF000520042F0010240F8302C089A6FF00040C7
:10DE0000824210D016A800EB830043F6C60440F807
:10DE10002C4C16A800EB8303520042F001020131A2
:10DE200043F8282CC9B209AA032048F046F90E206D
:10DE300016B010BD07230221CFE700BF3C42090006
:10DE4000F0B58DB00D46182000211646039347F01B
:10DE50009DFD174B036005AB0193164B039A00938E
:10DE6000044607233146284647F0B3FF069D124972
:10DE700040F29E2228461BF0CBFE089E059F9DF88F
:10DE800024009DF828109DF82C209DF81C3020734C
:10DE9000C4E9017606986173A2732561237518B1F0
:10DEA0000022012141F04AFB20460DB0F0BD00BF29
:10DEB000C8640800BC410900E88408002DE9F3416A
:10DEC000044601F134000E4602F03AFD2388102B7F
:10DED00005D0112B3FD0002002B0BDE8F0812F4DBE
:10DEE000002388224FF6FF7102FB03F7785B88421C
:10DEF00003D00133052BF7D1042388225343A18893
:10DF0000E952EA184FF000080E2307F16000D365CC
:10DF10002844234982F85A80A2F87680EA1903F04F
:10DF2000AFFDC6F81880206961696C373D4403C5B0
:10DF3000684650F033FBBDF80030228A9A4202D87E
:10DF4000628A9A4203D2A088694650F015FB0023EA
:10DF5000F3600120C0E7A388104F0025882202FB50
:10DF600005F1C85B984203D00135052DF7D1042592
:10DF700039440B4803F09AFD88235D437A194FF624
:10DF8000FF737B53002382F85A30D26D0E2A1EBFD6
:10DF90005360217A1172B361DBE700BFC006012034
:10DFA00011BE0300F0B58DB00D464FF48A7000210C
:10DFB0001646039347F0EAFC224B036007AB01933C
:10DFC000214B039A0093314605230446284647F027
:10DFD00000FF0798012204A91EF0C8FE059E26F046
:10DFE0000803102B04D0202E02D0184823F02AFC5E
:10DFF000089D049F022D11DC002D11DD099890B9B8
:10E0000000230A9AC4F81021204684F80C513246A5
:10E01000394640F006FB20460DB0F0BD062DEDD090
:10E020000B4823F0B7FB012204A948F070FB00283D
:10E03000E6D0059840F2591210211BF0A5FD049B73
:10E04000DFE700BF2065080084420900892B080033
:10E050000C2F08002DE9FF410C46D1F80080064640
:10E060000122606801A91EF081FEDDE9017517B982
:10E07000124823F0E7FB25F00803102B03D0202DD6
:10E0800001D00F48F5E7022E15D9A068012201A999
:10E090001EF06CFE0298019C40F2591210211BF0F8
:10E0A00073FD404623462A46394640F0BAFA0E2010
:10E0B00004B0BDE8F0810024F3E700BFDA2C0800CB
:10E0C000892B080010B50446084620F08DFC022874
:10E0D00005DC002805DD84F80C010E2010BD0628A3
:10E0E000F9D0014823F056FB0C2F08002DE9804899
:10E0F00085B002AF3B1D01931F4B009305460123E2
:10E100000E4600201BF0BCFC314628463AF080F950
:10E11000D7F80490DFF86CB0484621F019FA4FEABE
:10E1200060084FEA8803073323F00703ADEB030DC4
:10E130000DF1080A0024444505D1A4B10F4840F26E
:10E14000514123F02FFB6100042241F001014846B8
:10E1500022F022FB40F2472259461BF059FD4AF8B3
:10E1600024000134E7E7294601203246FFF78EFA02
:10E170000348214649F0CBFBAC4209006A4908003C
:10E18000EC420900E884080070B50E4605460028F8
:10E1900044D03AF03DF9324629460020FFF776FA9E
:10E1A00000F02AFA00231A4635F09EFE1C4B5C6AEA
:10E1B00094BB40F056FA78B3FEF7D0FD012818D092
:10E1C00002280BD1174A234656F82340A10702D153
:10E1D0002168914203D001339D42F5D10E2420469F
:10E1E00031F0F8FC00F0E0F8204631F0F3FC204676
:10E1F00070BD0D4B0D491A78234656F82340A007F1
:10E2000006D12068884203D1606800799042E6D048
:10E2100001339D42F1D1E1E70E24E3E70E24E6E766
:10E22000505C012020670800906701204C660800C0
:10E2300070B588B00D460C2000211646039347F0B8
:10E24000A5FB134B036004AB0193124B039A00939D
:10E25000314604230446284647F0BBFD40F23C41CA
:10E2600004983AF09DF89DF818109DF814209DF838
:10E270001C3011B1084823F0E5FA01792F2901D9A2
:10E280004FF0CAFC606020462272637208B070BD15
:10E290004C660800B4420900974A080010B5044CC7
:10E2A00023781BB90DF02AFD0123237010BD00BF98
:10E2B0003E6701202DE9F04F354BD3E900C7354BC0
:10E2C000D3E9008E344BD3E9006387B00024CDE955
:10E2D0000244019302EB8103059004934FF0FF3158
:10E2E0004FF00109049B934218D1029B13B1294BB3
:10E2F000C3E9008E039B13B1254BC3E900C71CB1D2
:10E30000254B019A1E605A6001313DD0059B002BC0
:10E3100035D107B0BDE8F04F0DF0F0BC52F8040B5A
:10E320008307DFD103681D4DAB42DBD1436890F812
:10E3300008B01979A1F12003C1F1200A29FA0AFADB
:10E3400009FA03F343EA0A0309FA01FABBF1000FE1
:10E350000FD04AEA080843EA0E0ECDF808B0407A1A
:10E360000028BFD0019C1C4301944AEA06060446DB
:10E37000B8E701254AEA0C0C1F430395EFE7084A6A
:10E3800000231360074A137007B0BDE8F08F00BF89
:10E39000D80A0120C80A0120E80A01204C660800BA
:10E3A000845F01203E670120F8B5394C394D636820
:10E3B00023F47F0323F47F43AB4223D04FF48072D6
:10E3C000002104F1080047F0E8FB334A00231370F2
:10E3D00023704FF080434FF44032C3F80429C3F850
:10E3E0001429C3F82429C3F83429C3F84429C3F8ED
:10E3F0005429C3F86429C3F874294FF47C12C3F874
:10E4000084296560254E264D0024D5E90001D6E912
:10E410000023C4F1200702430B430120A4F1200193
:10E4200000FA01F120FA07F73943A04002400B40FF
:10E43000134308D0E0B22FF07BFA204628F024FCEA
:10E44000204628F00FFD0134402CDED11549164836
:10E4500000220023C6E90023C5E90023C1E9002307
:10E460004FF40033C0F84833D0F80423920308D5A2
:10E47000C0F80833D0F844311BB14FF4A2714EF00C
:10E4800001FB0A4B00200021C3E90001F8BD00BFD9
:10E4900090670120AF0000AD80670120C80A01200D
:10E4A000D80A0120E80A012000400240F00A0120B9
:10E4B000F0B50B4687B000261446002A60D011F054
:10E4C000030760D10868414A90425CD16A464FF424
:10E4D000807049F0FCFA10B93D4823F05BF9DDE9A2
:10E4E0000035042CA5EB030536D0A30732D12368F1
:10E4F000384A934208D0384A934205D0374A93426B
:10E5000002D0374A934225D1012203A920461EF0AA
:10E510002DFC049BAB4202D0324823F093F99DF8C6
:10E520001410039C002240201BF0A0FB012801D006
:10E530002D48F2E7009B5A19B2F5807F02D92B488B
:10E5400023F05AF92A482A462146184447F0E5FAAA
:10E550000E2415E02748C0E73946284647F016FA4A
:10E56000009B5A19B2F5807F044604D820492A46F8
:10E57000194447F0D2FA2146284621F095F804467E
:10E58000204607B0F0BD002219464FF480701EF0FF
:10E59000F7FB042C054600F1010708D1B7F5807F91
:10E5A0009CBF134BC65C740044F00104E8E72046AE
:10E5B00020F01AFA4223FF22002104461BF0D4FA6D
:10E5C000B7F5807FBBD80A4BEC54C1E77C590800F3
:10E5D000304208006C5E080054560800705808006D
:10E5E000281C08005C2F08003B48080098320800EF
:10E5F00098670120D135080038B5084BD3E90045AC
:10E6000054EA050305D051F06DFA201A65EB0101BB
:10E6100038BD4FF0FF300146FAE700BFF00A012095
:10E6200070B52DED028B8AB00D46082000211646EC
:10E63000039347F0ABF9304B036005AB01932F4BCD
:10E64000039A0093044602232846314647F0C1FB53
:10E65000DDE90505B0F10E0218BF0122B5F10E0388
:10E6600018BF01239A4202D1254823F0EBF80E2867
:10E6700038D020F071F9B0EE408A51F033FAF8F753
:10E68000A9FFDFED207A07EE100A0E2DC7EE278ACC
:10E6900021D0069820F030FE05462FF067FE07A92E
:10E6A00033F018FF9DF8223001939DF8213000933C
:10E6B0009DF81F209DF820309DF81E10BDF81C000D
:10E6C00036F05CF8104B281A034407EE903AB8EE87
:10E6D000E78A38EE288AB4EEE88AF1EE10FA04D51B
:10E6E0000A48C2E79FED0A8AC7E7204684ED018AFF
:10E6F0000AB0BDEC028B70BD20670800D44209004F
:10E70000B62F080000007A4480BC92C7413108004F
:10E71000000000007FB50C46082000211546039339
:10E7200047F034F9094B036005AB0193084B039A9A
:10E73000009329460123204647F04BFB059840F201
:10E740003C4139F02DFE002023F024F894670800A6
:10E75000E442090008B5054B1B682BB1044A9342FB
:10E7600002D0044823F048F8004808BD6809012099
:10E77000A05D08007F31080008B5064BD3F8C03013
:10E780002BB1054A934202D0044823F035F80148E2
:10E7900008BD00BF68090120A05D08008C31080099
:10E7A0002DE9F843DFF8D4C0DCF800500446BDB1D1
:10E7B000686805F1080320F003000344DFF8C08017
:10E7C0002B48D8F80060002E14BFB6468646671C5A
:10E7D00004BFAEEB0304083C24B90020BDE8F88375
:10E7E000244BEBE7A007F8D1002914BF3046284698
:10E7F00044F0010908BB04F10807AEEB0300B8427E
:10E8000020DA002914BF2846304644F0010350BBEB
:10E81000002AE2D0184DD5F8A831002BDDD0012117
:10E82000384647F0BFF80028D7D0D5F8F830036055
:10E83000C5F8F80044F002040EE047684F4509D0DF
:10E840000068D7E751B127F00300AEEB0000C8F82D
:10E8500000000660002AEDD14460BFE71D60184645
:10E86000CCF80030F6E741689942F3D00068CEE773
:10E870000000042098680120505C0120805801208D
:10E880007458012013B54FF4C063019308B11128E7
:10E8900015D101A809F034FB0146134809F064FBC7
:10E8A000019B124A23F003030193A3F5C073934223
:10E8B00005D90F4830F05EFF4FF4C063019300228A
:10E8C000019811463EF079F8044648B9084830F0FE
:10E8D00051FF224621464FF4C0603EF06EF80446D8
:10E8E000204602B010BD00BF04E1080020BA0D00B0
:10E8F000BB34080070B58AB06846F8F781FB124C4B
:10E90000124E134D241A306800F580600022012158
:10E9100020443EF052F8A8B90246012104F5C8404F
:10E920003EF04BF84FF4C0430A4A2B600368136073
:10E9300053F8042C084922F003020A60074A1A60BF
:10E940000AB070BD3368EFE700000420D802012050
:10E950008C550120B45F0120B05F0120EF297801C0
:10E960000A4B1A6852B10A4B002808BF1A46002306
:10E97000D158814204D1064818447047044AF6E74A
:10E9800004333C2BF4D10020704700BF6C5F0120A2
:10E990006850012038B51C46084611464FF0021257
:10E9A0001BF03EF8206840F23C4139F0F9FC0021B0
:10E9B0000446082046F0EAFF074B036063790546EA
:10E9C0000BB94FF029F920794EF064F8207905F061
:10E9D000EFFE6C60284638BD1C68080008B540682A
:10E9E0003FF062FB004808BD3233D3C037B505465F
:10E9F00040683FF059FB314A4FF6FF73ADF80630DF
:10EA00000323C2F8F03501210023C2F8F435C2F81F
:10EA1000001519461A0102F1804202F5E042013365
:10EA2000082BC2F81415C2F81015F3D1234C4FF47B
:10EA30009053C4F818356B685B79C4F81435C4F882
:10EA400010350DF10603C4F82C360123C4F8303616
:10EA50002360D4F80031002BFBD018484FF48071AC
:10EA60004EF010F801236360144CD4F80431002BED
:10EA7000FBD012484FF482714EF004F80123A360DA
:10EA8000D4F81431002BFBD00C484FF48A714DF0B0
:10EA9000F9FF0023C4F80035BDF906209A42B8BF3B
:10EAA000ADF80630BDF90630181340EA830080B295
:10EAB000400040F0010003B030BD00BF00700040D6
:10EAC0001C4608B5084611464FF002121AF0A8FF7E
:10EAD00040F23C41206839F063FC0021042046F0FC
:10EAE00055FF034B0360FE21024822F05BFE00BF8E
:10EAF000946808006A4908002DE9F04F2DED088B55
:10EB00008FB009AB01936F4B009305231AF0B8FF48
:10EB10000021099825F0B6FC002106460A9825F048
:10EB2000B1FC044600210B9825F0ACFCE379012BE5
:10EB300005460AD1C379012B07D1A268012A04D95D
:10EB40008368012B01D99A4202D05F4822F07AFEF5
:10EB50006621B0684DF0F6FDE769217904903846EA
:10EB600002914DF065FDA368A0690299013B00FB8D
:10EB70000370B0EE40BA4DF05BFD0C98EF690E28C3
:10EB8000F0EE40BA26D1297938464DF051FD0D9866
:10EB90000E28F0EE408A20D1A868AB6929790138A7
:10EBA00003FB00704DF044FDE3690293EB690393AE
:10EBB000049BD6F81CB0D3F81C90B0EE409A4FF0EE
:10EBC000000AB36853450BD804980FB0BDEC088B0E
:10EBD000BDE8F08F1FF0C0FED9E71FF0BDFEE3E7F0
:10EBE000584631794DF024FDB369B4EEC0BAF1EE68
:10EBF00010FAB0EE408A9B4406DDC9ED008A0AF1A6
:10EC0000010A09F10409DCE7F4EEC0BAF1EE10FAEA
:10EC100002D589ED009AF2E7A7680023013FA269B7
:10EC20002179A7EB0308B8F1010F34D802980791B6
:10EC300002FB0300CDE905234DF0FAFC059A029B87
:10EC4000079902FB0730F0EE40AA4DF0F1FC039B60
:10EC5000D5F81880297905911A46069B08FB0320F0
:10EC6000F0EE409A4DF0E4FC039B059907FB083059
:10EC7000B0EE40AA4DF0DCFC38EE6A8A30EE4A0A6B
:10EC800079EEEA9A28EE008A88EE290A30EE0AAA7E
:10EC900089ED00AAB3E7CDE9061303EB5808029B00
:10ECA000059202FB08304DF0C3FCB4EEC08AF1EED1
:10ECB00010FADDE90521079B01D94346AFE7474636
:10ECC000AFE700BF88590900B83D08002DE9F047BB
:10ECD0002DED048B86B003AB0193504B00930323BF
:10ECE0001AF0CEFE0398002125F0CCFB8368012B9F
:10ECF000044640F29180C579012D02D0484822F0A7
:10ED0000A1FD007925F032FC81460498E6690E28C1
:10ED10005CD0002125F0B6FBC779012F054603D151
:10ED2000A26883689A4201D03E48E8E700799FEDE7
:10ED30003E8A25F01BFC82463046D5F81C80C84729
:10ED4000A36940461E44F0EE408AD047AB69B0EE5E
:10ED5000409A9844A368BB4218D8A368013B07EEC9
:10ED6000903AB6EE000AF8EE677A28EE008A67EE6F
:10ED7000887A17EE900A20F0030040F00200A0F11C
:10ED8000FF4006B0BDEC048BBDE8F0873046C847B5
:10ED9000A3694046F0EE409A1E44D04778EEA98A17
:10EDA00030EE499AF0EE486AD9EE286AAB6907EE70
:10EDB000907AB8EE677A9844C6EE877A0137B0EE5B
:10EDC000409A38EE278AF0EE698AC3E70598DFEDAE
:10EDD000168A1FF0C1FD3046B0EE408AC847A668CB
:10EDE000B0EE409AAE4202D828EE888AB5E72A46AD
:10EDF0002179E0694DF0E3FB07EE905A39EE009A75
:10EE0000B8EE677A39EE689A0135C9EE077AB0EE46
:10EE1000409A78EEA78AE5E70448B2E770590900FE
:10EE2000254608001346080000000000020080800C
:10EE30001E280CD03E280AD010F0010307D182070B
:10EE400007D10068044BC31A58425841704701204B
:10EE500070471846704700BFE81D0800F0B51B2832
:10EE60008DB006460C46154672D03CD80E2800F0F0
:10EE7000988004D8042840F2B180002430E01028A3
:10EE8000FBD115F0010206D115F00303F5D1296875
:10EE90006E4A9142F1D128461FF0A6FD0122054697
:10EEA00009A9204600F04EF9102E0A9F3DD1217984
:10EEB000002240201AF0DAFEA3686B4300FB03F146
:10EEC000E06846F07EFDA368E0606B43A360636882
:10EED0006FF31F2363601DB1013DC319002F34D1AF
:10EEE00020460DB0F0BD1D28CBD02428C5D101226D
:10EEF00003A9284647F00BFC00285CD0A10712D1DB
:10EF00002268534B9A420ED1012209A9204600F0F3
:10EF100019F901230093DDE90901DDE9032345F037
:10EF2000C5FC002858D11E24DAE7A1689DF82C0002
:10EF3000694300F05FF9C3680446CFE718460999B2
:10EF40003A4646F0EAFD03463B44013DF6D2C7E7A8
:10EF500009A90122204600F0F5F806A92846012259
:10EF60001DF004FF9DF82C10002240201AF07EFEB8
:10EF7000A168079EB6FBF0F6054631449DF82C00CB
:10EF800000F038F90446DDE90912C06846F0C5FD15
:10EF9000E0680A9B069906FB05F2184446F0BDFDA1
:10EFA0009EE70A682B4B9A423FF467AF29462046FA
:10EFB0003DF0C4FD94E7EA0702D5002022F0EAFB09
:10EFC000AB0703D12A68214B9A42F6D0284620F09D
:10EFD0004FFA0028A7D0F0E73E2481E7012209A9D3
:10EFE000204600F0AFF8012206A9284647F08FFB23
:10EFF000002898D00B9A012A21D05A2A21DC2032ED
:10F000000146089B012B1ED05A2B01DC2033014600
:10F010009342D2D123F00203642BCED0022E01D032
:10F020000029CAD0079B0093DDE90912069B3046F0
:10F0300048F0B7FC00280CBF1E243E2450E74222B3
:10F04000DDE70021DDE74223E0E700BFE81D08001F
:10F0500054560800705808002DE9F043012885B087
:10F0600006460F4608D08B0728D10B68274A9342E3
:10F0700002D0274A934221D1012201A9384647F004
:10F0800046FBD8B13146002240201AF0EFFD029B2A
:10F09000B3FBF0F100FB01F5AB4202D01D4822F0BA
:10F0A000D1FB304600F0A6F8019904462A46C06814
:10F0B00046F033FD204605B0BDE8F083384620F029
:10F0C00057FA054600B145102946304600F092F83F
:10F0D0000021044638461DF0A1FE4FF00008074607
:10F0E00038461EF041F803460028E3D025B91946FA
:10F0F00020463DF0EDFCF3E74246E16808F10109E6
:10F1000030461BF05BF9C846EAE700BF281C080040
:10F1100054560800BD360800012807B50B4606D135
:10F120000B68009340F61623019302206B460146BC
:10F130000022034821F022FA03B05DF804FB00BF6F
:10F140005C1E080070B50D460179044601F07F0190
:10F150001646402000221AF089FDE3682B60A26861
:10F1600042436A60227902F07F02AA602168094A5C
:10F1700091420BD194F90420002A01DBB20707D495
:10F180006268C2F3172200FB02332B60002070BDBF
:10F190000120FCE770580800074BC1E9003000234C
:10F1A000C1E90233054B02689A4202BF4368C3F3C8
:10F1B00017238B6008467047BC5E08007058080033
:10F1C00038B50D461C4611462846094A1AF028FC57
:10F1D000206821F0B7F9012D007804D1BDE838404E
:10F1E000002100F007B86168BDE83840FFF734BF80
:10F1F000040002007828F8B505460E4602D11148F1
:10F2000022F020FB0022014640201AF02FFD0021B1
:10F210000746102046F0BAFB0B4A0C4B0571012D36
:10F2200018BF1346036043686FF31F230446C0E909
:10F230000136002106FB07F046F0A8FBE0602046FF
:10F24000F8BD00BF583608006C5E08005456080030
:10F25000F8B50A79012A05460C460DD1194948F03E
:10F26000ACFAD4E90221284622F0D2FE28461649FB
:10F27000BDE8F84048F0A1BA144948F0AEFAA368D6
:10F28000002BF3D01249134F284648F096FA002677
:10F29000A368B34204D81049284648F08EFAE5E73F
:10F2A0001EB13946284648F088FA3246E16820798E
:10F2B0001AF0B6FD01220146284620F0A1FC0136D5
:10F2C000E6E700BFEC5D080080410900F85D08003A
:10F2D000035E0800665D0900B35609002DE9F0479A
:10F2E0000B4688B0044616460AB90025BCE011F06A
:10F2F00003058068DFF8009240F0CC800A68784F00
:10F30000BA4240F0C78002AA48F0E1FB10B9754844
:10F3100022F040FA2179042E01F07F012A464FF0B5
:10F32000400000F089801AF0A1FC16F003020546A7
:10F330004ED137680192384648F056FD6A4B019A23
:10F34000834238D13179402001F07F011AF08EFCE0
:10F35000A84202D0654822F075FA33684B45D6E9D9
:10F36000028A04D17368C3F3172305FB03AADDE9FE
:10F3700002072368E6683F1A4B45A8EB070729D127
:10F3800094F90430002BB0DA002FE3D16368C3F3A3
:10F39000172305FB036605FB08F2514605FB0060D9
:10F3A00046F0E3FB0399A2680298521A40446A436C
:10F3B00005FB016131E04E4B9F4209D1012DC9D1BE
:10F3C0002A4605A930461DF0D1FCDDE905A8CEE7A7
:10F3D00048489DE7002FDEDD6368B7EB132F0BD99C
:10F3E000A16839443046694346F0EBFA6368E0604F
:10F3F00067F31F23064663600298A268039940449E
:10F400003A44121A6A4301FB056105FB006046F0AD
:10F41000ACFB029805FB08F2514605FB006046F084
:10F42000A4FB6368C7EB132262F31F236360A36826
:10F430003B44A3600E2517E01AF018FC23684B45E7
:10F44000064615D12946102046F0A0FA054694E854
:10F450000F0085E80F00029A02EB112363F31F21CE
:10F460006960039B9B1AAB60284608B0BDE8F08733
:10F47000DDE902312079C91AFFF7BCFEDDE902326D
:10F48000E168D21A0546724306FB0311C06846F0D4
:10F4900044FBE9E7002219461DF072FC23684B4546
:10F4A000024611D16368042E00EB13220ED094F9AA
:10F4B0000430002BBFF619AF2079E168334600F025
:10F4C0007F001AF07BFFB5E7042EF5D12079E168C3
:10F4D00000F07F0008B0BDE8F0471AF0A1BC00BF03
:10F4E0007C59080030420800DDF20200113F08009C
:10F4F000281C0800D13508007058080010EE102AAA
:10F5000008B522F00043B3F17E5FB0EE406A12D33B
:10F5100019BF76EE467A9FED1F7ADFED1F7A9FEDD9
:10F520001F7A12BF87EE276AE0EE077AB0EE676AAD
:10F53000B0EE460A08BDB3F17C5F0BD2A3F5000321
:10F54000B3F1645FF4D320EE000AFBF777FBA0EE83
:10F55000066AEDE7B0EEC06AB7EE000A30EE466A22
:10F56000B6EE000A26EE000AB1EEC06AFBF766FBB3
:10F57000002AF0EE007AA0EE066A9FED090AA6EED8
:10F58000270A9FED066A36EE406AB8BFB1EE466ABA
:10F59000CEE700BF0000000000008003DA0FC93F83
:10F5A0006821A2B31FB58DED010A019B23F0004233
:10F5B000B2F18B4F00EE102A4FEAD3700BD319F043
:10F5C00091F9DFED1E7A30EE270A08B1B1EE400A5C
:10F5D00005B05DF804FB5B0014D5B7EE007AF0EEE1
:10F5E000476AE0EE006AF1EEE67A77EE807AC7EEDF
:10F5F000276AF0EE007AE0EE276AB0EE660A19F0AC
:10F6000071F9E2E7B2F1665F10D320EE007AF7EE0F
:10F61000006A37EE266AF1EEC67A77EEA67AC7EE72
:10F62000276A36EE800A19F0B1F8CEE7DFED047AEA
:10F6300070EE277ACDED037A039BC6E71872313F4F
:10F640000000807B1FB5044690B10E2810D00079D1
:10F6500040F0A7F960B94FF4E873039301A920467D
:10F6600003AB02AA15F0A6FA0399024822F0F2F8B9
:10F6700004B010BD3C290800F4EE400AF1EE10FA87
:10F6800010B5F0EE407A04D770EE207AB0EE670A3B
:10F6900010BD10EE902AB2F17E5F10EE103A03D149
:10F6A000BDE8104000F080B8940F04F0020444EA72
:10F6B000D37433F0004308D1022C59D09FED317A36
:10F6C000032C08BFF0EE477AE0E732F0004209D1A0
:10F6D000DFED2D7A9FED2D0A14F0010F18BFF0EE2B
:10F6E000407AD3E7B2F1FF4F10D1B3F1FF4F04F1ED
:10F6F000FF3407D1022C3ED8254B03EB8404D4ED14
:10F70000007AC3E7022C39D8224BF6E702F15061A8
:10F710009942DDD3B3F1FF4FDAD0A10703D503F14E
:10F72000506393420CD387EEA00AB0EEC00A00F0FB
:10F730003BF8012CF0EE407A04D1F1EE407AA5E7D7
:10F74000DFED157A022C0AD0002C9FD09FED130A12
:10F7500077EE807A9FED120A77EEC07A96E79FEDFA
:10F760000F0A77EE807A9FED0E0A70EE677A8DE7CA
:10F77000DFED0B7A8AE7DFED0B7A87E7DFED067ABC
:10F7800084E700BFDB0F49C0DB0FC93FDB0FC9BFF8
:10F79000D4560900E0560900000000002EBDBB331E
:10F7A000DB0F4940DB0F493F10EE102A22F00043E7
:10F7B000B3F1994F82B04FEAD2700ED3B4EE400A43
:10F7C000F1EE10FA07D69FED410ADFED417A0028ED
:10F7D00008BFB0EE670A02B070473E498B420BD8B3
:10F7E000B3F1665F5AD212F0FF4FF4D160EE007AA7
:10F7F000CDED017A019BEEE7374A9342F0EEC07AF5
:10F8000037D8A2F5D002934229D8F0EE006ABFEEB5
:10F81000007AA7EEA67A002377EEA67A87EE270A6B
:10F820005A1C60EE006A9FED2D6ADFED2D7ADFED48
:10F830002D5A26EEA67AE7EE067A9FED2B6AA7EE02
:10F84000876ADFED2A7AE7EE257A67EE877AE6EEB9
:10F85000267A60EE277A24D130EE670ABBE7B7EE4E
:10F86000007A77EEC76A77EE877A012386EEA70AD9
:10F87000D6E71F4A93420BD8F7EE086AB7EE007A34
:10F88000A7EEA67A022337EEE66A86EE070AC7E7F6
:10F89000BFEE007A87EE270A0323C1E74FF0FF335C
:10F8A000BEE7144A144902EB830201EB830393ED94
:10F8B000007A77EEC77A37EEC00AD2ED007A37EEDB
:10F8C000C00A002887D0B1EE400A84E7DA0FC9BF2A
:10F8D000DA0FC93FFFFFDF3EFFFF973F25AC7C3DBE
:10F8E0000DF5113E4712DABDA9AAAA3E98CA4CBE30
:10F8F000FFFF1B40FC5609000C570900F0B5002320
:10F90000DFF838C00C4E19460E27DCF80020934271
:10F9100001D30E20F0BD346804EB03124FEA031E3E
:10F920009568854208BF44F80E1003F1010304BF37
:10F93000C2E90117D160E8E7AC500120B4500120C2
:10F940002DE9F04387B0084611461A4602AB0193F1
:10F950002B4B0093042346F03CFA40F272210298AC
:10F9600038F01EFD40F297518046039838F018FD9C
:10F970004FF435710746049838F012FD0021064611
:10F98000282046F013F81F4B03601F4B9DF814907E
:10F990001D68044615B11D4821F02EFF186098F827
:10F9A000040004F005FF387904F002FF307904F018
:10F9B000FFFE174B98F8042084F82120C3F8642533
:10F9C0003A7984F82220C3F86825327984F8232014
:10F9D000C3F870250122C3F80455C3F80855C3F8CD
:10F9E0000C25C3F81025C3F81C25C3F82055C3F80F
:10F9F000249533F07FFB204607B0BDE8F08300BFBD
:10FA000008430900146A0800785801207628080085
:10FA10000050024010B5044690F823003EF03EFB33
:10FA20000A4BD3F8082142B194F826206FF3410223
:10FA300084F826200022C3F8082194F8263013F019
:10FA4000020F14BF3E201E2010BD00BF0050024018
:10FA500010B5044690F823003EF020FB0C4BD3F881
:10FA6000082142B194F826206FF3410284F8262041
:10FA70000022C3F8082194F826309A0701D400F038
:10FA800009F843F0080384F826300E2010BD00BFAB
:10FA90000050024008B5014821F0AEFE612D08007B
:10FAA0002DE9F04F2DED028B0D4689B055F8044B32
:10FAB0000392064694F823003EF0F0FA06AB019359
:10FAC0007E4B039A009329460223701E19F0D8FF3B
:10FAD0007B4B069DD3F808219DF81C1042B194F889
:10FAE00026206FF3410284F826200022C3F8082163
:10FAF00094F826309E070BD5714A0123536094F881
:10FB0000263043F0040384F826302023C2F808335B
:10FB100094F82630656061F3041384F82630284693
:10FB20003DF051FD08EE100A28463DF0FFFC04F1BF
:10FB30002403C00884F82500019305AB28460093F0
:10FB40000DF112020DF1130301213DF01AFD9DF894
:10FB500013309DF812205A4F5A49DFF878915B0113
:10FB600043EA821394F8262003F0600322F0600237
:10FB7000134384F8263094F82530013B18BF012345
:10FB8000C7F81C3594F824305D1E6B424FF000021C
:10FB90006B41C7F82835B7EE007A104690461646F6
:10FBA000D7F81C35012B01D18B794BB3464DF8EEBC
:10FBB000486A4FF0000CB1F9043099FBF3FE6B6812
:10FBC0009EFBF3F307EE903AF8EEE77AD5F800B033
:10FBD000D1F800A076EEE77A0CF1010CF0EEE77AAE
:10FBE00087EEA66A0835B4EEC76AF1EE10FA41BF97
:10FBF000B0EE467A1A465846D046BCF10B0FDAD121
:10FC00000136092E01F10801CAD12D4DC5F818851C
:10FC1000C5F8140594F8240094F82530628313FB8A
:10FC200000F318EE100A584300014FF47A73B0FB4A
:10FC3000F3F0033020F0030080B20021208345F070
:10FC4000A5FE0021A060208B45F0A0FEE06060686A
:10FC50003DF0ABFC94F8263023F00E0343F0020392
:10FC6000002684F826302046C4E9046684F8206023
:10FC700015F014FD238B154A9B08C5F8503520213B
:10FC80000123C5F80413C5F800352B60D2F8040130
:10FC900080060BD5D5F8140140B1C5F81461C2F83F
:10FCA00084110B4A106838B115F0F8FC0E2009B029
:10FCB000BDEC028BBDE8F08F6B60F7E728430900CD
:10FCC00000500240904309003843090000E100E081
:10FCD000785801200048E80110B5044690F8230048
:10FCE0003EF0DCF9064A0123536094F8263043F0D5
:10FCF000040384F826302023C2F808330E2010BDF8
:10FD00000050024038B5084B1B6800220446C3F877
:10FD10000025FF2500792DF00BFE607925712DF06F
:10FD200007FE65710E2038BDDC0201202DE9F0438D
:10FD30002DED028B8BB0084611461A4603AB01939A
:10FD40003F4B0093072346F044F840F2A521039867
:10FD500038F026FB40F2D7210646049838F020FB05
:10FD600000210546082045F011FE364B03609DF842
:10FD70001870DDF814807A07044602D0324821F06A
:10FD800061FD089B5B0701D03048F8E709989DF8B2
:10FD90001C9088B11EF0E0FDB5EEC00AF1EE10FA3D
:10FDA000B0EE408A06D4F7EE007AB4EEE70AF1EE40
:10FDB00010FA03DD2648E2E79FED268A307904F049
:10FDC000F7FC287904F0F4FC84F80690327922716B
:10FDD0002B796371B8F57A5F01D01F48CFE7102FF8
:10FDE00001D01E48CBE71E4B9FED1E0A1B681E4923
:10FDF000C3F840256279C3F8442528EE008A4FF005
:10FE00000462C3F804250022C3F82025FCEEC87A5A
:10FE10002822C3F81825C3F81C250122C3F80025A1
:10FE200017EE900AC3F86015C3F864251A601DF038
:10FE300037F820460BB0BDEC028BBDE8F08300BF65
:10FE4000D8430900CC6A0800974808002C2E080007
:10FE5000EC2B0800AE47E13D2042080004420800B8
:10FE6000DC02012000007A449C55012038B5084B83
:10FE70000C681B680022C3F800252079FF252DF0AF
:10FE800057FD607925712DF053FD65710E2038BD49
:10FE9000DC0201202DE9FF4105460E462B79FF2BA0
:10FEA000104601D12CF03EFE40F2BE3119F0C8FEE2
:10FEB00040F2BE320021044645F0ADFFB30706D143
:10FEC00032682F4B9A4202D12E4821F063FC022265
:10FED00001A9304646F01BFC00284FD09DF80C10BD
:10FEE000029E0022402019F0C1FEB6FBF0F0A042B5
:10FEF00002D2254821F0A6FC039B482B01D02348C1
:10FF0000F8E7DFF89480019ED8F800300122C3F8AA
:10FF10000825C3F86065C3F864451D4B4FF448508D
:10FF200043F001039847D8F800300022C3F80821B5
:10FF3000184AC3F8602501223746C3F86425D8F86B
:10FF40000030D3F808316BB106EB4406B7420CD150
:10FF5000AB7983B124F00104640044F0010004B0E3
:10FF6000BDE8F08100F00CFDE9E73B88A3F5004314
:10FF700027F8023BEAE724F00304EDE70E20EEE762
:10FF80001CAF0800224A08005C28080071390800EC
:10FF9000304409009C550120DC02012070B588B076
:10FFA000084611461A4605AB01931C4B00930323E8
:10FFB00045F00FFF0021142045F0E8FC184B0360CA
:10FFC00004460122059802A91CF0D0FE049B622B76
:10FFD00010D0A3F168014A424A4123F02001482988
:10FFE0000AD0422918D0012B07D00E484FF42271B5
:10FFF00021F030FC0122F0E702239DF81800079958
:020000023000CC
:10000000039D029EA073DB0020466660237362732B
:10001000A560216108B070BD0123EEE7104409001E
:10002000986B080065310800F0B51E460F4685B094
:1000300011463846204A19F0F3FC34681F4B234020
:10004000062B05D0A3070AD122681D4B9A4206D180
:1000500021461C4844F2267246F024F8044600214A
:10006000402045F093FC184B036014F00302054652
:1000700003D12168154B994202D0154821F0CEFBDF
:10008000012F16D97068022201A91CF06FFE4FF4EF
:1000900022730298019E4FF48062082119F094FDAA
:1000A000034628463246214604F06AFF284605B03A
:1000B000F0BD13461646F4E7040002000F0080FF6F
:1000C0005C1E0800545A0800946C08001CAF08001D
:1000D000873A08002DE9F04788B0084611461A46CD
:1000E00002AB0193374B0093062345F072FE40F2BA
:1000F0008E53FF220121029819F036FD40F29A2317
:10010000054602220498012119F02EFDDDF81C801D
:10011000B8F1000F064604DC40F2BD41012019F0A1
:100120001BFD059F082F04D0102F02D0264821F078
:1001300089FB05F10B000021800045F027FC234BD3
:100140000360044603989DF818A0C0088000E06092
:10015000002145F01BFC5FFA85F9FFB2F6B2606042
:1001600018B9A060E06818F03DFCE068002145F097
:100170000DFCA06008B96060F4E7277484F824904F
:1001800004F12C07DFF84890E674C4F8148084F872
:1001900012A00026B846AE4209DB94F8240041467E
:1001A0001FF09AFCA062204608B0BDE8F08700234B
:1001B0001A461946484600F061F8013647F8040B24
:1001C0004460E8E7384409006D360800A06D080077
:1001D000EC45090070B50D4688B055F8044B039204
:1001E000064620463DF0AAFF05AB01930E4B039A4D
:1001F000009329460323701E19F042FC94F8242032
:100200009DF818309A4203D840F28D5019F030FC16
:1002100004EB83049DF81C20E06A059904F05CFF60
:100220000E2008B070BD00BFE844090070B50D464F
:1002300086B055F8044B0392064620463DF07EFFFB
:1002400005AB01930C4B039A009329460123701EC2
:1002500019F016FC94F824209DF814309A4203D823
:1002600040F28D5019F004FC04EB83040022E36A91
:100270000E209A6006B070BDA844090008B5084673
:100280001146002219F0CCFB00211C2045F07EFB1A
:10029000034A0260002282604FF40042028308BDDC
:1002A000EC4509001FB502AB51F8044B0193074B15
:1002B00000930138022319F0E3FB20469DF80C203F
:1002C000029904F009FF0E2004B010BD004509009A
:1002D0001FB503AB0193134B51F8044B0093013846
:1002E000012319F0CDFB03981EF036FBF7EE007AE0
:1002F000B4EEE70AF1EE10FA04DCB5EEC00AF1EE56
:1003000010FA02D5084821F09DFADFED087A20EEB8
:10031000270A0E20BCEEC00A10EE103A238304B068
:1003200010BD00BF68440900033F080000000047FB
:100330001FB503AB0193064B51F8044B00930138F2
:10034000012319F09DFB00230E20A36004B010BD13
:10035000B044090073B58669069D04461EB92E6037
:10036000022002B070BD0029016B296090F93F1096
:1003700008BF00228A4212D190F9401000EB81019F
:1003800012B2496A01EB42021A60FF2380F83F3043
:100390002A68436C03EB520343640120E1E790F8C1
:1003A0003C10B1FA81F1490980F83C1080F8401006
:1003B000C2F1010200EB810180F83F204E6A1E600D
:1003C00045F076FC204645F056FC38B9286094F894
:1003D0003E30002B14BF00200220C2E7D4E90713EF
:1003E000A2696068C91A1A4401910092334601AAB1
:1003F0006946F8F7F1FDE369019A9B1A236210B18F
:1004000000202860ADE72A68636C03EB5203636445
:10041000204645F04DFC204645F02DFC236AB3F5FF
:10042000007F054606D3044B04F10800C4E90234FA
:1004300000F086FA284694E7BF5D0700F0B51E4637
:100440000F4685B0114638461B4A19F0E9FA346860
:100450001A4B2340062B05D0A3070AD12268184B5C
:100460009A4206D12146174844F2267245F01AFEF8
:1004700004460021482045F089FA134B036014F02C
:100480000302054603D12168104B994202D010485F
:1004900021F0C4F9012F0DD90222706801A91CF0C6
:1004A00065FCDDE901232846214604F067FE284665
:1004B00005B0F0BD1346F6E7040002000F0080FF10
:1004C0005C1E0800545A0800746F08001CAF080036
:1004D000873A080038B50446406A3DF017FE94F8A4
:1004E0003C00236B9FED120A04EB80045D08626AF6
:1004F00023F001031344934210D14EF08AFD07EE1E
:10050000905AF8EEE77AC0EE277A17EE900A20F0BC
:10051000030040F00200A0F1FF4038BD32F9021B99
:1005200007EE901AF8EEE77AA7EEA70AE3E700BF16
:100530000000000013B50446406A01913DF0E6FD5D
:100540000199064844F2267245F0ACFD014620466A
:1005500004F060FE0E2002B010BD00BF545A080027
:1005600038B50C460546406A3DF0D0FDA30703D1DF
:100570002268064B9A4202D0054821F04FF92846DE
:10058000214604F047FE0E2038BD00BF1CAF080016
:10059000873A0800F0B587B0084611461A4603AB03
:1005A00001932F4B0093032345F013FC4FF46F711D
:1005B000039837F0F5FE40F2A4410746049837F05F
:1005C000FBFE00210646242045F0E0F9254B0360A0
:1005D000254BBDF81450D3F8002512F00102044653
:1005E00017D003F5A043D3F80015C80711D503F5BC
:1005F0008053D3F80025D1070AD503F53043D3F84B
:100600000025D2072AD500231848A36021F0F4F86A
:1006100002221749A3608A5C22770022C3F80C25C6
:10062000A3680122C3F81025A2683B792376C2F89B
:100630006035387904F0BCF83EB1A268337963764E
:10064000C2F86835307904F0B3F8A3682D0A0122A6
:100650002046A582C3F8002507B0F0BD0322D8E7E5
:10066000704409009870080000C0014075470800F8
:10067000963E0900F0B50D468BB055F8044B039239
:100680000646A0683DF03DFD08AB01938A4B009300
:10069000701E2946039A022319F0F2F92046089D9C
:1006A0009DF824603EF042F810B120463EF049F833
:1006B000656084F8206028463CF085FF06462846A1
:1006C0003CF034FF0DF11303C008E076019305AB55
:1006D00004F1220200212846009304F121033CF09A
:1006E00050FF28463CF02EFF059DA0762846ADB26F
:1006F0004FF422724FF6FF71AD0019F051FA00214C
:10070000284645F043F994F82210E06019B92846CC
:1007100045F03CF9206106F574452335B5FBF6F547
:1007200006FB05F35D0805F5740505F51055B5FBE9
:10073000F3F56A08A16802F5740303F51053B3FBDF
:10074000F5F202EB5602B2FBF6F3013BC1F8483575
:10075000A268C2F828356B1EE382A368C3F8085567
:10076000A3680122C3F8142560683CF01EFF534AB9
:100770000023114652F8040B00283AD141F82340D7
:1007800032F0B8FC0023A377A3680422C3F8002248
:100790006068E56807AA06A93CF0E0FE02282CD1B3
:1007A00020463DF0CEFFA368D3F82025C3F84025AE
:1007B000A368D3F82425C3F84425A2680023C2F80F
:1007C0000831A268C2F80C31A268C2F81031A268E0
:1007D000C2F81431A268C2F80431A2680C21C2F830
:1007E0000413A16801220E208A606277E3770BB0C0
:1007F000F0BD0133042BBDD1C4E7E67EA37E079A8A
:10080000B2FBF6F2012EB2FBF3F2E68A94F8213045
:1008100005EB820130D1002B14BF4FF0800C4FF05C
:10082000000CA94214D8D4E90231C3F82015A368FA
:100830005200C3F8242594F82030002B35D1A3684A
:100840000028B0D10322C3F800220123A377AAE72E
:10085000069B5F1C06971B786344DBB22F467343ED
:100860001B0A27F8023B94F81AE0BEF1010F06BFFD
:1008700004353B803D46D4E7002B069F14BF4FF460
:10088000004C4FF0000CA942CDD937F8023B63442D
:100890009BB273431B0C2B8094F81AE0BEF1010F3E
:1008A0000ABF6B8002350435EDE700287FF47BAF8B
:1008B00060683CF07AFE76E7B84409004C500120AD
:1008C00010B50C4C206888B10B4B1B687BB94FF0FE
:1008D00005F923689842236836BFDB43C01AC01865
:1008E00040F2EE23984294BF0020012010BD00206A
:1008F000FCE700BF7C580120A450012008B50B4B39
:100900001B6893B90A4B1B787BB14FF0E7F8094B92
:1009100018601A6812B91A6801321A60064B01226F
:100920001A70064B03F16C025A6208BDA4500120F4
:10093000F56601207C580120F6650120505C0120FD
:1009400010B5044607F032F9E3681BB90A4A11688A
:10095000A14203D1BDE8104007F03AB9A360074BAC
:100960001968E160196809B119688C60116801B9EA
:1009700014601C60EEE700BFB0500120B8500120A9
:10098000F7B5134E33680BB3124D07F00FF92C78FF
:1009900024B103B0BDE8F04007F01AB90E4A0123B4
:1009A0002B703368346014600BB92B70F1E7D3E916
:1009B00000609F680190C3E9024407F009F90EB195
:1009C0000198B04707F0F2F83B46EDE703B0F0BD01
:1009D000B05001201C670120B850012008B51EF05E
:1009E00053F8C188034897290CBF4222972220F070
:1009F0001DFF00BF233708000749002251F832309D
:100A0000834203D801EBC202506870470132002BC9
:100A1000F4D11846704700BF983D0900F0B587B083
:100A2000084611461A4602AB0193224B0093042359
:100A300045F0CFF940F2C641029837F0B1FC4FF4CF
:100A400099610746039837F0ABFC00210646202049
:100A500044F09CFF184B0360DDE904238361174BCE
:100A60009A4288BF012300F1040598BFB3FBF2F35B
:100A700004464361394628463EF0FAFC48B904F181
:100A80000C07314638463EF0F3FC28B128463DF0CD
:100A9000F2FD204607B0F0BD0122114628463EF087
:100AA0004DFD0122114638463EF048FD20464EF0ED
:100AB000A9FBEEE7C84409003C71080020A107002B
:100AC00070B50C4688B054F8045B0392064628467D
:100AD0003DF03AFB28463DF043FB04AB0193094B44
:100AE000039A00932146701E042318F0C9FF079B48
:100AF00000932846DDE9052304992CF0A9FA0E207D
:100B000008B070BD4845090070B50C4688B054F86F
:100B1000045B0392064628463DF016FB28463DF04E
:100B20001FFB04AB01930A4B039A00932146701EEE
:100B3000042318F0A5FF01230193079B0093284687
:100B4000DDE90523049950F09FFB0E2008B070BD2D
:100B50008844090070B50C468CB054F8045B0392CD
:100B6000064628463DF0F0FA28463DF0F9FA05AB76
:100B700001930E4B039A00932146701E072318F031
:100B80007FFF00230193099B0093DDE90512089B79
:100B9000284650F079FB0B9B009328460A9B079A46
:100BA00005992CF055FA0E200CB070BD10450900C7
:100BB00070B50C4688B054F8045B0392064628468C
:100BC0003DF0C8FA28463DF0DBFA04AB01931D4B1B
:100BD000039A00932146701E042318F051FF4FF42E
:100BE000896301220021059818F0BEFF40F23943C5
:100BF000012200210446069818F0B6FF4FF41E7338
:100C0000092208210646079818F0AEFF04990E4AFB
:100C1000B2FBF1F301FB13228AB9EB6104F001048A
:100C200095F8203006F00106A40044EAC60423F03B
:100C30000C031C430E2085F8204008B070BD013322
:100C4000EBE700BF5846090020A107002DE9F0415D
:100C500086B0084611461A4603AB0193374B009302
:100C6000032345F0B6F84FF42971039837F098FB49
:100C70004FF47F718046049837F09EFB40F2EF31CD
:100C80000646059837F098FB00210746242044F0DB
:100C90007DFE05462A4B45F8043B0446414628465E
:100CA0003EF0E6FB024620B14FF42971254820F0C2
:100CB000D1FD94F820102846C1F380013EF03EFC9F
:100CC000BEB104F10C08314640463EF0D1FB02466D
:100CD00028B128463DF0CFFC4FF47F71E6E794F849
:100CE000203043F00203014684F8203040463EF0B5
:100CF00025FCB7B1394604F114003EF0B9FB50B100
:100D000028463DF0B8FC1EB104F10C003DF0B3FCE8
:100D100040F2EF31CAE794F8203043F0010384F841
:100D200020300523E36194F82030204623F00C03A3
:100D300084F8203006B0BDE8F08100BF0846090005
:100D400034720800772A08002DE9F04F0D468FB065
:100D500055F8044B0392064620463DF0FBF9204629
:100D60003DF00EFA0AAB01934B4B039A00932946D0
:100D70000423701E18F084FE0A98022207A91BF0B3
:100D8000F5FF9DF824100022402018F06FFF0B9B08
:100D900006930646089B0C99B3FBF0F305AA06A838
:100DA00005934BF05AFE069D0598754346430695FC
:100DB0000596002E55D09DF83430039394F82030DA
:100DC000DDF81C80DF0702D4344820F03BFD980793
:100DD000E76903D5206900213EF09DFB464408EBFE
:100DE000050A04F1140B3544039E4FF008094FF037
:100DF000000894F82030990703D52069F1093EF0E6
:100E00008AFB94F820100A072FD4384625F032FFC9
:100E100094F82010A068C1F3800181F0010101F075
:100E200001013EF078FB58463EF037FB94F8201065
:100E300040EA48000B075FFA80F823D4384625F0D3
:100E400019FF94F82010A068C1F380013EF063FB05
:100E50007600B9F10109F6B2CBD10AF8018B5545FC
:100E6000C2D10E200FB0BDE8F08FC1F3800181F038
:100E70000101A06801F001013EF04DFB384625F06C
:100E8000F9FED0E7A068C1F380013EF044FB38468C
:100E900025F0F0FEDCE700BF20460900922C080098
:100EA0002DE9F0430D468DB055F8044B03920646EC
:100EB00020463DF04FF920463DF062F909AB019321
:100EC0003C4B039A009329460323701E18F0D8FD6B
:100ED0000998012206A91BF049FF9DF82010002265
:100EE000402018F0C3FE0A9B05930546079B0B990B
:100EF000B3FBF0F304AA05A804934BF0AEFD059BE9
:100F000004986B43454305930495002D37D094F81E
:100F100020200698920702D4274820F093FC05442D
:100F2000E76900EB03081D4418F8016B4FF008094E
:100F3000F10920693EF0EFFA94F820100B0722D453
:100F4000384625F097FE94F82010A068C1F3800180
:100F500081F0010101F001013EF0DDFA384625F093
:100F600089FE94F82010A068C1F380013EF0D3FA06
:100F70007600B9F10109F6B2DAD1A845D4D10E2034
:100F80000DB0BDE8F083C1F3800181F00101A068DC
:100F900001F001013EF0BFFA384625F06BFE94F8EF
:100FA0002010A068C1F380013EF0B5FA384625F064
:100FB00061FEDDE740460900982C08002DE9F04F5E
:100FC0000D4695B055F8044B0392064620463DF079
:100FD000C1F820463DF0D4F80EAB0193584B039A6C
:100FE000009329460623701E18F04AFD0E98012230
:100FF0000BA91BF0BBFE9DF834100022402018F016
:1010000035FE109B1199079305460C9BB3FBF0F33B
:1010100006AA07A806934BF020FD0F98022208A904
:101020001BF0A4FE9DF828100022402018F01EFEA0
:10103000129B05930646099B1399B3FBF0F304AA90
:1010400005A804934BF009FD069B059A0498079F99
:101050006B43724346436F43B3420797069305922F
:10106000049602D0374820F0EDFBABB194F8200095
:101070000B9D0899860701D5C00701D43248F2E7D5
:101080000B441344E669039301EB02082F4404F177
:10109000140B039B984503D10E2015B0BDE8F08FCB
:1010A00017F8015B4FF0080A4FF00009E9092069C1
:1010B0003EF031FA94F820100A072AD4304625F081
:1010C000D9FD94F82010A068C1F3800181F00101DE
:1010D00001F001013EF01FFA58463EF0DEF994F8A7
:1010E000201040EA49000B075FFA80F91ED4304611
:1010F00025F0C0FD94F82010A068C1F380013EF0F7
:101100000AFA6D00BAF1010AEDB2CFD108F8019BDD
:10111000BFE7C1F3800181F00101A06801F0010186
:101120003EF0F9F9304625F0A5FDD5E7A068C1F3FA
:1011300080013EF0F0F9304625F09CFDE1E700BF6C
:1011400078460900AA3608006C4A08002DE9F041EB
:101150000E2A064686B00846174602D1304820F0CF
:10116000F5FA8A0706D109682E4A914202D12E4823
:1011700020F010FBC30716D5B488431093FBF4F599
:1011800004FB15339CB2ADB2042F2AB20FFA84F8D7
:1011900020D1414630463EF06EFA400040F001005A
:1011A00006B0BDE8F08103AA022145F0FAFD039BD9
:1011B00018681DF019FC039B84B258681DF014FCDC
:1011C000B388A34285B202D9F388AB42DCD8174872
:1011D00020F0CCFA384601921DF006FCB37B019A50
:1011E00030FA03F3074602D0114820F02BFB03A985
:1011F000304601340135ADF80E2001920593ADF86B
:101200000C80ADF81040ADF812500DF0B9F8304632
:10121000019A3B46414640F0ADFE0E20C0E700BFBC
:10122000DB4908007C590800722F080016430800AB
:101230002B4308002DE9F04F2DED028B8FB008AB4A
:1012400001939E4B0093062318F01AFC9C490898C2
:1012500040F2EB2218F0DCFC994940F2FC420446D3
:10126000099818F0D5FC9649804640F2FD420A984C
:1012700018F0CEFC81460C980E2828D01DF06CFB8F
:10128000F0EE408A0D980E2824D1B7EE008A38EE91
:10129000688A0B9D8B494FF42C72284618F0B8FCD5
:1012A0006268D8F8043095F804A09A420CD1A37B68
:1012B00098F80E10994207D1D9F804108A4203D148
:1012C00099F80E209A420AD07F4820F0BBFAF6EE39
:1012D000008AD7E71DF040FBB0EE408AD9E70AF15B
:1012E000FF32082A0ED8DFE802F0090D090D090DBA
:1012F000090D0500082B07D07448E6E7102B03D032
:101300007348E2E77348E0E7A388ADF81830002699
:10131000E388059605A92046ADF81A3007960DF02A
:101320002FF8F0EE687AFEEECC7ABAF1090F17EEDC
:10133000907AF0EE487AFEEECC7A17EE905A3ED1D3
:1013400032464FF67F761AE0A089B8F80CC0B9F89B
:101350000CE002FB00F3A06800EB8300D8F8083033
:1013600002FB0CFC03EB8C0CD9F8083002FB0EFEE0
:1013700003EB8E0E0021A388994209DB0132E3883A
:101380009A42E1DB0E200FB0BDEC028BBDE8F08F7E
:101390001EF801301CF801A06B4307FB0A33B3426F
:1013A0000BDC13F1800A48BF03F27F1A4FEA2A23AD
:1013B00023EAE37343540131DDE7FF23FAE70AF040
:1013C000FB0E3246E3889A42DCDAA189A368B9F8B9
:1013D0000CB0514303EB8103B8F80C100293D8F81A
:1013E0000830514303EB81030393D9F8083002FB23
:1013F0000BFB03EB8B0B4FF0000AA3889A4501DB34
:101400000132DFE7039B3BF81A1033F81A60BEF194
:10141000030F03D176BA49BAB6B289B201F4784360
:1014200006F478406B4307FB00332B4883423DDAD8
:1014300013F5F84348BFFF331B1223EAE37303F4A9
:10144000784301F4FC60684306F4FC6C07FB0C0C69
:10145000224884452DDC1CF57C7048BF0CF2EF401F
:10146000001220EAE07000F4FC6001F01F01694303
:1014700006F01F0607FB061641F6F0718E421BDCD4
:1014800016F10F0148BF06F58771091221EAE171D3
:1014900018430843BEF1030F80B201D140BA80B2B5
:1014A000029B23F81A000AF1010AA6E74FF47843D9
:1014B000C7E74FF4FC60D8E71F21E9E74047090080
:1014C000C886080048880800A1480800EB290800E1
:1014D000052A08003E3308000085F7000FDD0700ED
:1014E0002DE9F04F97B00FAB0193484B00930723C2
:1014F00018F0C6FA46490F9840F2762218F088FB99
:101500000122044609A910981BF030FC139E149D7B
:10151000DDE9118A721C08BFA6886B1C08BFE5882C
:10152000B8F1000F0CDBBAF1000F09DB464507DB11
:10153000554505DBA388B34202DBE388AB4202DA00
:10154000344820F013F9A5EB0A039DF82C10A6EB04
:101550000807002240205F4318F088FB0A9BB3FB7A
:10156000F0F9159B04900E2B039307D018461DF03D
:101570003BFA05904F4504D92748E2E7002305933D
:10158000F8E7A37B099F4FF0010909FA03F909F174
:10159000FF330693D1464D4534D1002320460CA994
:1015A000ADF83080ADF832A0ADF83460ADF836500B
:1015B0000E930CF0E5FE0E2017B0BDE8F08F049BF3
:1015C000022B19D0042B1AD017F8013B03990E29CE
:1015D00002D00599994208D0069907920B402046FF
:1015E0000FFA8BF140F0C6FC079A0BF1010B5E4538
:1015F000E5D109F10109CEE737F8023BE6E757F8F4
:10160000043BE3E7C3460FFA89F2F0E7004809001C
:10161000C886080016430800AF3C080070B588B0C3
:1016200004AB0193274B0093042318F029FA2649B1
:10163000059840F2FB4218F0EBFA2349044640F2C9
:10164000EB22049818F0E4FA079E204905464FF46F
:101650001272304618F0DCFA3379069E1C49039367
:101660004FF4A062304618F0D3FA606869683279A6
:10167000039B884202D0174820F0D0F8A97B10299C
:1016800003D0012901D01448F6E7511E082910D8CB
:10169000DFE801F0050F050F050F050F0A00A17B1C
:1016A000102908D00D48E7E7A17B082903D00C4892
:1016B000E2E70C48E0E72846214603F0EDFD0E2066
:1016C00008B070BD38480900C8860800B472080028
:1016D0004888080065360800C0440800D444080063
:1016E000E6440800F846080030B589B003AB019322
:1016F0001A4B0093052318F0C3F91949039840F2D7
:10170000EB2218F085FA817B069B01228A409342E6
:1017100002D3144820F096F8079C6FF000418C42E9
:1017200003D0A24201D81048F4E7BDF91010BDF96A
:101730001420002902DB8588A94201DB0B48E9E778
:10174000002AFBDBC588AA42F8DAA34202D0009443
:101750003DF009F80E2009B030BD00BFA0470900D8
:10176000C8860800494708003C360800F4420800D3
:1017700000B589B002AB01930F4B0093062318F01C
:101780007FF90298079A817B01238B409A4202D30A
:101790000A4820F057F8BDF9183001920093BDF9BE
:1017A0001020BDF91430BDF90C103DF0DAF80E2010
:1017B00009B05DF804FB00BF70470900F44208005F
:1017C000F0B58FB008AB0193274B0093062318F0B8
:1017D00057F9089E0D9FB37B01229A40974202D38E
:1017E000224820F02FF80998BDF92810BDF92C20C7
:1017F000BDF93030ADF80800002402A8ADF80A1099
:10180000ADF80C20ADF80E30049440F00CFBB3881A
:10181000ADF8183002AAF388059405A91046ADF872
:101820001A30079440F010FB02A930460CF0A8FDD6
:10183000BDF90840BDF90C30A34202DC0E200FB008
:10184000F0BDBDF90A50BDF90E30AB4202DC0134E7
:1018500024B2EFE72A463B4621463046013540F0A8
:1018600089FB2DB2EFE700BF10470900F4420800E2
:101870002DE9F0432DED028B9FB011AB0193474B47
:1018800000930D2318F0FCF8DDE91145A27BAB7B3A
:101890009A4202D242481FF0D5FFA1881398490806
:1018A0004FF07AF8E1880646490814984FF074F82A
:1018B000A9880746490817984FF06EF8E9888046CE
:1018C000490818984FF068F80FAB02930DF13E03EA
:1018D0000193169B159900930DF1420210AB8146BE
:1018E00020464EF0B2FF0DAB02930DF1360301938B
:1018F0001A9B0093284619990EAB0DF13A024EF04F
:10190000A4FF1B980E2842D01DF026F8F0EE408A66
:101910001C980E2808D01DF01FF8B5EEC00AF1EE95
:1019200010FAB0EE408A01D5B7EE008A1D980E2855
:1019300030D01DF059F80022BDF934300993BDF9BB
:1019400036300893BDF938300793BDF93A30CDE908
:101950000593BDF93C300293BDF93E300193BDF9CA
:1019600040300093CDE90A02CDE903582046BDF985
:101970004230F0EE480AB0EE680A3A4631463DF091
:10198000B6F80E201FB0BDEC028BBDE8F083DFED92
:10199000058ABDE701220020CEE700BFA846090066
:1019A000B34408000000000030B58DB005AB0193D2
:1019B0001F4B0093072318F063F81E49059840F267
:1019C000762218F025F9089C0699631E012B05D98B
:1019D000042C03D0184821461FF03CFF079B022B24
:1019E0001FDC002B20DD9DF82C2002929DF8282082
:1019F00001929DF824200092224603F081FD0E20E2
:101A00000DB030BD0122AA400C4D1540002DEAD189
:101A1000D20209D5012CE6D00948182221461FF030
:101A200019FF1D1F1C2DEDD906481946D4E700BF2C
:101A3000C8470900C8860800103E080011100010B1
:101A4000FA3D0800D93D080038B50C4BD3F80031F9
:101A500004460D464BB901210C2043F097FF2A465E
:101A60002146BDE8384000F00BB89A68A24202D186
:101A70005A68AA4201D01B68ECE738BD505C0120CF
:101A800070B5094CD4F800512B462BB9C0E900526F
:101A90008160C4F8000170BD9E688E4202D15E680C
:101AA0009642F8D01B68F0E7505C012030B50A4A36
:101AB000D2F8003102F580724BB19C6884421C68F8
:101AC00006D15D688D4203D1146000221A6030BDDA
:101AD0001A462346F0E700BF505C012008B5074BCB
:101AE000187838B1064843682BB13DF0AFFA00389A
:101AF00018BF012008BD1846FCE700BFEF650120B4
:101B0000804F012008B50348012103F0C5FE0E20D7
:101B100008BD00BF3C5101201FB502AB01930B4B28
:101B2000009304310223013817F0AAFF08490298F4
:101B30004FF4107218F06CF8044603981CF00CFF78
:101B4000204603F0E9FD04B010BD00BF3C40090091
:101B50004C75080013B5012103F09EFE68464CF059
:101B6000FDFC3CF015FB00210C2043F00FFF064B61
:101B700003609DF800200DF10101520804463DF07C
:101B800008FA204602B010BD4C7508002DE9F0415E
:101B90000646806986B0F8B9114D044607464FF6EF
:101BA000FF782B8843450DD0EB6D0E2B03D12846D3
:101BB00000F07AFCE86506AB03EB8403EA6D43F8BA
:101BC000142C01340137052F05F18805E9D101A94D
:101BD00020461DF081FFB06106B0BDE8F08100BF76
:101BE000C006012008B501481FF0D4FDBF49080018
:101BF00010B50C4686B0A068012203A944F087FD09
:101C000088B19DF80430227962F347038DF80430DF
:101C1000039B1A68CDF805209B88ADF8093001A810
:101C20004CF09EFC10B103481FF02AFE0E2006B0B7
:101C300010BD00BFEF2708002DE9F04F2DED028BFE
:101C400095B00CAB51F8044B01935C4B00930138F9
:101C5000082317F015FF0C98012209A91BF086F83C
:101C60000D9800230E28CDE90633089303D00122F6
:101C700006A91BF07BF8119B0BB9514B11931198DE
:101C80001CF06AFEDFED4F7AB4EEE70AF1EE10FACF
:101C9000B0EE408A06D4DFED4C7AB4EEE70AF1EEFE
:101CA00010FA04DD494A4A494A481FF0D3FD0A9B0D
:101CB0009DF838509DF83C80109E1F2B05D925B10A
:101CC000079B13B144481FF0DBFD13980E280FD07B
:101CD0000DB94248F7E742494FF43E7217F098FFBA
:101CE000074694F84430DDF848901BB13D48EAE7D8
:101CF0000027F6E7E36813B1204603F03BFFDDF869
:101D000028A02946504602F071FBDDF81CB0294698
:101D1000584602F06BFBBAF11F0F04D9BBF1000F5C
:101D200004D03148CFE7BAF1000F02D00FB12F48ED
:101D3000C9E7002E38D1B8F1000F18BFB42661688A
:101D400019B9FF2011F06CFE6060A16819B9FF207D
:101D500011F066FEA060DDE90912606843F0DDFE67
:101D6000DDE90612A06843F0D8FECDE90497BDF87E
:101D70001C300393A3680293BDF828300193636875
:101D80000093B0EE480A3346424629462046FAF709
:101D900011FE3CF0FDF901230E2084F8443015B00B
:101DA000BDEC028BBDE8F08F114B124A7343934296
:101DB000C5D91148B4211FF063FD00BFB83E09002A
:101DC000CECC4CBE0AD7A33C0AD72341AA3E090079
:101DD000B03E0900CA3D0800024A0800CE2D0800A6
:101DE0004C750800D947080041290800352808002B
:101DF00040420F000FBCBA0A4D3108002DE9F04FE8
:101E00002DED068B93B00AAB51F8044B01937C4B3C
:101E100000930138082317F033FE0D980E2823D0C5
:101E20001CF09AFDF0EE408A0E9B0BB9754B0E9399
:101E30000F9B0BB9734B0F930E981CF08DFDDFEDCC
:101E4000727AB4EEE70AF1EE10FAB0EE408A06D4E8
:101E5000DFED6E7AB4EEE70AF1EE10FA07DD6C4AB8
:101E60006C496D481FF0F6FCDFED6C8ADCE7F5EE9F
:101E7000408AF1EE10FA07D0F4EEC08AF1EE10FAC3
:101E800002D567481FF0DEFC0F981CF065FDB4EE2C
:101E9000C08AF1EE10FAB0EE409A01D56148F1E740
:101EA0000A980023049348B1012203A91AF05EFFA7
:101EB000039812F0EBFA08B95B48E3E723699DF851
:101EC0003050DDF82CB0109F9DF84480DDE903A967
:101ED0003BB193F8293013B954481FF0D1FC0023CB
:101EE0002361E36843B16268934202D1112002F09A
:101EF00003FB204603F03EFE00212C2043F046FD6C
:101F00004B4B9FED4CAA0646002240F8083B594631
:101F10004CF0B8F9002D776214BFFF271F2700216E
:101F2000C6E907A907F10800266143F02FFD2369E0
:101F3000586000F1080303608780064601203AF0EC
:101F400074FB3CF025F921693B48FFF77DFD68EE05
:101F50008A6A9FED3A7AC6EE877AF6EE009A77EEB5
:101F6000A97AFCEEE77A17EE907AB7F5803F01D3B5
:101F7000334887E737B9F5EEC08AF1EE10FA01DD94
:101F800030487FE70E22002106A843F006FE28EE27
:101F90000A8ADFED2D6AADF81E7088EE267A45F4C8
:101FA000807545EA880525F0FA05314606A8ADF8A2
:101FB000185029EE0A9A37EE297AC9EE267ABCEE35
:101FC000C77A77EEA97A17EE103AFCEEE77AADF809
:101FD0001A3017EE903AADF81C304CF0E5FA054691
:101FE00040B115482169FFF761FD002323612846B0
:101FF0003CF0CEF8206913B0BDEC068BBDE8F08F45
:102000000C3F0900CECC4CBE0AD7233B66D62342F8
:10201000F83E0900023F0900CA3D08000000000028
:10202000424108005E4708006A2E0800422F08005F
:10203000A07B080000247449A5F0050000401C4660
:10204000724508003241080000401C44022838B59F
:102050000D46144613D1930701D01E2038BD1268D7
:10206000084B9A42F9D1A168A86844F045FE0028BF
:10207000F3D02A7923799A42EFD13E20EEE700206F
:10208000ECE700BF4C75080010B588B00846114653
:102090001A4603AB0193134B0093022343F099FEBE
:1020A00000210C2043F072FC0F4B03600446012218
:1020B000039805A91AF05AFE069B062B03D00B487D
:1020C00006211FF0C7FB049A032A03D940F24220DD
:1020D00017F0CEFC20460599D2B23CF05AFF2046BC
:1020E00008B010BDAC3F09004C750800E043080083
:1020F00010B50B4688B0044605A9986801221AF06D
:1021000035FE059908780B794A7903904878029052
:1021100088780190C97800912046024945F05DFB1E
:1021200008B010BD4C3F0900062837B50C4618D141
:102130008D680D4B2B40062B11D128094BF00AFD61
:1021400030B901A928461EF0D5F901994BF0E8FCF9
:1021500023795840400040F0010003B030BD68686A
:10216000EEE70020F9E700BF0F0080FF2DE9F04FF8
:1021700097B00DAB0193394B00930431092301381B
:1021800017F07EFC36490D9840F2D74217F040FD1B
:102190003449064640F281520E9817F039FD0F9DE2
:1021A000EBB215F0C0050746089303D040F2574044
:1021B00017F05EFC9DF8409048463CF0F4FE9DF818
:1021C00044A050463CF0EFFE129C002C04DA40F292
:1021D000DA31284617F0C0FC14989DF84C800E2880
:1021E00006D1B8F1000F14D09CB120461DF082FA40
:1021F0000DF1280B012259461AF0B8FD0B9BA342A2
:1022000004D8B8F1000F06D0A34204D016481FF03E
:1022100019FB1648ECE715980E281CD01EF092F911
:10222000034600212820099343F0B0FB099B104A84
:102230000260CDE905B3089B0093CDE90348CDE9E1
:10224000019A3B4600223146054603F0FBFC284636
:1022500017B0BDE8F08F0023E3E700BFBC3F0900E3
:102260005C7C0800F47C0800CE3C08003C6108005F
:102270007877080010B54368044653B10146064814
:10228000FFF714FC0023C4E90333C4E90633636099
:1022900063610E2010BD00BFF1DF060070B52DEDAB
:1022A000028B86B0084611461A4603AB0193214BB8
:1022B0000093032343F08DFD1F49039840F29B22B6
:1022C00017F0A6FC40F23F510646B7EE000A04980C
:1022D00017F08AFC059D002DB0EE408A04DC40F228
:1022E0008921012017F038FC0021242043F04EFB07
:1022F000124B036004460121284643F047FB9FED43
:10230000100A666028EE000A0023BCEEC00AC4E989
:102310000305C4E905330B4884ED020A84F8203034
:10232000E3612146FFF790FB204606B0BDEC028B2F
:1023300070BD00BF04400900787708007876080077
:1023400000007A44F1DF060008B501481FF022FAC8
:10235000AA4A0800C3691BB1D3E902011DF0BCBB46
:10236000004870474C5D080037B58B680192044601
:102370000D4673B1084945F030FAA968019A204624
:1023800000F088FC0549204603B0BDE8304045F028
:1023900024BA0349F8E700BF743F090080410900EF
:1023A000843F09001FB502AB51F8044B0193084B61
:1023B00000930138022317F063FB20469DF80C20A0
:1023C0009DF8081003F0AAFC0E2004B010BD00BF59
:1023D00024400900084930B50022882505FB02F495
:1023E0006318645A844204D00132052AF6D10020D1
:1023F00030BD1846FCE700BFC006012030B587B0ED
:1024000005AB51F8045B01930F4B00930138012396
:1024100017F036FB6868039000F018F805990398E8
:102420000BF016FC6C68204600F010F86368D3E9E6
:1024300002011DF051FB6B680446586844F04CFFE4
:10244000204607B030BD00BF3440090008B53CF05D
:1024500013FE10B901481FF081F908BDE64A0800D3
:1024600038B544680F4D2046FFF7F0FF94F87430FC
:102470000BB16B6A93B1B4F86C3007EE903AF8EE9A
:10248000E77AB7EE047A67EE877A17EE900A20F0C3
:10249000030040F00200A0F1FF4038BDFEF770FAE3
:1024A000E4E700BF505C012010B50446C06D0E2863
:1024B00007D100210C2043F069FA024BC0E9003437
:1024C000E06510BD8478080030B585B003AB51F8E5
:1024D000044B01931D4B00930138012317F0D0FAF0
:1024E00064681B4D2046FFF7B1FF94F85A30012B6A
:1024F00001D16B6AEBB194F85A30022B22D0012340
:10250000144984F85A302088114D4CF033F83BF0D0
:102510003FFE94F85A30012B01D16B6A63B16B6AAC
:1025200083B994F85B1069B1882908D10A481FF073
:10253000B5F9FEF725FAD8E7FEF722FAE9E70748EA
:102540001FF0ACF90E2005B030BD00BF1C400900E3
:10255000505C0120833D090012330800D532080089
:102560002DE9F0478CB005AB0193394B0093043152
:102570000723013817F084FA3649059840F29B2268
:1025800017F046FB344940F281520646069817F090
:102590003FFB9DF81CA0804650463CF004FD9DF892
:1025A000209048463CF0FFFC099D002D04DA40F2E3
:1025B000DA31002017F0D0FA0B989DF828700E2819
:1025C00004D187B17DB128461DF094F8012202A9FB
:1025D0001AF0CCFB039BAB4202D837B1AB4204D01C
:1025E0001E481FF02FF91E48F0E70021182043F085
:1025F000CDF91C4BC0F80880C0E900360023044622
:10260000838280F816A080F81790DDE902011DF0A2
:102610005BF8E060A7B9B5F5007F05DD124A4FF41D
:10262000007112481FF016F92582A774F3691BB1D7
:10263000214630463CF0C9FC20460CB0BDE8F0878E
:10264000B5F5FF7FF0DD0A4A4FF4FF71E9E700BFFF
:10265000C840090078770800F47C0800CE3C0800E8
:102660003C610800347908004D1708005A3F080003
:102670005817080037B58B68019204460D4673B1B0
:10268000084945F0AAF8A968019A204600F002FB23
:102690000549204603B0BDE8304045F09EB80349E7
:1026A000F8E700BF4C40090080410900584009008C
:1026B000130670B504460E4615460DD4022A0BD1FA
:1026C00040F22D204BF058FA0146204645F075F8AF
:1026D0000549204645F071F82A4631462046BDE8B6
:1026E00070401BF08BBE00BF4B17080010B543684D
:1026F00004464BB101460548FFF7D8F90023C4E969
:102700000233C4E9053323610E2010BDEBCF07006F
:1027100008B501481FF096F8AC2C08002DE9F047E9
:1027200088B0084611461A4605AB01932E4B00931C
:10273000032343F04EFB2D49059840F29B2217F0EE
:1027400067FA069D002D064604DC40F2892101202F
:1027500017F002FA07980E283CD1B6F81280002133
:10276000302043F013F9224B03607368B47D9B79EA
:10277000074640F2FD10804504F0300228BF804635
:1027800004F0060413B1134622461C4632B308F186
:10279000020A05FB0AFA0021504643F0F7F8814689
:1027A000FCB10021404643F0F1F8002105464046C7
:1027B00043F0ECF804460023CDE902833846CDE926
:1027C000005453464A463146FAF7D0F9384608B025
:1027D000BDE8F0871CF008F98046C0E791469246B4
:1027E000DEE72546E7E700BF1041090078770800DB
:1027F000987A08001FB50446084663680BB92AF0AA
:1028000091F9022201A91AF0B1FADDE9011220467C
:102810003CF0BCFC002803DA414204481FF01AF8DF
:10282000400040F0010004B010BD00BF3449080072
:1028300010B58AB002AB0C460193144B00930431DF
:102840000223013817F01CF9246863680BB92AF0D9
:1028500069F90298012207A91AF088FA039800235F
:102860000E28059303D0012204A91AF07FFA059BD4
:102870000093DDE90712049B204603F0A1FB20EA48
:10288000E070400040F001000AB010BD00410900B6
:10289000F8B5254C254B23603CF05AFB002842D06C
:1028A000234B1A781AB9234A1278012A09D12248EF
:1028B00000221A70436823B1204B1B780BB103F040
:1028C00067FB194803F074F9E36813B1164803F085
:1028D00051F900231A4DA3614FF6FF7705240E2608
:1028E0002888B84202D013214BF052FE013CEE651D
:1028F00005F18805F4D14DF0F5F80B48214602F0BA
:10290000CBFF4FF42A230F4A1B68934205D14FF4A3
:102910003122D2F8FC2F9A4201D000F0F5FABDE83E
:10292000F84030F0D3BDF8BD3C510120D074080010
:10293000F66601205E670120D84F0120EF65012077
:10294000C00601203130444230B589B003AB51F8A4
:10295000045B01930E4B00930138022317F090F8AB
:102960009DF81040039805A901221AF0FFF984F0A0
:102970000104E8680094DDE90523D0E902103BF08A
:10298000B0F8002814BF3E201E2009B030BD00BFA3
:10299000A840090030B587B0084611461A4604AB76
:1029A0000193124B0093022343F013FA0498104949
:1029B00040F2815217F02CF99DF81420039205463D
:1029C0000021182042F0E2FF0A4B03600446002079
:1029D00042F059FE039A03462946204639F0C1F8D1
:1029E0003BF0D6FB204607B030BD00BFB840090021
:1029F000F47C08005C7C080037B58B6801920446C3
:102A00000D4673B1084944F0E8FEA968019A2046D2
:102A100000F040F90549204603B0BDE8304044F0DD
:102A2000DCBE0349F8E700BF7C4009008041090093
:102A30008540090008B501481EF0ACFEE72E0800ED
:102A400010B5022888B00B46144624D1A20720D125
:102A50002168124A91421CD19A79012A09D1A2799E
:102A6000012A06D19A88A3889A4212D13E2008B042
:102A700010BD184669463CF098FC04A920463CF07D
:102A800094FC10220DEB0201684643F034F8002854
:102A9000ECD01E20EBE70020E9E700BFF47C080043
:102AA00008B58B7813B904481EF0EAFE0B888380C2
:102AB0008B78837108BD00BFAA3208001FB58379E7
:102AC000012B02D106481EF041FE69463CF06DFC28
:102AD000102168461CF0F8FD05B05DF804FB00BF4E
:102AE000544108002DE9F04106468EB008461146D3
:102AF0004FF002121C4616F093FF0021082042F00E
:102B000045FF066005462068C30706D410F003029F
:102B100012D101683E4B99420ED11BF065FFB0F512
:102B2000803F02D33B481EF08DFE0123A880AB718D
:102B300028460EB0BDE8F081374B0340062B05D088
:102B4000002A4BD10268354B9A4247D101A91DF0AA
:102B5000D1FC019B242B01D03148E4E7037A2D2BD3
:102B6000FAD1437B2D2BF7D1837C2D2BF4D1C37D60
:102B70002D2BF1D1471E00F12304002617F8018FF9
:102B8000404633F01DFB20B10EAB3344013603F851
:102B9000208CBC42F2D1202EDED106AC0DF11708FC
:102BA000002620784DF0DCFC074660784DF0D8FC1C
:102BB000023640EA0710202E08F8010904F1020449
:102BC000EFD1BDF8142000238DF814308DF81530A6
:102BD00002A9AA8028463CF0D0FBA9E7012206A959
:102BE00043F095FD08B90F489DE7079B102B01D0D6
:102BF0000D4898E7069B02AC03F110061868596867
:102C0000224603C20833B3421446F7D1D9E700BFC6
:102C1000E81D08001B3208000F0080FF5C1E080042
:102C20002B320800433208004F49080010B588B025
:102C300003AB51F8044B0193144B0093013802236A
:102C400016F01EFF0222039805A91AF08FF8A0794A
:102C5000049B069901280CBF1022802203EBD202AC
:102C60008A4202D90A481EF0EDFD059A012802EBBE
:102C7000030107D1A088D054A3881B0A4B700E20F3
:102C800008B010BD20463CF090FBF8E784410900F5
:102C90000549080010B58A79012A92B004460B460E
:102CA00006D18A881E4912B0BDE8104044F095BD97
:102CB0000EA918463CF079FB9DF838300D939DF82D
:102CC00039300C939DF83A300B939DF83B300A93C2
:102CD0009DF83C3009939DF83D3008939DF83E30B7
:102CE00007939DF83F3006939DF8403005939DF87B
:102CF000413004939DF8423003939DF84330029392
:102D00009DF8443001939DF8453000939DF847208D
:102D10009DF846300349204644F05FFD12B010BDD7
:102D200028410900354109002DE9F04F754C87B065
:102D3000002600AFA4F108084FF0880909FB0683BC
:102D400093F87830002B66D04CF0CCFED4E91E23EB
:102D5000801A61EB0301B0F57A7F71F100035AD359
:102D6000002134F8080CF981032307F10E026D46A7
:102D70004BF03EFC002848D1FB8934F8080C07339F
:102D8000DB08A5EBC3039D4607F10E02032369464A
:102D9000EA464BF02DFC002837D1B4F8502014F847
:102DA000060C022141F06DFDFB89834658B1C288B3
:102DB0009A4205D100F10801684642F09CFE20B31A
:102DC000584642F0F0F900233B7414F8063C3A8A66
:102DD000F889F88243F4007302F0FE0223F0FE0348
:102DE00013433B82B4F850307B8234F8083CBB82FA
:102DF0000FF028FC0222834607F110012CF0B0FAF4
:102E0000FA89514658464EF0F8F809FB068300222D
:102E1000AD4683F8782009FB068393F87930002BC0
:102E200040D014F8060C002846D0B4F82EA0524624
:102E3000012141F026FD054650B1C288502A04D137
:102E40002146083042F057FE38B3284642F0ABF92D
:102E5000002023F0A9FD04F1490B054614F8062CC7
:102E60006DBB0123A7F812A04FF0500A62F30005D2
:102E70007B74504634F8083C3D74BB82A7F816A01A
:102E80000FF0E0FB0222054607F110012CF068FA72
:102E90005246214628464EF0B0F809FB0683002230
:102EA00083F879200136052E04F188047FF446AFBB
:102EB0001C37BD46BDE8F08FB4F812A0B7E76B78B9
:102EC000012B1AD12B7803F00103934215D1EB8823
:102ED000502B12D10622594605F151007B6042F079
:102EE0000AFE50B97B6821461A4605F1080042F0F7
:102EF00002FE10B1284642F056F9284623F054FD50
:102F00000546ABE7C806012073B5104D4FF42A24DF
:102F10004FF00106200B2E704BF080FB08B92CF00F
:102F20000FFA04F58054B4F5322FF3D1084B019316
:102F300001A901224FF42A202CF012FA054801229F
:102F400001A92CF00DFA02B070BD00BF436701204B
:102F500031304442FC1F0B00032A05D11E2914BF47
:102F60000449054944F029BC1E2914BF03490449FA
:102F7000F8E700BFF1160800F61608005817080019
:102F80004D1708002DE9F0430D4689B005A9074605
:102F9000914628680122984619F0E8FE68680122E7
:102FA00002A919F0E3FE00229DF81010402016F04F
:102FB0005DFE0128024602D01A481EF02FFCDDE912
:102FC0000540022F04EB000610D9A9680E2902D093
:102FD00019F0D6FE0444032F08D0E9680E2905D065
:102FE0000698059E012219F0CBFE0644A64208D39E
:102FF000DDE90223CDF80090311B204641F056FC5C
:1030000028B9B8F1000F0AD007481EF01BFC059B39
:10301000C01A400040F0010009B0BDE8F0834FF055
:10302000FF30F9E7573508003D45080070B588B016
:103030000D460C2000211646039342F0A7FC154BC9
:10304000036004AB0193144B039A009331460423AD
:103050000446284642F0BDFE40F2C641049835F0D1
:103060009FF94FF499610546059835F099F929794A
:103070000279069B914203D140F23F4016F0F8FCE2
:103080000022626029460246204603F01DF82046D1
:1030900008B070BDF07E08007848090070B50C4695
:1030A0008EB054F8045B03920646A87A3BF023F8EE
:1030B000287A3BF060F80AAB01931D4B039A00930A
:1030C00021460423701E16F0DBFC0B98022207A990
:1030D00019F04CFE9DF824100022402016F0C6FD89
:1030E000089B0D99B3FBF0F30446069306AA0C9BCC
:1030F000059305A849F0B1FC069E4FF42272012108
:10310000304642F088FE059A06FB04F362430592BE
:1031100006934BB1079928460A44BDF8281003F0DE
:1031200093F808B11EF04AFB0E200EB070BD00BF30
:10313000D048090070B50C468EB054F8045B039279
:103140000646A87A3AF0D7FF287A3BF014F80AAB83
:1031500001931A4B039A009321460423701E16F024
:103160008FFC0B98012207A919F000FE9DF824108E
:103170000022402016F07AFD089B0D99B3FBF0F376
:103180000446069306AA0C9B059305A849F065FC26
:10319000059A069B012100910799624305926343BA
:1031A0000A442846BDF828100693F9F745FD08B1F2
:1031B0001EF004FB0E200EB070BD00BF5848090081
:1031C000F0B50C4697B054F8046B03920546B07AFC
:1031D0003AF091FF307A3AF0CEFF0FAB0193304BCB
:1031E000039A009321460723681E16F049FC1098A5
:1031F00001220CA919F0BAFD9DF8381000224020D8
:1032000016F034FD0D9B1399B3FBF0F305460893BC
:1032100008AA129B079307A849F01FFC11980222E5
:1032200009A919F0A3FD9DF82C100022402016F0EA
:103230001DFD0A9B1599B3FBF0F30446069306AAFD
:10324000149B059305A849F008FC069F4FF484627F
:103250000121384642F0DFFD079A089BBDF83C107B
:10326000039100206A436B430090059D0C980792E0
:10327000654302447C433046099F089305950694B4
:10328000F9F7DAFC38B944B1039923467A19304684
:1032900002F0DAFF08B11EF091FA0E2017B0F0BD6F
:1032A0009848090070B50C4688B054F8045B039246
:1032B0000646687A3AF019FF287A3AF057FF04ABCD
:1032C0000193184B039A00932146701E042316F0B5
:1032D000D7FB4FF4896301220021059816F044FCC6
:1032E00040F23943012200210446069816F03CFCC6
:1032F0004FF41E73064609220798082116F034FC85
:10330000C0B2082802D005201EF058FA0499F3B282
:10331000E2B228463CF06AF80028F4D00E2008B04B
:1033200070BD00BF7849090070B588B00D460C200B
:1033300000211646039342F029FB194B036004ABAE
:103340000193184B039A0093314604230446284600
:1033500042F03FFD4FF42971049835F021F84FF405
:103360007F710646059835F027F840F2EF310546A3
:10337000069835F021F8034618B915B90A481EF029
:1033800061FA9DF81C2012B108481EF003FA626031
:1033900020462A46314602F09FFF204608B070BD05
:1033A00010800800F0480900132C0800532A080078
:1033B00010B50446407A3AF098FE63681B68D3F86B
:1033C0002435B3F1805F23D013D8B3F1006F21D03F
:1033D0000BD8B3F1007F1FD01248B3F1806F18BF34
:1033E0000020400040F0010010BD0F48B3F1206FF5
:1033F000F5E7B3F1804F11D006D8B3F1A05F0FD03D
:103400000A48B3F1005FEAE70948B3F1004FE6E785
:103410000848E6E70848E4E70848E2E70848E0E744
:103420000848DEE790D003000024F40080841E00EA
:1034300000127A0040420F0020A1070048E8010076
:1034400000093D000048E80170B50C468EB054F804
:10345000045B03920646687A3AF047FE287A3AF00F
:1034600085FE0AAB01931A4B039A0093214604236D
:10347000701E16F005FB0A98022207A919F076FCC7
:103480009DF824100022402016F0F0FB0B9B0C99B5
:1034900006930446089BB3FBF0F305AA06A8059320
:1034A00049F0DBFA0699059A614362430691059259
:1034B00052B107989DF83430014428463BF0C8FFCC
:1034C00010B905201EF07AF90E200EB070BD00BFB5
:1034D0004049090070B50C468CB054F8045B039267
:1034E0000646687A3AF001FE287A3AF03FFE09ABC8
:1034F0000193194B039A009321460323701E16F083
:10350000BFFA0998012206A919F030FC9DF8201095
:103510000022402016F0AAFB0A9B05930446079B55
:103520000B99B3FBF0F304AA05A8049349F095FAAC
:10353000059B049A634362430593049242B1069942
:103540002846194402F0ECFF10B905201EF036F9A8
:103550000E200CB070BD00BF6049090070B50C466C
:1035600094B054F8046B03920546707A3AF0BDFDAE
:10357000307A3AF0FBFD0EAB01932B4B039A00938C
:1035800021460623681E16F07BFA0E9801220BA92D
:1035900019F0ECFB9DF834100022402016F066FB79
:1035A000109B1199079304460C9BB3FBF0F306AAFA
:1035B00007A8069349F051FA0F98022208A919F0BA
:1035C000D5FB9DF828100022402016F04FFB129BDF
:1035D000139905930546099BB3FBF0F304AA05A8CC
:1035E000049349F03AFA069B059A049807996343B5
:1035F0006A4345436143AB420791069305920495A4
:1036000002D00A481EF01EF953B1089802440B98E4
:103610000144304602F048FF10B905201EF0CEF8F4
:103620000E2014B070BD00BF10490900AA36080072
:103630002DE9F04F2DED028B9BB0084611461A463E
:103640000EAB0193A64B00930C2342F0C2FB40F259
:10365000BA410F9834F0B0FE40F25A5107460E9826
:1036600034F0AAFE40F2B6418046169834F0A4FE2B
:1036700040F2D2210646179834F09EFE40F2B14146
:103680000546189834F098FE8246B8F1000F03D131
:103690005FB994481EF0D6F8474514D0B04512D013
:1036A000A84510D080450ED02FB1B7420BD0AF4205
:1036B00009D0574507D01EB1AE4204D0564502D0BE
:1036C0002DB1554503D140F23F4016F0D1F94FF4EA
:1036D0001E7309221198052116F046FA129B824AA0
:1036E000934283462CD0814A93420CBF4FF002098B
:1036F0004FF00009022296230121139816F034FAA4
:1037000014981BF029F9B0EE408A4DF04DF99DF860
:103710006430039301212C2042F048F9744A02607E
:103720005FFA8BFB109B0493BBF1080F1599039B69
:10373000044608D06F4808224FF41E711EF08AF824
:103740004FF00109D6E7BAF1000F00D113B16A4872
:103750001EF020F8694BC0F804A01A68D2F80025C2
:1037600012F00F0206D09A68D2F80025120740F036
:103770001A81012203EBC2031FFA81FB636040F24E
:103780007B420121584642F03DFBB9F1020F01D1C5
:103790005B487FE7002E3AD1B5F1000A18BF4FF021
:1037A000010A00238DF83730B8F1000F32D098F8B5
:1037B000043007938FB33B7908938DB32B7909932A
:1037C0008EB333790498CDE90A3411F0E3F9B9F1F5
:1037D000000F4FF0030318BF4FF00E098DF835A00E
:1037E0000C908DF834308DF83690D4F80490454A1A
:1037F00099F8043024214B4302EB030A9AF8201075
:10380000039199B1404A4149414844F073F84FF05F
:10381000010AC6E74FF0FF33CBE74FF0FF33CBE7AA
:103820004FF0FF33CBE74FF0FF33CBE707A9484614
:10383000059339F0E6F8334A059B3649CAF8041077
:103840000B99D1509DF83430D9F8000005934FF40E
:10385000887149F017F9D9F800004FF4907149F0D8
:1038600011F9D9F800004FF4927149F00BF9D9F829
:1038700000004FF4A27149F005F9D9F800004FF4A7
:10388000AC7149F0FFF8D9F800202349C2F80413BD
:10389000059BD9F80000194640F30730F8F730F8D7
:1038A000D9F8000040F3073037F0D6FDD9F80030E2
:1038B0000822C3F80025039BCAF814300122CAE984
:1038C00006338AF8202087B3594604F110004AF0E5
:1038D000D9FC28BB606823F08BFD584615F082F8B0
:1038E0009849090034460800108108003481080016
:1038F0007C810800692D0800D22E080000030120F9
:10390000952D0800E05B01200500AD0B083A08008A
:10391000F01B0800EB0208001003420000007A448C
:10392000387984F8270000F043FFB8F1000F2ED05B
:1039300098F8040084F8260000F03AFF5EB330796E
:1039400084F8290000F034FF4DB3287984F828006A
:1039500000F02EFF1FED0F0A049BA36028EE008AE3
:103960000023BCEEC88A84F82530606884ED038AA1
:1039700004F1240123F0B8FC0C4B984202467FF47A
:1039800042AF20461BB0BDEC028BBDE8F08FFF2399
:1039900084F82630D2E7FF2384F82930D4E7FF23C8
:1039A00084F82830D6E7024874E600BF0000AD0B6B
:1039B000B345080010B51FF013FB044690F827002C
:1039C0003AF08DFBD4ED037A9FED077AF8EE677A33
:1039D000C7EE877A17EE900A20F0030040F002004D
:1039E000A0F1FF4010BD00BF00007A4410B51FF0E9
:1039F000F7FA044690F827003AF071FB63681868FC
:103A000040F30730002801DBF7F768FF0023C4E923
:103A10000733A36163681B681A0B43F30733002B5A
:103A200007DB02F01F0101228A405B09024941F8CD
:103A300023200E2010BD00BF00E100E038B52DEDC1
:103A4000028B0D461FF0CCFA044690F827003AF09E
:103A500046FB28461AF080FFB0EE408A4CF0A4FFE7
:103A60009FED050A28EE008A0E20BCEEC88A84ED80
:103A7000038ABDEC028B38BD00007A4407B50A4AC0
:103A800040F279138A4208BF4FF4A073019340F2C9
:103A9000CF13009305494FF406734FF4237243F09C
:103AA0009CFE03B05DF804FB10810800F849090092
:103AB00037B50C462046114606221D4615F0B0FFCC
:103AC00034B92146012003B0BDE83040FBF792BB7A
:103AD0002968CA0705D48B0708D10A680F4B9A4298
:103AE00004D1012C08D00E481DF098FE012003B02F
:103AF000BDE83040FBF7B0BA08461AF075FF014642
:103B000001902046FBF776FB019A04460021C0682D
:103B100042F043F8204603B030BD00BFE81D080066
:103B2000B3470800084608B5194612B104481DF00D
:103B300031FE18B1BDE8084000F006B8014808BDE4
:103B4000C73E08003C61080070B50546086810F0E3
:103B5000030390B00E4603D10168414A914228D038
:103B6000404C00EA0402062A04D033BB02683E4BF4
:103B70009A4222D1023D012D6ED80CA91CF0BAFC4C
:103B80000546306800EA0403062B14D1000949F009
:103B9000E1FF04460C9A34B911462846019249F0D7
:103BA000BFFF019A04462E48002143F093FCC560F4
:103BB000446010B070BD4468ECE7012D4CD110F0AA
:103BC000010413D0421002D500201DF03BFE114627
:103BD0000CA801924DF0ABF9019A0E98002141F02A
:103BE000DCFF0CA91E481BF00BFFE2E703AAB12182
:103BF00019F08AFD039B2BB103AA2146204642F00F
:103C00005CFAD6E730682A4605A942F080FD20B16B
:103C1000DDE905011BF058FDCBE730681BF0A8FC7F
:103C200098B910210CA84DF070F9306808A919F066
:103C3000F5F80446204619F097FA0028D1D01AF07A
:103C4000D3FEFF2803D90948BFE74110EAE7C1B214
:103C50000CA84DF0B8F8EDE705481DF0DFFD00BFFA
:103C6000281C08000F0080FF5C1E0800CA360800F0
:103C7000B3470800F0B585B0054617460C461AF064
:103C800003FF6946064628461CF034FC042F05460F
:103C900020D1A307009814D122680F4B9A4210D16B
:103CA00001AA214643F013FF10B90C481DF072FD24
:103CB000DDE901123046521A29441BF001FF05B01C
:103CC000F0BD0022214619F05BF8285C400040F06E
:103CD0000100F4E70020F2E77C59080030420800B8
:103CE0008B072DE9F14F04460D46164611D001F021
:103CF0000F03022B17D1D7074FEA111104D401B0DB
:103D0000BDE8F04F07F04ABD01B0BDE8F04F07F045
:103D100053BA4968CBB22D2B00F083800BD8062B09
:103D20000ED02C2B13D0534A2946204601B0BDE8B3
:103D3000F04F07F047BD2E2B00F088809D2BF2D16D
:103D4000002EF0D105F10802090A204683E0022A7C
:103D500002D0A96807F066FAEF68002FE3D017F0E9
:103D60000309E0D17B68DAB28E2AB8460DD1022E63
:103D70004FEA132805D007F1080A08F1FF3BD9459F
:103D800015DB08F1010857F8288098F80430312B2A
:103D900027D1022E13D1A06A42F039FCA06A562224
:103DA0006FF0020101B0BDE8F04F3FF004BA5AF8DD
:103DB000041B204607F036FA09F10109DFE7D8F8BD
:103DC0000810204607F02EFA012EE7D1A06A5822EB
:103DD00002213FF0F0F9A06A01B0BDE8F04F42F0D7
:103DE00042BC322B9FD1012EA06A0AD142F051FB76
:103DF000D8F80810A06A090901B0BDE8F04F42F0F8
:103E0000F6BA022E01D142F006FCD8F80830A06ABA
:103E10001B0918226FF0010101B0BDE8F04F3FF01F
:103E2000D3B9AA68002A3FF47EAF002E7FF47BAF9F
:103E30005168090A022907D1D3682BB1980703D129
:103E40001B79AC2B3FF46FAF08327EE7002A7FF47A
:103E50006AAFA96821B901B0BDE8F04F00F00CB815
:103E60008E0703D10B79922B0A46E1D005F10802A7
:103E700001216AE7053708002DE9F7430D460139AE
:103E8000044690464FEA012900264FF0FF3719F506
:103E9000807F0CD17B1C04D1A06A2B4630223FF0DE
:103EA000D3F90026AE4221D103B0BDE8F08358F823
:103EB00026307BB19A070DD11A79222A0AD101370F
:103EC0000CD1A06A019149EA060331223FF0BCF906
:103ED000019937460136A9F58079D8E7094A19468C
:103EE000204603B0BDE8F04307F06CBC58F826103C
:103EF000B74208BF896800222046FFF7F1FE01366D
:103F0000D0E700BF2040080001F00F03022B2DE98D
:103F1000F34705460C4605D1090902B0BDE8F04754
:103F200006F0B2BF00295FD011F003065CD10B7917
:103F30002C2B41D1896807F075F9E668002E53D023
:103F400016F0030850D17768FAB28E2A334609D1A9
:103F50003F0A06F1080907F1FF3AC24519DC0137AB
:103F600056F827301A79312A1BD19968284607F06C
:103F700059F9A86A019042F029FB019842F047FBE9
:103F8000019856226FF0020102B0BDE8F0473FF001
:103F900012B959F8041B284607F044F908F1010842
:103FA000DBE7322A20D19968A86A0222090902B007
:103FB000BDE8F04742F000BA2D2B15D18C689CB1BA
:103FC00063681B0A022B01D1E36843B904F10807B7
:103FD0006368B6EB132F0FD302B0BDE8F0879A07E2
:103FE000F4D11B79AC2BF1D1074A2146284602B007
:103FF000BDE8F04707F0E6BB57F8041B2846FFF77B
:1040000083FF0136E4E700BF4537080010B5137899
:1040100003F06003202B144644D1234B9288187878
:1040200090420ED093F8B80890423BD103F6B80303
:1040300001206278203A032A34D8DFE802F0041421
:10404000172B0020F5E729B90722991D204631F0EA
:10405000EBFA06E0022904D1144A12B1991DAFF31C
:10406000008001201FE00029FBD1EDE719B92046AF
:1040700031F0C8FAF5E70229F3D162881A7102F02B
:10408000010181F0010483F82C40C2F3400231F0B9
:10409000F9F9E6E70029EAD00229E2D1618831F096
:1040A00099FADEE7002010BD240D01200000000079
:1040B000F8B5294B41F270120021184641F06DFD10
:1040C0000346082601244FF48235067300F13801B7
:1040D0004FF0FF0C4FF4424783F8C46803F50F66B6
:1040E0000022016180F805C04FF47841C780048147
:1040F0004561C3F8C86840F2FF7003F5876E03F5A9
:104100004F66DA83C3E909E51A8498835A8659838E
:104110009A8683F82C40A3F8D6281886D98583F888
:10412000BDC8A3F8BE78A3F8C048C3F8CC58A3F81C
:10413000D408A3F8D218A3F8D828C3F8DC68C3F8C9
:10414000E05883F8E448A3F8E808A3F8E618A3F8D1
:10415000EA28A3F8EC28F8BD240D01202DE9F74347
:104160004B79022B04D00025284603B0BDE8F0832C
:104170008B79022BF7D1DFF8A09099F802701FB16C
:1041800099F8BA38ABBB012740F6B8067E438B7866
:1041900009F806300C7809EB06080C440925637809
:1041A000242B20D1AA4219D26378042B12D163792F
:1041B0000A2B0FD12778F31C02364E4402220096B8
:1041C0004B441146E0194CF05DFA90B10E3517FAE8
:1041D00085F5ADB2404637F053FFC5E723781D445F
:1041E000ADB21C44DBE7052BDED1204633F082FD67
:1041F00038B94FF0E023D3F8F03DDB07B3D500BE6C
:10420000B1E740F6B80202FB0797A3787B702378EA
:104210001D44ADB21C44C7E7240D012070B50F4CFE
:10422000002504F11000256025714BF01DFF04F1FD
:1042300024004BF019FF012604F6C80084F82C6016
:10424000C4F8B85884F8BC584BF00EFF04F6DC00F4
:104250004BF00AFF84F8E46870BD00BF240D012014
:104260002DE9F7433D4C1D46E3788B420E4617D0AF
:10427000A3788B4214D094F8BB388B422ED094F89C
:10428000BA388B422AD04FF0E023D3F8F05D15F016
:10429000010501D000BE0025284603B0BDE8F0832B
:1042A0000027E378B34214D104F63808AAB2414695
:1042B00004F110004BF064FF6379FF2B04D005F686
:1042C0003809A144C8450DD1254BD3B9204637F054
:1042D000D7FEA378B3421ED00125DDE704F6B8046B
:1042E0000127DEE7617918F8013B9942EAD1E28BB8
:1042F000238C92B29BB29A42E4D0384631F04AF90C
:10430000E0E7E28B238C92B29BB29A42DED0384631
:10431000AFF30080DAE7134B13B13846AFF30080F8
:10432000384631F0FBF80028D6D104F124004BF0D8
:10433000A6FE0028D0D1002DCED015F03F02CBD163
:10434000A078019233F0BCFC019A05460028C3D046
:10435000A078114633F0DEFD9EE700BF240D01205A
:10436000000000000000000010EE103AC3F3C75236
:10437000A2F17F01162982B013DC002913DB124A57
:104380000A411A420DD0DFED117A30EE270A002BD8
:104390008DED010AA8BF9B18019923EA020300EEE4
:1043A000103A02B07047DFED097A30EE270A002B91
:1043B0008DED000A009A04DB5A0018BF4FF07E53BF
:1043C000EDE74FF00043EAE7FFFF7F000000807B4E
:1043D000054B4FF0FF32072843F8202084BFC01858
:1043E00080F85020704700BFB45A0120FF2808B55C
:1043F00002D821B1EE2802D901481DF023FA08BDE8
:1044000047280800830773B5044603D102680A4BA6
:104410009A420AD0094E0025204616F8011B0123B6
:104420006A4619F0ABF9009808B1012002E00135A5
:10443000032DF1D102B070BD401E08006292090048
:1044400038B50023C3714FF0FF33C364054641F014
:10445000F9FB044630BBB5F84E224AF655239A4282
:1044600022D114490B2205F1500041F044FBE8B180
:1044700095F85030EB2B03D01833DBB2012B17D853
:104480000D49032205F1860041F035FB40B10B498F
:10449000052205F1A20041F02EFB002818BF0224DE
:1044A000204638BD0424FBE70324F9E70124F7E79D
:1044B0000224F5E78F5609009B5609009F56090014
:1044C00008B501481DF098F93F2A080008B5074BC8
:1044D0000340062B05D0830706D10268044B9A429D
:1044E00002D104481DF09AF908BD00BF0F0080FFFB
:1044F0005C1E0800573508000D2808B5014612D08B
:1045000006D804280BD0072810D00A481DF0B8F9A7
:1045100043F202039842F8D107481DF01FF90749FA
:10452000074843F0DCF907480021FAE706481DF088
:1045300089F900BFE1320800582D0800442D080019
:10454000D41B0800A85508004D2B0800012808B509
:1045500004D103484FF4E8711DF07CF908BD00BF99
:104560003C29080008B510B901481DF06BF908BDD9
:10457000A72A080073B504461E460D4651B11868B7
:1045800001921AF081FA6368019A834202D00548C9
:104590001DF044F9A0683346294602B0BDE87040DA
:1045A00016F006BC9C3508002DE9F04F2DED028B6E
:1045B00083078DB004460D4609D10368784A9342BB
:1045C00005D111F0030802D10A689A4202D0754859
:1045D0001DF024F948F054F818B1284648F050F876
:1045E00008B97148F4E7267930461FF0BFFF029002
:1045F00028791FF0BBFF0690304621F0E5FED4E994
:10460000037305903246E07901930AA9CDE90A3790
:1046100048F07CF8C3690493D4F81CB0EB69DDF86A
:1046200010A003930646D946B8454CD105F10C01BC
:104630006622E879089148F069F80899C3690590FD
:104640006622E879079348F061F8C1694FF00008E5
:1046500089468A46B84567D1019A049B746904FB70
:104660000234079B01EB870503EB8709A7EB020BDD
:104670009046019B08F1FF3A534500F28C80059863
:104680000DB0BDEC028BBDE8F08F48460793029B4E
:104690009847059B504698477269079B9244A269C8
:1046A00001339144019A9342EFD1D6E90523019950
:1046B00002FB11339A44D4E9053202FB11339944C9
:1046C00008F10108B0E70023ECE7CDE908315846CE
:1046D000029B9847FAEC017AA269089B0999A0EE1F
:1046E000278A934401339845EFD10398069B08919C
:1046F0009847029B584630EE488A9847C8EE007AA1
:10470000CA466FF0030303FB08AA0899E9EC017A93
:10471000D4E9053202FB18339B44039AAB691A446F
:10472000039208F1010895E79FED208A0023DAE75C
:10473000029B2046CDE9032198470499B369F1EC27
:10474000017A039AE0EE278A1C440132BA42EFD381
:104750004745B06935ED018A2CBFD8464FF00008B7
:104760004FEA8B0308F1010838BF0023A3EB88034D
:1047700000FB184899444046029B984738EE688AE7
:104780000BF1010BC8EE007AC9ED007A7469A8EB51
:104790000404D0466DE7DFED058A49464246D5E779
:1047A000DCCB0800DA3A0800613D08000000000098
:1047B0004109064A012300F01F0003FA00F052F8F5
:1047C0002130184342F82100704700BFF05001200B
:1047D0002DE9F04F042A97B080468946144635D01B
:1047E000A84E30680EF0A4FD002C4BD0A64B9C4286
:1047F00048D0002502AB03932A46A44B04932146DC
:1048000003A802951BF092F9029804300122294670
:1048100020F0030038F0D1F83060B8B10368099394
:104820009DF82830029A43F001038DF8283007AB39
:10483000CDE9072505932A46954B0693214605A801
:104840001BF074F933681A68029BD554914C924B53
:10485000206800251D600FF051FC25608F4C904AA8
:104860002368934211D16268A24202D3631C9A4228
:1048700029D98C4D106851682B4603C39068186085
:10488000656020E000233360E0E78749D4F8C0206A
:104890008B42E8D085498B420DD1854B9A4240F03E
:1048A0009E81D4F82831A34240F09981012120460D
:1048B0003BF02AF907E07F4A934204D1626804F191
:1048C0000805AA42D6D1D4F8C0307B4A934240F0C2
:1048D000A7807A487A4D01213AF001FF0023B4F80D
:1048E0000A11B4F808016B622EF062FF7348294682
:1048F0003AF009FF7348744D01F05AF9714801F01C
:1049000039F9D5F80061002E40F0AD802DF08CFF14
:10491000D5F8C870002F40F0F18029F025F80DF08F
:1049200027FDD5F808A150460FF0B0FD0646002837
:1049300040F0E880C5E941AA079003F037F9634BDE
:104940000DF11C0A1868D346002840F0DE80079A53
:104950001A605F4B01901F605E4B5F4F187003F051
:1049600037F931F015FEAB8A0198C5F8B40101336F
:10497000AB820FF0FBF90198C5F8A80140460EF094
:10498000D7FC48460EF0D4FC0FCF5E460FC60FCFC3
:104990000FC60FCF0FC697E8070086E80700DFF8BD
:1049A00058910023CA46D9F800701FB13E68002E06
:1049B00040F0C480002BF2D1DAF800301BB15A6805
:1049C000D20700F1E280D5F8F830002B40F0E1800A
:1049D000424B434D1B684349434AC5F800B0002B86
:1049E00000F0FA801B684B62118B0B445362226803
:1049F0002E4B9A4203D12948002103F033FD22684F
:104A00002C4B9A4205D1E069F9F7AAFF00B1006882
:104A1000E06100232B6017B0BDE8F04F2FF0D0B855
:104A2000324A934204D10021244802F021FB61E77D
:104A30001F4A93427FF45EAFD4F828011AF024F89D
:104A400070B12B4B98420BD01C4801213AF01BFF50
:104A50001B4928483DF06EFE012384F8223149E7C6
:104A600028F01CFF46E7D5F8A8314BB171688B429E
:104A700006D8D5F8AC31994202D2B068FDF716F8E5
:104A8000366840E7785F0120BC5C012061160700B2
:104A9000970E0800AC500120B45001206809012095
:104AA0004C8B080070090120EC8C0800A8BB0800A2
:104AB000689808001CC008009C890800280A01208A
:104AC000900101203C510120505C0120B050012098
:104AD000B85001201C670120685001201861012096
:104AE0006C5F01207404012020040120E08A08008A
:104AF000A05D0800300A012080580120384612F0DD
:104B000049F905E7DAF80CA00DE782680192D5F8BB
:104B1000A8212AB1904203D3D5F8AC21904207D303
:104B2000CAF80000074600F1080A866001980BE702
:104B30001022002141F031F82B4BF7E77A689007FB
:104B400020D57268D1071DD507F10800F9F708FFD5
:104B500006F1080303607A6833683B6022F00302C1
:104B600002F108087368019342463946304640F026
:104B7000FCFF06EB0802019B46F808605360C9F889
:104B800000200123D9F800900DE71B68CAF8003017
:104B900012E71E68154A1768C6B93B6813607B6840
:104BA0000837384623F00308F9F7DAFE0122814678
:104BB00031464046F9F7F4FD00F108034246394614
:104BC000184640F0D2FFC9F80000FCE6BE4238BFEC
:104BD0001A4633463668DEE753624B6207E70448FD
:104BE00003F0E0FB6FE600BFB0500120485D0120FC
:104BF0006809012013B54FF4AB616A4618F05EFDF9
:104C000000216A46084641F058FA084C42F019FB68
:104C100008B102B010BDFBF7B3FE616A0029F8D1FC
:104C20006A46084641F049FAF0E700BF505C0120AF
:104C300010B59CB000904068FFF7DCFF002042F008
:104C4000AEFB012202A9019018F090F809A847F0E4
:104C5000ECFE0446D8B9009B05AA586840F2A25160
:104C600018F02CFD009B1B7A5B0043F0010305AAA2
:104C7000214607930220019B089341F01EFA21F080
:104C8000D5FE009B586839F00EFC1CB010BD009B8F
:104C9000586839F008FC0A9C064920681AF02AFC7A
:104CA00020B1009B0448197A1CF0D4FD204621F065
:104CB00095FE00BF005508007F2C08002DE9F34742
:104CC0000C461D4616461EF073F9DDE90A98837CF2
:104CD0005B4288F80030E307074611D414F0030A5A
:104CE00003D12268384B9A4206D020461AF0C0FB06
:104CF00078B3BAF1000F24D12268334B9A4220D105
:104D0000204619F0AFFE0314337003122B7089F89C
:104D10000000BB7C002B4ED13A7B042A4BD17A7C1D
:104D2000002A48D032782978914244D199F800205D
:104D30008A4201BF88F8002033702B7089F8003058
:104D400039E0204619F008FEFDEEC07A17EE900A11
:104D5000D9E76A4601A9204619F0D4FD04220321AF
:104D6000019840F2AB2314F02FFF009B1868F8F76E
:104D70005DFA009B30705868F8F758FA009B28706D
:104D80009868F8F753FA019B89F80000032BC0D903
:104D9000009BDC6820461AF06BFB78B1204619F0C6
:104DA000DBFDDFED0A7A20EE270AFCEEC07A17EE73
:104DB000903A88F8003002B0BDE8F087204619F03C
:104DC00051FE88F80000F6E7E81D080000007F4368
:104DD00070B52DED028B0646B0EE408A1EF0E8F865
:104DE0009FED1F0A80ED068A28EE008A4289BCEEFC
:104DF000C88A044618EE103A9BB29A4209D0058937
:104E00004268416A4381B3F5807F02FB05F503D117
:104E100059B9BDEC028B70BD39B9284640F0B6FDDA
:104E2000216A60622A4640F078FE0023AB420AD134
:104E300094F82830002BECD0BDEC028B3046BDE856
:104E4000704039F0D9BBA27C0AB19A0706D0D4E9E8
:104E500008126089D25C42431212CA540133E5E75A
:104E60000000804383B5F9F719FAF9F7C5FB154C33
:104E7000154F01910125A560064665602420BD718E
:104E8000F6F718FD114B6560C4F84833C4F80833D1
:104E90000F4B104C00254FF47A40BD7143F00103D5
:104EA000984740F2FF33278823802FF09DFA01991D
:104EB00027804FF480632A4630462FF015F828F0FB
:104EC0000DFD00BF004002401F67012003000F00DE
:104ED000903D09002C06012038B5F7F73FFF012867
:104EE00007D0022819D10E480E4B036000234360FF
:104EF00038BD0B4A0C490D4B136008780C4C00234D
:104F0000536054F833100D79854202D15160044842
:104F1000EEE70133302BF4D1F9E70E20E8E700BFCC
:104F20005C50012020670800906701204C66080053
:104F3000C49F080070B5104B0122002604465A6039
:104F4000C3F80065FF2590F8210028F0F1FC94F8E3
:104F5000220084F8215028F0EBFC94F8230084F818
:104F6000225028F0E5FC054B84F823501E60BDE874
:104F700070402EF0A5B800BF0050024078580120C4
:104F800070B5044690B00163164601F10800002296
:104F90001D4600233EF02CFA206B06AB102207A919
:104FA00008303EF056FD10B105201CF007FC069BB2
:104FB000102B0BD14249042207A840F09CFD28B9D0
:104FC0004049082209A840F096FD18B14FF44F70EF
:104FD00014F04EFD206B06AB042205A908303EF00C
:104FE00038FD0028E0D1069B042B02D1059A142A33
:104FF00002D935481CF026FC206B06AB0BA9083003
:105000003EF027FD0028CFD1BDF82C300599012BAB
:105010000CD1BDF82E20022A08D8BDF83A30102B4A
:1050200004D8122904D1BDF83C1009B12748E1E7A2
:10503000206B0C99A16284F82420A376042206AB8D
:1050400004A908303EF005FD0028ADD1069A042AD7
:1050500006D11F49019204A840F04DFD019A08B104
:105060001C48C7E7206B06AB03A908303EF0F1FCF3
:10507000002899D1069B042BA8D1039B6361236B65
:105080001B6C238335B16D0866602E44E562E660D3
:1050900010B070BD4FF48070E062294640F076FC9D
:1050A000606018B9E560E06A13F09CFCE06A29468C
:1050B00040F06CFCE0600028EAD16560F3E700BFD7
:1050C0003453090039530900712B0800523308008A
:1050D0009FF80800212808007FB5044608460D46C1
:1050E000164638F070FA63685B69984202D01F4830
:1050F0001CF0A8FB284638F025FA6368DB7C834265
:1051000001D01B48F4E7284638F010FA63681B7C8E
:10511000834201D01748EBE70DF10903019303AB7C
:1051200000930DF10B020DF10A030021284638F01F
:1051300028FA63689A7C9DF80A309A4201D00E489A
:10514000D6E72846A560267338F02FFA04F114023A
:1051500004F11001284638F001FA63699B08636185
:10516000431E58425841607304B070BD913008002E
:105170007530080051300800AA300800F8B5044620
:105180004FF40060C4E907000F46002115461E4693
:1051900040F0FCFBA06128B9204639F091FAE069A3
:1051A00013F020FC4CF0D9F8606030B9204639F09B
:1051B00087FA1649164842F092FBEB0744BF06F106
:1051C000FF360135B6F5105F09D3656205F59055D8
:1051D000A56239462046BDE8F84000F01BB8002122
:1051E0004FF4905040F0D2FB606228B9204639F06D
:1051F00067FA4FF49050D3E700214FF4905040F0FD
:10520000C5FBA0620028E4D1F0E700BF0428080035
:10521000D41B080030B5044689B00D4602F0C6FC28
:105220000022A563002305F108003EF0E1F8E369E0
:1052300023624FF47F43E387204640F0C2FD2046BF
:1052400040F019FD4FF490520021606A40F0A5FC37
:105250004FF490520021A06A40F09FFC01A9204623
:1052600014F096FB054602F0B3FC1DB90849094845
:1052700042F035FB039B6363029B84F83D30059B42
:105280005A009B00E36200232263636409B030BDCF
:10529000A3290800F01B08002DE9F04F91B002AFE0
:1052A00007EE901AC188396141687960032A8188C4
:1052B000F96106465AD0D11FD1F1000802F0FD0273
:1052C00048EB0108052A01D148F002088B4AF86929
:1052D00052F82350FB6969784FF0020B1BFB013336
:1052E00003EB43035B0007336A46DB08A2EBC3030F
:1052F0009D46FB694FF0030919FB013901EB81035E
:105300005B0002AC03EB800304EB410204EB4909B0
:105310001C4403461F3368465B11A0EB43139D46B4
:10532000EA4617EE900AFA62C7F830907C630023D1
:105330004AF8081B41463FF022FA6B7800934A4630
:10534000012341463FF01BFA6B78009322465B46EF
:1053500041463FF014FA4FF000094C463B6999452D
:1053600080F2BD80FB6ABB61002322E04FF00108A0
:10537000ACE7BA6932F9132014447F2CCCBF012268
:1053800000220AF80320CCBFFF220022A41A24B274
:10539000E91C4FF0000C2A78944501F1030144DB2D
:1053A000AA7812FB04F4002CB8BFFF3444F30F2496
:1053B0000133FA699342DCDB5246494630464BF0F2
:1053C000D1FE7B6BD7F830B07B613B63BB697B63FD
:1053D00009F10103FB60D7E903239342C7F82CB01E
:1053E0007DD06B780093BA6909F1030317EE900A38
:1053F00041463FF0C4F9FB69013B31D2F96852469E
:1054000030464BF0AFFE7B69FB62BB69C7E90C3BE2
:105410006B78009317EE900A09F104035A4641464F
:105420003FF0ADF909F1020998E711F9022C07F1F3
:10543000380000EB820211F9030C52F80CBC11F990
:10544000012C184412FB04F23BF810E0002AB8BF0C
:10545000FF320EEB22222BF810200CF1010C9AE700
:105460003BF81320144422B27F2AD4BF002101212B
:10547000802AB4BF0022FF22A41A0AF8031024B223
:10548000E91C4FF0000C2A78944501F1030108DB78
:10549000AA7812FB04F4002CB8BFFF3444F30F24A5
:1054A000AAE711F9022C07F1380000EB820211F98A
:1054B000030C52F80CEC11F9012C181AB860B868FA
:1054C00012FB04F23EF81000002AB8BFFF3200EBD6
:1054D0002222B8680CF1010C2EF81020D3E77A686C
:1054E000002307F120013046C7E909233B6208F099
:1054F00047FF3C37BD46BDE8F08F00BF04560900AA
:105500002DE9F04F2DED028B91B000AF984697F842
:1055100070307B6297F874303B6197F87830FB60AD
:10552000837B08EE101A012101FA03F30646013BC2
:1055300018EE100A9246FB6117F052FC7368B861CE
:10554000002407F134013046C7E90E347C6308F0CB
:1055500017FFB388FC6208FB03F303EBCA034FEAAF
:10556000CA02013B93FBF2F30AFB03F3BB62033372
:1055700023F003027A61BA6A23F00303013207338E
:1055800022F00102DB083A627B60B6F80690FB6A03
:105590004B4505DB4437BD46BDEC028BBDE8F08FC3
:1055A0006B4608EE903A7B686A46A2EBC3039D46C1
:1055B000FB686D46A3B1FB6A09F1FF39A9EB03094A
:1055C00000233B63BB69BA6A5C68294618EE100A7F
:1055D00007F13003A047396B29B108461CF0EEF8FB
:1055E000D7F82C90ECE7BB6A834202D0494842F0DE
:1055F00076F93B69A3B1BAF1020F0CD0BAF1040FEE
:105600000ED17A692B46A9188B4209D01A6812BAB2
:1056100043F8042BF8E73A6A2B4651198B4210D114
:1056200008F1FF33AB460024BB600FFA89F9B38859
:105630009C420BDB18EE903A9D46FB6A0133FB62FD
:10564000A3E71A8852BA23F8022BE7E7B8F1080F4C
:105650000BDCB8F1000F11DDBB68072B0ED8DFE8BB
:1056600003F00F270D360D0D0D45B8F1180F42D080
:10567000B8F1200F4AD0B8F1100F39D0002309E05B
:105680007B6AE1108BB1E34303F007026B5C1341CB
:1056900003F00103FA6921B2134030464A463CF058
:1056A00069FC01340BF1030BC1E704F00702EDE7DD
:1056B0007B6AA11043B1E34303F003035A006B5C20
:1056C000134103F00303E5E704F00303F6E77B6A05
:1056D000611043B1E34303F001039A006B5C134193
:1056E00003F00F03D6E704F00103F6E72B5DD1E7E3
:1056F00035F81430CEE79BF801309BF800201B02F0
:1057000043EA02439BF802201343C3E755F82430D1
:10571000C0E700BF0454080070B52DED028B8AB0BD
:1057200002A9B0EE408A36F043FC0E22002106A802
:1057300040F033FA9FED480A9FED487A28EE000AC0
:10574000A023C0EE077AADF81A30ADF81C3004AAD9
:1057500001248DF81940B6EE007A77EE877AFCEED8
:10576000E77A17EE903AADF81E303D4B186859684D
:1057700003C23C4801A9FCF767F900238DF8063005
:1057800004AA234606A902A848F0F8FE044630B150
:10579000344801A9FCF78AF9204638F0F9FC9DF855
:1057A000063063B12F4801A9FCF780F9BDF8046009
:1057B0004FF6FF739E4205D12B481CF061F8FBF7B2
:1057C000DFF8ECE7002021F0EFF80446B8B1637889
:1057D000012B34D12378DB0731D506220DF10901E5
:1057E00004F1510040F087F948BB04F1240204F1B0
:1057F0003601304648F0CEFEB0FA80F46409002548
:10580000694630468DF800508DF8015048F0C4FECE
:105810004FF40071304648F0D5FE29462A463046FE
:1058200048F0AEFE114B882101FB05F2D018D25A88
:10583000B24206D00135052DF6D10D48BDE7204610
:10584000C1E70123837080F85A40FCF72DFE0AB0AF
:10585000BDEC028B70BD00BF0024744900401C46A3
:10586000E61608000D16070096290800C00601205C
:1058700086290800074A00234FF6FF7132F813000B
:10588000884205D14433B3F5AA7FF7D10020704791
:1058900001207047C00601202DE9F04790B00D4669
:1058A000044639F055FBA84200F03881002D00F085
:1058B0001D819C490B7853B10020F5F7FBFF9A4AF4
:1058C00000231360994A0B701360994A1360994E34
:1058D00099493068029002A848F0C7FE002840F0BD
:1058E0008F80964991F816335A09EC231341DB0750
:1058F00040F1F980924B9A68002A00F0F0801A6813
:1059000042F480021A608F4A0023C2F800318E4AA6
:10591000012713704FF005088C4A0392032308A94E
:1059200020208DF820708DF82280ADF8243048F0CA
:105930000FFE002864D1CDE90900854B039A089336
:1059400008A9402048F004FE002859D1CDE90800FC
:105950000A90039A8DF8207008A922208DF82280E1
:1059600048F0F6FD00284BD1CDE908000A904FF42D
:105970000073039A8DF8207008A92320ADF8223017
:1059800048F0E6FD00283BD1CDE908000A903843F5
:105990008DF82000039A08A9A02048F0D9FD78BB13
:1059A000CDE909004FF4DC53039A089308A9A1201C
:1059B00048F0CEFD20BBCDE908000A904B23039AA6
:1059C0008DF8203008A9384648F0C2FDC0B903A8B8
:1059D00048F0C0FDA0B99DF8103004A93B43022057
:1059E0008DF8103048F00CFE50B95A4A7068516872
:1059F00006AB03C306A848F0D3FD08B948F0B8FDCC
:105A0000019010F0ABF8019838F0C2FB002D72D075
:105A1000514DDFF85C9100263746A5F1080A88232E
:105A200003FB06A34FF6FF7845F8047C25F8088CA5
:105A3000502283F85A70002105F8067C284640F071
:105A4000ACF80136A5F108014846FCF72FF8052E01
:105A500025F8088C05F18805E1D1404B06A8C4E97A
:105A60000D3448F07BFD38F093FB9DF81A203C493B
:105A70003C4B100902F00F02085C8A5C9A729DF898
:105A800019205872100902F00F02085C8A5C1A7320
:105A90002022D8725F73344804AB0DEB020147F04B
:105AA000BDF9054630B99DF810301BB99DF820505E
:105AB00045F47F452C48294602F056FACDB908A88E
:105AC00039F055FA2949224604F11C00FBF7D8FFAA
:105AD0002CF0AAFE10B0BDE8F047FDF725B94FF451
:105AE00080030B600FE742F2020089E748F0BBFD3C
:105AF00086E71C48E4E71D482146FBF7D7FFE3682B
:105B000013B1204600F036F80E4A0023C2F80031E7
:105B10000D4AC4E90333C4E90133137010B0BDE882
:105B2000F08700BF35670120445C0120485C0120FC
:105B30004C5C0120841608000BF0070000E100E037
:105B40005C5F0120505C01204367012000E00020E1
:105B50000104040188160800C8060120D5DB0600F0
:105B6000733D090043060120603D0900BDDE0200CF
:105B700011BE030038B50C4B04461878FF2812D02C
:105B800048F0F4FC214605460848FBF78FFF002348
:105B9000E36084F8443035F0080304D02846BDE8BB
:105BA000384038F0F5BA38BD33060120C5C70600C5
:105BB00038B50369044663B148F0F8FC2369054829
:105BC0000122002583F829205D602169FBF76EFF23
:105BD000256138BDA5F005002DE9F74304460F46C1
:105BE000154649F07FFFDFF85890064688466369FE
:105BF0009D4212D80DF1070029F0C0FB04F10C0002
:105C00002A46394648F064FB04469DF8070029F00F
:105C1000D9FB204603B0BDE8F08349F063FFA268DA
:105C2000831B61EB0801934271F10003E2D2FAF7A2
:105C3000A7FED9F82430002BD9D00024E9E700BF13
:105C4000505C01202DE9F74FDDE9116B0446002778
:105C50000D469DF830009DF83410DDF83C809DF82D
:105C600040A0A78291469DF83820A075C4E9015351
:105C7000E17522762782E760E6B1244B72682282C2
:105C8000D3F8A811336819B31846019200930EF0A7
:105C9000FDFBDDE90032C8B1394690B23FF076FE37
:105CA000228A316807463FF038FFE76000203FF066
:105CB000EAFCE061BAF1000F20D1B8F5007F0AD903
:105CC000134A4FF4007113481BF0C4FDE360EDE785
:105CD000E360E161EEE7A4F8128084F826A0AB79D6
:105CE00023B1A4F8149003B0BDE8F08F60685A4661
:105CF000214603B0BDE8F04F39F079BAB8F5FF7F1F
:105D0000E9D9054A4FF4FF71DDE700BF505C01207F
:105D10004D1708005A3F080058170800F0B5478C87
:105D200085B00C46164617B91B481BF0A9FD436801
:105D30009A791AB919491A4841F0D1FDD86837F053
:105D40000EFE054639F090F90023002ECDF80530FF
:105D50008DF809304FF0010314BF022100218DF8A6
:105D6000043002230C43ADF80A306B44ADF8024016
:105D7000ADF80670039301A9284648F02BFC48B102
:105D800020F00203112B02D1FAF7FAFDF3E738F005
:105D9000FFF9F0E705B0F0BD6F2C08009C49080042
:105DA0006CAE08002DE9F04F43689A7985B004463F
:105DB0000D466AB1D86837F0D2FDA37D0146A08AAE
:105DC000C3F340132A4605B0BDE8F04F39F063B97C
:105DD0004B6890F82610428A21B19A4206D0284892
:105DE0001BF030FD9A4201D22648F9E7A08A2A46E4
:105DF0004FF6FF7139F07BF900264FF6FF7A4FF02E
:105E0000020B214B33F8167057452FD094F81680AB
:105E100018F0060F2AD00DF10603618C039302AA35
:105E20003846CDF808B048F0E7FB43F2014398420A
:105E300023D10023ADF8063018F0040FBDF806900A
:105E400008D019F0010F05D0A08A01232A4639464F
:105E500038F0F3F818F0020F08D019F0020F05D04F
:105E6000A08A02232A46394638F0E7F84436B6F5C8
:105E7000AA7FC6D105B0BDE8F08F38F089F9DBE71D
:105E8000583308006F330800C006012008B50148E8
:105E90001BF064FC582D080070B543685D6804462B
:105EA000E86837F05CFDAB790A4601462BB1A08A61
:105EB0000023BDE8704039F0EEB8A57C5068238A15
:105EC00025B1984206D006481BF0BCFC984201D987
:105ED0000448F9E7A08ABDE8704039F008B900BF6E
:105EE000583308006F33080070B5064686B0084680
:105EF0000D46144639F0B8F800234FF400722048DC
:105F0000019401A9CDE90223ADF810508DF81430A9
:105F1000FBF79AFD00223146284648F059FB11282C
:105F20000446F7D030B1164801A9FBF7BFFD204663
:105F300038F02EF99DF81430B3B1BDF8100039F0E7
:105F400093F801A90E48FBF7B1FDBDF8121089B214
:105F500091B140F20513994209D040F20F139942D2
:105F600008D008481BF08CFCFAF70AFDE2E7064867
:105F70001BF094FC0548FBE7039806B070BD00BF1A
:105F8000F5BF0600C3320800FA2A08000C2B0800EF
:105F900070B50A4D04464FF6FF76A38C9BB213B939
:105FA00094F82D302BB1E38C9BB2B34201D06B6AD5
:105FB00003B170BDFAF7E4FCEFE700BF505C0120CD
:105FC0002DE9F3479846C3690A9D04460F461646D5
:105FD00013B93A481BF054FCC38C4FF6FF799BB2BF
:105FE0004B4504D14FF0FF3002B0BDE8F08739F0E7
:105FF00092F80028F6DB7219904204DA40F225414B
:106000002F481BF027FC238D934202DA4FF477715F
:10601000F6E7A28C984216FA82F2A8BF184682428E
:1060200010D9DFF8A0A0A38C9BB23BB1E38C9BB24C
:106030004B4503D0DAF82430002B39D0DAF824307D
:10604000002BCFD1E38C4FF6FF729BB29342C9D0A5
:106050000DF1070029F092F994F82A3004EB83033C
:10606000D3F81C90A38C9BB22BBB2A4641464846D2
:106070003FF053FDA38C15FA83F39BB2A384A08C4D
:106080003246394619FA80F03FF047FDA38C9DF85F
:10609000070016FA83F39BB2A38429F093F994F8CE
:1060A0002D30354413B9204647F06DFD28469BE757
:1060B000FAF766FCB7E70025E1E700BF50340800B7
:1060C00096310800505C0120F0B51646354A0D4661
:1060D000117A85B004461F4611B1137D3BBB0121E7
:1060E0000C2303FB012262602879012146F0E0FCC9
:1060F0000121307946F0DCFC0A2020F0BBFD287934
:10610000002146F0D5FC3079002146F0D1FC032077
:1061100020F0B0FD307946F016FD70B9307927F0E7
:1061200007FC287927F004FC1F481BF065FB436837
:10613000002BD9D11D481BF085FB287946F003FDC3
:106140000028EBD0327901924FF0CC7202920722F4
:10615000ADF80C20164A2B79009397421AD94FF0CC
:10616000C862029263723079A072FEF721FB28792F
:10617000FEF71EFB636801221A726068694621F00F
:106180002DF80C4B98420BD0204639F01AF9052017
:106190001BF014FB084A9742E4D94FF08062E0E715
:1061A00005B0F0BDE8040120E42C080068440800B4
:1061B0007F1A06000000AD0B8FD0030038B543688E
:1061C0001C681A790623C4F800351E4B0546342096
:1061D00000FB0233022283F82D200023C4F8881527
:1061E000C4F84435C4F8483501232362A360D4F8C9
:1061F00050311BB9D4F82431002BF8D04FF4A871DA
:10620000204646F03FFC01236361D4F80431002BA3
:10621000FBD04FF48271204646F034FCD4F8243190
:1062200073B120464FF4927146F02CFCD4F8C4347C
:10623000C4F8C4340024686820F0B4FF204638BD98
:106240000124F8E7785B01202DE9F04F16464268FB
:10625000DFF880801C46137912688B460621C2F84D
:106260000015342202FB0383022289B0054683F81D
:106270002D204FF6FF794FF0010A69685CB9144B85
:106280006868019320F08EFF019B184609B0BDE8B5
:10629000F04F2FF04DBB0023CDE905364C45274686
:1062A00028BF4F460793049708798DF80CA08DF806
:1062B0000DB04FF0340C03AA096800FB0C802FF0DE
:1062C000E7FB034A90420346DAD1E41B3E44D4E79D
:1062D0000000AD0B785B01202DE9F04F1D465E4BB1
:1062E0000746D3F8000510F00F0085B0144606D01D
:1062F000A3F54043D3F800351B0704D10120574BC9
:1063000003EB001078607B6813B955481BF09AFACC
:1063100091F804A0D3F8089087F809A05046FEF73A
:1063200047FA3CB32479BC722046FEF741FA25B304
:106330002D79FD722846FEF73BFAD7F804B0494E96
:106340009BF80480242303FB08631B7F63B9484642
:10635000FAF752FB8146B8F1000F11D1B0F1206F6E
:1063600002D0B0F1A05F0ED1384639F05DF80520BB
:106370001BF024FAFF24BC72D9E7FF25FD72DCE78D
:10638000B8F1010FF0D1242303FB08F3F118002228
:10639000DBF80070F2504A60504646F0B8FB03A8A4
:1063A000CDF80CA020F05EFB039B03F5E073012207
:1063B000FF2C40F8232049D0204646F0A8FB204679
:1063C00046F084FBFF2D44D000212846019546F07D
:1063D0006FFB019B242202FB08F20192B21838469F
:1063E00082F82150FF2582F820500222C7F860254C
:1063F0000022C7F808A51146C7F80C45C7F81035A4
:10640000C7F8249546F0CAFB019BC7F8C055F3585E
:1064100013B14022C7F804230721C7F800155BB168
:10642000DBF8000040F30730F5F76AFADBF800000C
:1064300040F3073035F010F8242303FB08660023EF
:1064400073770123337705B0BDE8F08F4FF0FF3449
:10645000B8E74FF0FF33BDE700F002402C360900EB
:1064600011450800185B012010B50D4B42689A4297
:10647000044611D010339A4210D10123094A012158
:10648000D154607A20F0CCF9A07A20F0C9F9E07AF2
:10649000BDE8104020F0C4B90023EFE710BD00BFF5
:1064A0002C3609002C6701202DE9F04F1746426871
:1064B000DFF86090DFF860A0DFF860B087B0984642
:1064C0001368019306460D46B8F1000F01D1012073
:1064D00017E07268019BD468444528BF44464B4589
:1064E00004D12246294650463FF017FB706802A9A6
:1064F000CDE90254CDE9047420F05CFD584503D089
:10650000002007B0BDE8F08F25442744A8EB04081D
:10651000DAE700BF00F0024000E000200000AD0B11
:106520002DE9F04F15464268DFF860A01368DFF8E8
:106530006080DFF860B087B081460E4601930DB9E8
:1065400001201BE0D9F80420019BD768AF4228BF87
:106550002F46534515D13A46314640463FF0DDFAC5
:106560004246D9F80400002402A9CDE90227CDE96A
:10657000044420F01FFD584505D0204607B0BDE873
:10658000F08F3246EDE73E44ED1BD8E700F00240C5
:1065900000E000200000AD0B10B50446406820F07C
:1065A00027FF94F8260027F0C3F994F8270027F076
:1065B000BFF994F8290027F0BBF994F8280027F0D8
:1065C000B7F961680A4A4FF6FF73E3842385914265
:1065D0004FF00003C4E90433C4E90733A36103D0D7
:1065E0000832914203D10123024A0021D15410BD47
:1065F000000301202E6701202DE9F3471E46436862
:106600001B68D3F81435013304468846154602D179
:106610002D481BF017F949F065FADFF8B4A00746DA
:106620008946A3699D423AD86368186840F30730E9
:10663000002846DA04F110072A464146384647F05A
:1066400047FE94F8253005468BB104F12401012260
:106650003846019147F064FE0199606820F044FEDD
:1066600094F8290046F053FA002384F82530636833
:106670001A68130B42F30732002A07DB03F01F01ED
:1066800001238B405209114941F822301DB90B23D7
:1066900033604FF0FF35284602B0BDE8F08749F07F
:1066A00021FAE368C01B61EB0901984271F1000314
:1066B000BAD2FAF765F9DAF82430002BB1D0002508
:1066C000E9E7F5F70BF9B5E79E2C080000E100E0DB
:1066D000505C01202DE9F04F83B0984643681B6859
:1066E000D3F80C35013300AF81460D46144602D174
:1066F0004F481BF0A7F8002A71D001F0604ABAF1A8
:10670000005F10D0802A20D94A4BD3F8A831E3B1DA
:10671000002110460DF06EF8034629462246184621
:106720003FF0FBF90546D9F80430187920F054FE03
:1067300090B905F06043B3F1005F10D03E4AC8F84D
:1067400000203E493E4841F0D5F8E31D23F0070301
:10675000ADEB030D6B46E0E7FAF712F9E3E7D9F882
:10676000046096F804B0584620F036FE08B1354A69
:10677000E5E7354B242202FB0B324FF49071546154
:10678000956030687A6046F07DF930684FF4AC71FE
:1067900046F078F97A68316890685369C1F8440521
:1067A000C1F848353168012088605268E2B10023A1
:1067B000C8F80030D9F80430187920F00DFE002810
:1067C00032D1BAF1005F0AD01A4BD3F8A83133B1F5
:1067D00028460DF05BFE10B128460DF08FFC2046D8
:1067E0000C37BD46BDE8F08F3268D2F82001D2F8F0
:1067F000581118B90029F8D0144A09E00029FBD132
:106800000121D1603168D1F85821002AFBD0104A0B
:106810000D4B242101FB0B33002159610C4BC8F8AF
:1068200000209A42C3D08CE7FAF7AAF8C2E700BF6B
:10683000A52C0800505C01200A00AD0B083A0800A6
:10684000F01B08000B00AD0BE05B01200800AD0B56
:106850000000AD0B10B50379FF2B04460ED0084A9B
:10686000002142F82310007920F00EFA207920F060
:10687000F9FA207927F05CF8FF23237110BD00BFDF
:10688000941E0120F8B504468180C28003FB01F00C
:106890001F304009A08180B250430E468000002185
:1068A0001D4617463FF072F80023082DA06084F8BB
:1068B0002230A57306D9102D04D0202D02D00E4809
:1068C0001AF068FFE37301212022B2FBF5F2914236
:1068D000E37B0CD3012202FA03F3013BAA402361BC
:1068E000013A00232284268363616783F8BD013364
:1068F000E3734900EBE700BF5F2B08002DE9F04F81
:106900002DED048B91B00CAF0446B7F87C00786095
:1069100097F8900097F868C0F860002084F8950018
:10692000B7F8548097F88800D7F880B0B7F894602B
:1069300097F89C50CDF828C097F864C0CDF824C0D3
:1069400097F860C0CDF820C097F85CC0CDF81CC0A7
:1069500097F858C0CDE9058CB7F850C0CDF810C0F5
:10696000B7F94CC0CDF80CC00028B7F948C00CBF2F
:106970004FF48070FF2004F10809CDE9010C00906C
:106980004846B0EE408A07F081FD97F86C3084F8F5
:10699000923097F8703084F8933097F8743084F818
:1069A0009430B7F88430A4F88C30FB6883F001038E
:1069B00084F8963097F88C3084F8973097F89830B0
:1069C00084F898301DB108F1FF335D425D41A4F8B1
:1069D0008E604FF47A7384F89950B3FBF6F64FF05B
:1069E000000AA4F890607B689A4533D3554BA366A0
:1069F000BBF1000F1BD09BF8040038F0D2FFB0B100
:106A0000002204F168050092B7F8A03059462846E4
:106A100001F0ECFB002800F083804B4BA366594645
:106A2000284638F025FD9BF8040038F0CFFFB0EE83
:106A3000480A204600F090F82046444938F063FEAA
:106A4000F968204638F04BFE1437BD46BDEC048B88
:106A5000BDE8F08FBB6F03EB0A0898F9013098F896
:106A60000150BB6008F1020309EE103A05F07F0502
:106A700048463BF0B1FC002839D094F8973008EE36
:106A8000903ABBB36B4608EE903A05F1080303F069
:106A9000F803ADEB030D98F800208DF830200CAB17
:106AA00019EE101A6E1C2A460DF131003B603FF0C2
:106AB00034F800963B68666AA06801220021B0475E
:106AC00018EE903A9D4648463BF0D4FCBB68002B3C
:106AD00023DA6E1C023518F80500FF2808BF4FF4B2
:106AE000FA70023616F0DCF95AFA86FA7BE7F9F703
:106AF00047FFBDE70123009318EE901AA068666A6D
:106B000043460122B047009519EE103A18EE902A3C
:106B1000A068666A0121B047D5E72E460A20E0E763
:106B20000B4BE06EA36625F089FE94F8703009499E
:106B300003F07F02012393400A5C13430B54636FFD
:106B4000187972E7A05D0800E88408009001012030
:106B5000A8BA0800306701202DE9F0412DED028B25
:106B600090F8983086B00446B0EE408A1BB9F7EE34
:106B7000007A37EEC08AA36E324A934210D1DFED1D
:106B8000327A68EE277A04F16800FCEEE77A17EEB5
:106B9000903A99B238F07CFF84ED228A012015E00A
:106BA0002A4A93420CD1DFED2A7AE06EB4EEE78AEE
:106BB000F1EE10FACCBF0121002138F0ACFCEBE77C
:106BC000B4F88C30B3F5807F05D1002006B0BDEC61
:106BD000028BBDE8F08104F1080840463BF0FCFB65
:106BE0000028F2D0DFED1B7A94F8976094F88C209F
:106BF000676AA0688DF8142068EE277AFCEEE77AC1
:106C0000CDED037A9DF80C305EB18DF8153002237E
:106C10000093012205AB0021B84740463BF02AFC17
:106C2000BAE701258DF813302A4605AB31460095A9
:106C3000B847676AA06800950DF1130332462946EC
:106C4000EAE700BFA8BA080000FF7F47E884080011
:106C5000A4707D3F00007F432DE9F04F2DED028BA6
:106C600099B090F89A3006AF0446F3B1826EB04BFB
:106C70009A421AD1683038F010FC94F89730834269
:106C800008D100233B6138694C37BD46BDEC028B0F
:106C9000BDE8F08F2CF014FA0021B4F88230A26F16
:106CA00084F89A10204647F02BFEE3680BB90123C5
:106CB000E8E7204638F02FFD0028E2D104F1080B68
:106CC00058463BF08CFB38610028DAD094F862100B
:106CD000002900F0E2800023636404F13C037B623E
:106CE00094F89C30002B40D020463BF088FEB4F84E
:106CF0004850B4F84AA06D08EB1DE946DB08A9EB43
:106D0000C3039D460DF118082A46772140463EF000
:106D100044FFB4F8923087F83C3058463BF05CFBB7
:106D2000012394F89E200093A068666A07F13C0353
:106D30000021B04758463BF09DFB00233B623B8C53
:106D4000534508D258463BF047FB3B6A01333B6250
:106D5000002840F0B3802046CD463BF0DDFD754D68
:106D600094F89A30002B40F0B780724B5B6A002B8E
:106D700087D120463BF043FE6B46796A07F130022B
:106D8000584608EE103A3BF035FB002800F04581EC
:106D90007B8EF98E07F13000C91A202594F8523005
:106DA000B5FBF3F53BF09FF8B0EBC51F89B24FEA96
:106DB000C51A00F298800123FB6180B28A468023C5
:106DC0009B004009FB600130073323F00703F862A2
:106DD000ADEB030DFB6A9B00073323F0070306AE00
:106DE000ADEB030DB4F89430B3F5807F0CBF0123F5
:106DF0000223BB60FB6833440DF118097B604FF040
:106E000000087A8EFB8E9B1AB4F88C209BB2B2F5E8
:106E1000807F3B6217D00020B4F88E3094F88A103F
:106E2000049007F13000039094F89E00003818BFDA
:106E30000120029000200190B4F890000090D2B29E
:106E400058463BF039FBB4F8923087F82B30B8F154
:106E5000010F04BFB4F8943087F82B3058463BF04C
:106E6000BBFA012394F89E200093A068656A07F19D
:106E70002B030021A84758463BF0FCFA0023C7E942
:106E80000533BB8AFA699A4256D8BA6808F10108F4
:106E90005FFA88F39A42B4D8BFE0E06800283FF474
:106EA00006AF08F06DFC786200283FF400AFB4F83C
:106EB0008C30B3F5807F7FF413AF0CE794F89E20FD
:106EC0000095A068666A43460121B04758463BF0EA
:106ED000D1FA2FF05DFB32E76B6A002B7FF445AFF0
:106EE000F9F74EFD3CE73B8EB88EC01A80B2BAFB74
:106EF000F0FABAF1010F38BF4FF0010AB1FBFAF313
:106F00000AFB13119AB289B2FA6119B1134601331F
:106F10009BB2FB611AFB00F080B2B0FBF5F293B2BA
:106F200005FB1202002A3FF44BAF01339BB247E747
:106F3000E8840800505C012000237B643B8E7A8E3D
:106F4000B98EBB87BB69A7F84010396AD3188A4548
:106F50009BB288BF3A6AFB8797BFBB699B185344B3
:106F6000D21888BFA7F842303B6A98BFA7F84220E2
:106F7000A3EB0A039BB207F13C003B623AF0B3FF7C
:106F800094F852300822B2FBF3F3FA6AB0FBF3F341
:106F90009200002148461D463EF0FFFDFA680021A0
:106FA00030463EF0FAFD94F89B30002B56D001237A
:106FB000984584F8573011D1062384F8563033466B
:106FC0004A4607F13C0158463BF057FA03E094F873
:106FD0005930002BF3D194F899300EE0072384F850
:106FE000563033464A4607F13C0158463BF045FAD5
:106FF000B8F1010FEFD094F898301BB133467A689E
:10700000934217D158463BF0E7F97B6901337B6126
:10701000BB6953449BB2BB6188B918EE103A9D46D8
:107020007B6A9B687B62002B7FF4A6AE20463BF018
:1070300073FC28E61A68D24343F8042BDFE7ABB2AF
:1070400094F89E200093A068656A33460121A84702
:1070500058463BF00FFA2FF09BFA12E7B8F1010FF8
:10706000BFD194F85820002AB1D084F85730A6E751
:10707000034B0830002908BF19463BF05BBB00BF3B
:107080009001012010B50C4B426A9A42044611D07F
:107090000021806A38F03FFA4FF47A701FF0EAFD61
:1070A000A06A012138F037FA4FF47A701FF0E2FD40
:1070B000012010BD0020FCE7A05D08002DE9F7438A
:1070C0001C464B1ED3F1000848EB030815463C4B09
:1070D00042690A9F9A4206464FD100258DF8075013
:1070E0002744BC421CD1C5B19DF807307068C5F17A
:1070F000080503FA05F501220DF107018DF8075087
:10710000FFF70EFA0121306A38F005FA01201FF06E
:10711000B1FD306A002138F0FEF903B0BDE8F0831C
:10712000013515F007059DF807307068A14613D1A9
:1071300048EA430301220DF107018DF80730FFF7FC
:10714000EFF9706801222146FFF7EAF999F800305B
:107150008DF807300134C4E7C5F109029340C5F149
:10716000080208FA02F2134322782A4113438DF8E9
:10717000073001220DF10701E6E78069414638F04A
:10718000CAF9012D14D12744BC42C6D001222146A0
:107190007068FFF7C5F90121306A38F0BCF90120A9
:1071A0001FF068FD306A002138F0B5F90134EBE7D3
:1071B00070683A46214603B0BDE8F043FFF7B0B926
:1071C000A05D080010B50446406804F10803984229
:1071D00001D138F0F6F86269044B9A4205D104F106
:1071E0001400BDE8104037F046BA10BDE88408002E
:1071F00010B50A4B42699A4204460CD000218069BE
:1072000038F089F904201FF035FDA069012138F01C
:1072100082F9012010BD0020FCE700BFA05D08003E
:107220002DE9F0470446A6B081610022002301F158
:1072300008003CF0DDF8A06901AB8A2203A9083000
:107240003CF007FC10B105201AF0B8FA019B8A2B1C
:1072500006D16C49022203A83EF04DFC054618B148
:107260004FF44F7012F004FCDDF816302381DDF886
:107270002A30BDF8288084F82180A3F1030CDCF1CA
:10728000000343EB0C0384F82030DDF81E30A380AC
:10729000DDF82230E38001462420DDF81A70DDF8A5
:1072A0003A603EF073FB584B03604FF080734361CC
:1072B0001023984585808371E0612ED1372F02D845
:1072C00094F820300BB3DDF84230E360DDF846304F
:1072D0002361DDF84A30636194F82110A3880729FF
:1072E0004FF008008CBFCA080122B0FBF1F0002863
:1072F0007FD112FB03F39AB299071CBF22F003025D
:107300000432628126B0BDE8F0874FF478734FF401
:10731000F840C4E903031F23DDE7B8F1080F59D88B
:1073200016B9012606FA08F6002110203EF02EFBC1
:10733000364B03600546B0B2A860002100013EF064
:1073400025FB4FF0000A012E686085F80DA036D0AD
:107350004FEA86091FFA89F9514648463EF016FB66
:107360008046A0690022002308303CF041F8A06963
:1073700007F10E0292B2534608303CF039F8A0698A
:1073800002AB4A46414608303CF063FB0746002802
:107390007FF459AF029B994507D01D481AF052FA65
:1073A00058F82120284638F060FAB9B28E4207F129
:1073B0000107F5D840460CF0A1FEE5618CE7524686
:1073C0005146284638F051FA6FF07F42314638F086
:1073D0004CFAF2E70C2F3FF47FAF282F3FF47CAF3D
:1073E00027F010036C2B3FF477AF0A4839461AF0A8
:1073F00031FA4B43DA061CBF23F01F032033DB08AE
:1074000063817FE71E5609007C870800948E080080
:107410007C320800A92D080070B5554CD4F8C03056
:1074200033B92368002B54D1BDE870402CF038BB31
:10743000504DAB42F5D0504A93421FD1002104F188
:10744000C00038F04CF9D4F8CC302BB193F82A2096
:107450006FF3410283F82A20D4F82831474A934237
:1074600005D1474800F04EFFC4F8C050D9E7454A5F
:107470009342F9D1424837F0FEF8F5E7424A934289
:1074800021D194F85A3183B104F1C00031F02EFFBC
:107490002BF016FE0021B4F84231D4F8382184F8DC
:1074A0005A1104F1C00047F02BFAD4F8CC302BB1BC
:1074B00093F82A206FF3410283F82A20D4F8282178
:1074C000304B9A42D5E7314A9342CDD126F0E6F9C6
:1074D000CAE7284EB342A7D02D4A934210D1606824
:1074E0002C4B984201D137F09FFFA06938F0E9FAA0
:1074F000206A38F0E6FAA06A38F0E3FA266093E7EB
:10750000254A934203D11A48FFF75CFEF6E7234A67
:1075100093421ED1002594F830002844C0B20135B2
:1075200026F006FA082DF6D1E368187926F000FA5D
:107530006369187926F0FCF9636A187926F0F8F97E
:10754000E36A187926F0F4F9E369187926F0F0F97E
:10755000D4E7134A934203D1054800F023FFCDE757
:10756000104A9342CAD1024801F0ECFAC6E700BFC4
:1075700068090120A05D08009C890800A8BA0800DD
:10758000900A0120E8840800E08A08006898080052
:107590004C8B080070090120EC8C080074B40800C2
:1075A000A8BB08001CC00800F8B5C38A13B9164868
:1075B0001AF048F990F850301B070ED500F124015D
:1075C00000231D46048B9AB2944218D890F850308C
:1075D00043F0020380F8503002E0416A0029EFD105
:1075E000F8BD94B20CFB0414013204F80E50478B22
:1075F000B0F818C096B2B742F3D80133E2E70022E0
:107600001FFA83FEF3E700BF1F3108007FB5044671
:10761000C08A984202D829481AF014F994F8500008
:10762000050746D504F12400258B02FB05004354D1
:1076300094F85030258BD807238CA1EB030191FBE4
:10764000F5F305FB13110EB254BF04F12C0001A891
:10765000002EA38BBCBF49190EB213FB06F39BB2DD
:107660000380A18B0B448380638C618BD21A92FBC5
:10767000F1F301FB132215B2002DE38BBCBF5218AE
:1076800015B213FB05F39BB24380E28B1344C38016
:1076900094F85030DB0705D504F12C0201A91046FF
:1076A0003AF02BFC94F8503043F0010384F850304A
:1076B00002E0606A0028B7D104B070BD1F31080035
:1076C0002DE9F04F2DED028B1F46002380F89030FE
:1076D000044681668FB040F25B400D4690461AF03A
:1076E0000DF8E066C369002B00F09A8028469847A1
:1076F00086B2E36EA06E1B69984783B208EE103A1B
:10770000E36EA06E5B69984783B208EE903AE36E31
:107710005B6A04F1080B002B00F08480A06E984790
:107720008146E36EDD6A15B1A06EA8470546E36E9B
:107730009B69002B7DD0A06E98475FFA80FAE36EBC
:107740001B6B13B1A06E98470346E26E526B002A82
:1077500072D0A06E0D9390470D9BCDE909300021AA
:107760004FF48073CDE90033CDE9075A18EE903A13
:10777000CDE90569CDE9031118EE102A02915846AA
:1077800006F084FEE36E1B6A13B1A06E984783B2C5
:10779000A4F88C30E36E9B6B002B4FD1B4F84830CB
:1077A00094F852205343DB10A4F88E30E36EA06EA1
:1077B0005B6804F170019847B4F88C30B4F84A0063
:1077C000B4F88E1040F2563200FB0131606F3EF08B
:1077D00022FB87F0010384F89130E36E9B6A002B53
:1077E00034D0A06E984780B2A4F888004FF47A7322
:1077F000B3FBF0F0A4F88A00B8F1000F03D04146C3
:10780000204600F027F8124958463AF093FF3946CF
:1078100020460FB0BDEC028BBDE8F04F38F033B816
:10782000102666E7072E8CBF4FF000094FF00109C4
:1078300077E74FF0020A82E710468EE7A06E98477E
:1078400080B2A4F88E000028B0D1A7E73C20CBE797
:107850009001012010B5B0F84C305A2B04462CD0C2
:10786000A3F5877CDCF1000343EB0C035A2926D0F7
:10787000A1F587704242424193421FBFB4F848309D
:10788000B4F84A20A4F84820A4F84A3004F10800CB
:107890003AF079FF0B4B9C4207D12CF001F9B4F878
:1078A0004A10B4F848002BF083FFE06848B104F1B7
:1078B0002C01BDE810403BF0F1B90123D6E70122CD
:1078C000DAE710BD280A01202DE9F74F00F5A0489E
:1078D000071D04460D46C8F8BC1D45F6B8520021E8
:1078E00038463EF05AF94FF00109AC4B88F8B99D83
:1078F0006364AB4BA364AB4BE36465660023002277
:1079000005F108003BF074FDD8F8BC3D00269B69EA
:10791000E365A66549463846F0F7F2FC00284CD0EE
:1079200004F15807A36C314638469847E368B3F52D
:10793000A07F40DC314624203EF028F89A4B0360BB
:10794000D4E9031205461023FEF79CFFC8F8C05D7A
:107950003146A36CD4F85C8004F5DC753846984752
:10796000636C4FF4805229463846984794F9C231E7
:1079700094F8C2A1002B0246A8EB000621DB0D23E0
:107980004FF0000942F21071CDE900914FF001086B
:10799000934221DB08F1FF3804F5A044019BC4F8B1
:1079A000CC3D009BC4F8C49DC4F8C88DC4F8D03D3C
:1079B00003B0BDE8F08F022323624FF44F7012F042
:1079C00057F80AF007034FF0020A0AFA03FA0AEB23
:1079D0004A0A0AF10D03D3E7A2EB030BBBF5817F43
:1079E0000FDAE9185A4628463EF0BFF8636CCBF52B
:1079F000805205EB0B013846984700230BEB000241
:107A0000361AE95C2C2947D03B29C3D02129C1D1A2
:107A1000E818417890F802C0F92914D1BCF1040F9C
:107A200011D10179407941EA00210229B8BF022130
:107A30000A2041430098814289442BDC0198884206
:107A4000A8BF0846019003F1020AD4440CF10203D6
:107A5000AC449CF801B0BBF1000F99D09B440BF1F2
:107A6000010315F80BB0A2EB030A0BF2011151450B
:107A7000F1DBE918524628463EF077F8636CCAF508
:107A8000805205EB0A013846984700230AEB0002B2
:107A9000361AE0E70091D6E79342BFF67BAFE818CD
:107AA00003F10A0A90F90930417A002B07DA01F054
:107AB0000701022303FA01FC0CEB4C0CE2440AF12F
:107AC000010BA2EB0B0A01F20111514513DB9345A7
:107AD00042DA05EB0B01524628463EF046F84FF0DD
:107AE000000BCAF58052636C05EB0A0138469847D3
:107AF0000AEB0002361A0BF1010315F80BB0BBF1CB
:107B0000000F2ED1E85C3B2805EB03013FF444AFA6
:107B10001EB9D01A1F287FF73FAFE06DB0F5805F28
:107B200008F101087FF734AF002E7FF731AFA2EBE9
:107B3000030A524628463EF018F8CAF58052B2426F
:107B4000A8BF3246636C05EB0A013846984700230C
:107B50000AEB0002361A1BE7ABEB020B4FF0000AF0
:107B6000BFE7B3F5406F16DD002E14DDA2EB030A6C
:107B7000E918524628463DF0F8FFCAF58052B24255
:107B8000A8BF3246636C05EB0A01384698470023CC
:107B90000AEB0002361A9B44ADE700BF91B3060022
:107BA000C7B30600E5AF0600C886080010B5064C4E
:107BB000236813B9054827F0E1FBBFF35F8F236803
:107BC0000133236010BD00BF4C5F01201D67012001
:107BD00010B50F4B1A6812B9052025F093FE1A68EC
:107BE000013A1A601B6893B9BFF35F8F094B9A681B
:107BF0006AB1094A127852B9EFF3108072B6074998
:107C00001C680C605C684C609A6000B962B610BD7C
:107C10004C5F01205C5F01201D67012000E100E056
:107C20000C4B1868A8B1C10710D4820710D44307C1
:107C300006D5094B1B78002B14BF03200220704788
:107C400010F4D81F14BF032006207047042070478B
:107C500005207047845F0120806701202DE9F04FE7
:107C6000A04BADF2944D16010190894617460FCBFB
:107C700003AD85E80F0004362A46002352F8044B72
:107C8000D4F800B5BBF1000F10D1D4F8601500296D
:107C90000CDAD4F86415002908DAD4F8681500293C
:107CA00004DAD4F86C150029C0F2B5800133042B36
:107CB000E4D100242546D4E0012231460CF074FCC6
:107CC000C6E00132D20019F800B092B280201BEA5F
:107CD000000F48F20C0E08BFE64625F813E001330A
:107CE0009BB293424FEA5000F1D101318AB2D300E6
:107CF00097429BB21046E4D84FF4004225F8132077
:107D000001339BB2760825F81320B6B20023142263
:107D1000C4F80C35C4F80435C4F80825C4F8143583
:107D2000C4F81035C4F82055C4F82465C4F82835C3
:107D3000C4F82C35019B5B681B79C4F860350125BC
:107D40004FF0FF33C4F864354FF48871C4F86835D8
:107D50002046C4F86C35C4F8005544F093FEA56085
:107D6000D4F810310BB34FF48871204644F08AFEEA
:107D70000023C4F800354FF0FF33C4F86035C4F871
:107D80006435C4F86835C4F86C35002023F02AFB4C
:107D9000043041F10001CAE900010DF2944DBDE843
:107DA000F08F002148F2050CA0E7F8F7E9FDD7E7CE
:107DB00019F802B008214FF0800CD4F804E0AEEBC3
:107DC000030EBEF1460FF8D96368D5F808E51BEA43
:107DD0000C0F4EEA060EC5F808E512D0D4F804E000
:107DE000AEEB030EBEF1280FF8D9D5F80CE501393A
:107DF0004EEA060EC5F80CE54FEA5C0CDDD1013207
:107E00005CE0D4F804E0AEEB030EBEF1110FF8D93C
:107E1000EBE762B6B9E740F284439E4221D9DFF82E
:107E2000D48085F800B0284646F021FCD8F8002020
:107E3000DFF8C4A0B24212D2DAF8FC0008B1C8F8E8
:107E400000B02A78002A3FF437AF31463DF0B9FD43
:107E5000CAF8FC00DAF8FC200AB1C8F80060DAF8C9
:107E6000FC50DFF898A0002023F0BCFADAE90023E8
:107E7000904271EB0303F6D30DB1002C91D172B691
:107E8000019B194C5B6802A81B7902931EF0EAFD66
:107E9000029B164A01269E40D2F8FC3043F08073C4
:107EA000C2F8FC3023684FF4307843F001030546F4
:107EB000236008FB07F800226068134691B28F42E6
:107EC0003FF676AF6268D21A462AFBD963681B1A5E
:107ED00043459ED3064B4FF4964043F00103984729
:107EE000E9E700BF98160800001000E000ED00E090
:107EF000803E0900745F0120505C0120E00A0120EF
:107F00002DE9F04387B00DF1080806460DF1030393
:107F100014481022414644F081FF0446B0B99DF850
:107F20000330E3B9024601A940462AF031FA074678
:107F3000019D95F8009048462EF02EF950B9454520
:107F400002D0B9F1000F08D049F47F44204607B0B1
:107F5000BDE8F08301350195EAE73760F6E74FF6B3
:107F60002274F3E704E10800012910B502460C462B
:107F70000BD9042909D0054905483EF002FA2046EC
:107F80000449BDE810400DF0B7B910BD0A4808001B
:107F90000CDF080071BB0500F7B5044600270DF1A2
:107FA00006000D468DF8067046F061FB9DF8063020
:107FB000E3B10DB9012011E00DF107008DF8077054
:107FC00046F04DFB9DF807606EB1AE4228BF2E46CD
:107FD000F1B2204646F045FB10B1002003B0F0BDE1
:107FE0003444AD1BE5E7F8F7CBFCE2E70D4E4FF468
:107FF0008071304644F046FD012333602544AC4295
:1080000002D101207060E9E7D6F80031002BFBD0E7
:108010004FF48071304644F035FDD6F8083504F849
:10802000013BECE700D0004010B50A4B82699A4250
:1080300004460CD00021C06937F06DFA04201EF010
:1080400019FEE069012137F066FA012010BD002019
:10805000FCE700BFA05D08002DE9F34704460020BF
:108060000D4616469846F4F769FE002802DA00200D
:1080700019F090FB2D4B770043F820400021384643
:108080003DF084FCA06010B9384610F0ABFCDFF87E
:10809000C09099F80070E7B91EF096FDDFF8B4A023
:1080A000CAF8000010B9224819F0A6FB214B224A59
:1080B0001F60224B6946CDE900371EF0F9FFDAF860
:1080C0000000394644F07EFDDAF800301B680122DA
:1080D0001A6099F80030013389F800302B79237148
:1080E00001220023E381A3712382A681E27184F837
:1080F00005806361A3612879FCF75AFB104B207956
:108100001A88ADF800209B780E4A8DF80230694637
:108110001EF024FE0C4B984201D00C48C4E7207995
:108120001EF0D4FD02B0BDE8F08700BFA0460120DC
:1081300075470800705F01204147060004000307EF
:1081400094160800E5D402000000AD0B624608005A
:10815000406701201C61012010B504460079FF280A
:1081600021D01EF091FD20791EF07CFE2046F4F710
:10817000E5FD002802DA002019F00CFB0A4B002272
:1081800043F82020207925F0D3FB084AFF232371F0
:108190001378013BDBB213702BB9054BBDE81040DF
:1081A00018681EF031BD10BDA046012040670120B7
:1081B0001C61012008B5836893B102691279C3F884
:1081C0006025043000F09EF8064A1378013BDBB2CC
:1081D00013702BB9044B1868BDE808401EF014BD9D
:1081E00008BD00BF41670120206101202DE9F04F4B
:1081F00085B000269DF838B004460F469246B14639
:1082000098461BB9022005B0BDE8F08F0DF10D02B4
:108210000DF10E01184603F02DFF0028F2D0BDF835
:108220000E309DF80DC036480193324650F8045B7D
:10823000D5F8001511F001035DD0BBF1000F55D149
:10824000D5F808E5019B9E4550D1D5F80C3563451E
:108250004CD15B4603F5AC7E55F82EE0BEF1FF3FF6
:1082600041D101F001064FFA83F96560002D45D038
:10827000237AE76069F3060323723879FCF798FAEA
:10828000237AC4F814806BF3C7132372E368187958
:1082900044F01CFC63680022C3F8002586B96068BE
:1082A00024F0CCFAC0B225F0A9FC6368BDF80E201A
:1082B0009DF80D10C3F80C15C3F80465C3F8082524
:1082C000237A6268397903F07F0303F5AC732046A3
:1082D00042F8231063680122C3F80025514637F0A5
:1082E000D7FB00208FE70133042BB3D10132042ADE
:1082F0009CD10025B9E799461E46B6E7062082E7DD
:108300001036090070B543680446EBB1C3680F4DE1
:10831000187944F0BFFB6668304624F08FFA217A62
:10832000012301F07F0203FA02F22B5C23EA02032D
:108330002B54002501F07F013046656045F0D7FBE6
:10834000E06837F0BEFBE56070BD00BF306701201C
:1083500008B5072817D8DFE800F01804060A0D0F43
:10836000111445F059FC4FF4567011F081FB074889
:1083700019F068FA0648FBE70648F9E7064819F0DD
:108380003BFA0648FBE70648F9E708BD212A080042
:108390007D4A0800E9460800754708006246080063
:1083A000F92708002DE9F0410446D0F8840030B1E7
:1083B0001EF04EFC1EF028FC0023C4F88430284B2D
:1083C00094F8B7701A6804F11406964204BF0022AC
:1083D0001A60002504F18C08AF4235DC94F8B870BF
:1083E000002504F1AA08AF4234DC04F1B4003CF0EB
:1083F0004DFC04F1B5003CF049FC04F1B6003CF042
:1084000045FC636A93B1304633F035FBA06B18B17D
:1084100037F067FB0023A363E06D18B137F061FB11
:108420000023E365606A08B137F05BFB702200212E
:1084300030463DF0B2FBA06837F053FB0023C4E99F
:108440000033A360BDE8F08108EB05003CF01EFCA2
:108450000135C1E708EB05003CF018FC0135C2E727
:10846000F80A01202DE9F04F012685B0044680F876
:10847000BB60D0F884000D461EF0EAFB1EF06AFED9
:10848000002D00F0838004F1080132462846656023
:10849000019114F06BFC0199606803223EF037F9FA
:1084A000B4F88810002801F1FF3114BFC823482315
:1084B000B140E06823610022314314F061FC04F113
:1084C00014067022002130463DF067FB94F8BD2071
:1084D00094F9BE300AB15B425BB2D4F88490002BB1
:1084E00008BF0123B9F1000F00F0A68294F8B7503D
:1084F000B4F88A8084F87B300627B5FBF7F594F84A
:10850000B87094F8B50094F8B9E094F8B4C094F851
:10851000B61094F8BC20A4F87080052D28BF05255E
:10852000052F28BF0527002BB8BF5B4284F8765083
:1085300005EB4505DBB26D0013FB08F3EDB24FF020
:10854000000884F84800C4F81490A4F8723084F845
:1085500079E084F8777084F875C084F8581084F84E
:108560007C20C4F85C80C4F83880284637F0AEFA26
:10857000606218BB02252046FFF714FF022D00F0B1
:108580005582032D00F04F8245F046FBA06837F07E
:10859000A8FA606A37F0A5FAE06D37F0A2FAA06B8E
:1085A00037F09FFAB4F88800656037F08FFAB4F8B6
:1085B0008830E360C823A060236180E7380137F08A
:1085C00085FA8146E06500285AD004F18C01606A82
:1085D0002A463DF0A2FA04F1AA014346DAB29742D4
:1085E00046D8C14BD4F884001E601EF031FBBF4A50
:1085F000BF491EF05DFD636A002BBBD094F8753057
:10860000039303A81EF02EFA002580462F464FF054
:10861000010994F876105FFA85FA01EB4103BAEB91
:10862000430F33DB17F07F4F14BF0823002317F4E9
:108630007F0F18BF43F00403FAB217F47F4F18BF3F
:1086400043F002030AB143F00103013B01250B2B68
:1086500000F23981DFE813F02F002F0033012F00E3
:108660003701370137012F00370137013701330157
:10867000E26D11F8010B02EB031201331073ADE749
:10868000606A37F02EFAC4F8249073E7636A03A88F
:1086900013F80A3003931EF0E5F9804505F1010552
:1086A00040F0CC81636A13F80A3003F01F0309FA23
:1086B00003F31F43ADE784F8745094F8773094F8CF
:1086C000792094F8740005FA03F3B4F8725084F832
:1086D0007A300735DBB205F4FF655D43554394F806
:1086E0007C304543256603B16D0011FB00F1062087
:1086F00000FB015037F0EAF90346A06300283FF47D
:1087000039AF2B44A3622A4600213DF046FA94F883
:10871000740094F87530012840F0EC80626A03F030
:108720001F03127800FA03F3C2F3C102E3623B4372
:10873000236384F87820002394F876205F1C02EBF2
:108740004202DBB2B3EB420FC0F2BF8094F8791063
:1087500094F87A204FF47A43B3FBF2F301228A4073
:10876000013AB3FBF2F3632B40F20A81A366A36ED6
:108770006366002594F8483084F87E5003A803937C
:108780001EF070F900F5A16094F84830E06303A88A
:1087900003931EF067F994F84830012703F01F0394
:1087A00007FA03F300F20C502064636403A894F802
:1087B000583003931EF056F900F5A16094F8583034
:1087C000E06403A803931EF04DF994F8583003F0C9
:1087D0001F039F4000F20C5094F8753020656765C8
:1087E00003A803931EF03EF9039B03F5E07340F2E8
:1087F000033740F8237094F8750044F088F994F832
:108800004830039303A81EF02DF9039B03F5E07392
:1088100040F8237094F8480044F079F994F85830FF
:10882000039303A81EF01EF9039B03F5E07340F8C1
:10883000237094F8580044F094F994F8763005F1D8
:10884000010803EB4303EDB2B5EB430FC0F29A808E
:1088500094F87730012505FA03F3023BDBB284F884
:1088600081300027A84640F2033994F87720FBB204
:108870009A4200F2988094F87530039303A81EF092
:10888000F1F800F5A16094F87530A06103A8039396
:108890001EF0E8F800F20C50E0613046F2F776FF87
:1088A000B4F88A20A168304632F0E6FD304633F055
:1088B0001BF9002384F8BB3005B0BDE8F08F02231C
:1088C00084F87430F9E60423FAE7D4E90921D25C8C
:1088D00094F8785002F01F0200FA02F2ED00EA402C
:1088E000CA543B4628E700BFF80A01207DDC05009A
:1088F0005856090003F01F03012101FA03F302286F
:1089000047EA030721D1626A1278C2F30012C4E970
:108910000B3784F87820002394F876205F1C02EB54
:108920004202DBB2B3EB420FBFF610AFD4E909202D
:10893000D25C94F8785002F01F0201FA02F22D0185
:10894000EA4020F813203B46E6E70022C4E90B3753
:1089500084F87820134694F876205D1C02EB4202DE
:10896000DBB2B3EB420FBFF6F1AED4E90920D25C23
:1089700002F01F0201FA02F240F823202B46EAE738
:108980006423F3E6636A03A85B5D03931EF06AF851
:10899000039B03F5E07340F82370636A585D44F06D
:1089A000B6F8454649E7D4F85CB04FEA031A0BEB3A
:1089B000031303A81B7B03931EF054F800F5A1607A
:1089C0004BF80A00E36D03EB0A0B03A89BF80C308D
:1089D00003931EF047F800F20C50CBF80400E26D50
:1089E000524403A8137B03F01F0308FA03F39360B8
:1089F000E36D53441B7B03931EF034F8039B03F594
:108A0000E07340F8239094F881302B42E36D534497
:108A1000187B05D044F0A5F86D00EDB2013724E7CE
:108A200044F075F8F8E73D2011F022F804490548B4
:108A300040F2E9123EF05EFF03259CE501259AE530
:108A400079290800D41B0800F7B501711379437127
:108A5000194B43F821001646427943F82200174B80
:108A60001A88ADF804209B78154A8DF80630044624
:108A70000D46007901A91EF071F9124B9842074684
:108A800002D0114818F0B8FE0D4A607901A91EF015
:108A900065F9B842207902D01EF0E4F9F1E71EF042
:108AA00015F960791EF012F92846FBF781FE30793E
:108AB000FBF77EFE03B0F0BDC0460120EE160800B5
:108AC000E5CD02000000AD0B6246080010B501794B
:108AD000FF2904461BD00E4B002243F82120417988
:108AE00043F8212000791EF0CFF860791EF0CCF811
:108AF00020791EF0B7F960791EF0B4F9207924F0DE
:108B000017FF607924F014FF4FF6FF73A38010BDA8
